:020000040800F2
:1000000000060020E1020008E3020008E302000805
:10001000E3020008E3020008E3020008E30200082C
:10002000E3020008E3020008E30200089920000848
:10003000E3020008E3020008E3020008E30200080C
:10004000E3020008E3020008E3020008E3020008FC
:10005000E3020008E3020008652400089124000878
:10006000BD240008E924000815250008E302000863
:10007000E3020008E3020008E3020008E3020008CC
:10008000E3020008E3020008E3020008E3020008BC
:10009000E3020008E3020008E3020008412500082B
:1000A000E3020008E3020008E3020008E30200089C
:1000B000E3020008E3020008E3020008E30200088C
:1000C000E3020008E3020008E3020008E30200087C
:1000D000E3020008E3020008E3020008E30200086C
:1000E000A5250008E3020008E3020008E302000877
:1000F000E3020008E3020008E3020008E30200084C
:10010000E3020008E302000841260008E3020008B9
:10011000E3020008E3020008E3020008E30200082B
:10012000E3020008E3020008E3020008E30200081B
:10013000E3020008E3020008E3020008E30200080B
:10014000E3020008E3020008E3020008E3020008FB
:10015000E3020008E3020008E3020008E3020008EB
:10016000E3020008E3020008E3020008E3020008DB
:10017000E3020008E3020008E3020008E3020008CB
:10018000E3020008E3020008192600082D260008F3
:10019000E3020008E3020008E3020008E3020008AB
:1001A000E3020008E3020008E3020008E30200089B
:1001B000E3020008E3020008E3020008E30200088B
:1001C000E3020008E3020008E3020008E30200087B
:1001D000E3020008E3020008E3020008E30200086B
:1001E000E3020008E3020008E3020008E30200085B
:1001F000E3020008E3020008E3020008E30200084B
:10020000E3020008E3020008E3020008E30200083A
:10021000E3020008E3020008E3020008E30200082A
:10022000E3020008E3020008E3020008E30200081A
:10023000E3020008E3020008E3020008E30200080A
:10024000E3020008E3020008E3020008E3020008FA
:10025000E3020008E3020008E3020008E3020008EA
:10026000E3020008E3020008E3020008E3020008DA
:10027000E3020008E3020008E3020008E3020008CA
:10028000E3020008E3020008E3020008E3020008BA
:10029000E3020008E3020008E3020008E3020008AA
:1002A000E3020008E3020008E3020008E30200089A
:1002B000E3020008E3020008E3020008E30200088A
:1002C000E3020008E3020008E3020008E30200087A
:1002D000E3020008E3020008E3020008E30200086A
:1002E00002E000F000F8FEE772B6384880F30888B4
:1002F000374880F3098837483749086040F20000E2
:10030000CCF200004EF63471CEF200010860BFF36B
:100310004F8FBFF36F8F40F20000C0F2F0004EF637
:100320008851CEF200010860BFF34F8FBFF36F8F8B
:100330004FF00000E1EE100A4EF63C71CEF20001E3
:100340000860062080F31488BFF36F8F01F086FDEC
:1003500001F028FD01F0FCFD4FF055301F491B4A0C
:1003600091423CBF41F8040BFAE71D49184A9142FB
:100370003CBF41F8040BFAE71A491B4A1B4B9A424F
:100380003EBF51F8040B42F8040BF8E7002018496F
:10039000184A91423CBF41F8040BFAE701F040FDD6
:1003A00001F058FE144C154DAC4203DA54F8041B0E
:1003B0008847F9E700F042F8114C124DAC4203DADD
:1003C00054F8041B8847F9E701F028BD0006002017
:1003D000002200200000000808ED00E000000020DE
:1003E00000060020F0280008002200203022002013
:1003F00030220020702F0020E0020008E0020008F8
:10040000E0020008E00200082DE9F04F2DED108A0F
:10041000C1F80CD0D0F80CD0BDEC108ABDE8F08F3C
:10042000002383F311882846A047002001F08CF9AF
:10043000FEE701F0FFF800DFFEE7000038B501F04D
:1004400071FC054601F0A4FC0446D0B90F4B9D4257
:1004500019D001339D4242F2107512BF04460025A7
:100460000124002001F068FC0CB100F077F800F0E6
:1004700025FD00F0EDFB284600F0F0F800F06EF8E6
:10048000F9E70025EDE70546EBE700BF010007B0FF
:1004900008B500F0A9FBA0F120035842584108BD5F
:1004A00007B541F21203022101A8ADF8043000F0B3
:1004B000B9FB03B05DF804FB38B5302383F3118832
:1004C000174803680BB101F0FDF90023154A4FF4FA
:1004D0007A71134801F0ECF9002383F31188124C70
:1004E000236813B12368013B2360636813B1636819
:1004F000013B63600D4D2B7833B963687BB90220F3
:1005000000F072FC322363602B78032B07D1636801
:100510002BB9022000F068FC4FF47A73636038BD99
:1005200030220020B9040008502300204822002077
:10053000084B187003280CD8DFE800F00805020803
:10054000022000F047BC022000F03ABC024B00221F
:100550005A6070474822002050230020F8B5394BDC
:10056000394A1C46196801316BD004339342F9D1E2
:100570006268364B9A4264D9354B9B6803F100633D
:1005800003F500339A425CD2002000F087FB022082
:10059000FFF7CEFF2F4B00219A6C99641A6F1967F1
:1005A0001A6FDA6CD9645A6F59675A6F1A6D1965E8
:1005B0009A6F99679B6F72B64FF0E023C3F8084DAE
:1005C000D4E90004BFF34F8FBFF36F8F224AC2F804
:1005D0008410BFF34F8F536923F480335361BFF30B
:1005E0004F8FD2F8803043F6E076C3F3C905C3F3EA
:1005F0004E335B0103EA060C29464CEA8177013948
:10060000C2F87472F9D2203B13F1200FF2D1BFF37C
:100610004F8FBFF36F8FBFF34F8FBFF36F8F536950
:1006200023F4003353610023C2F85032BFF34F8FDD
:10063000BFF36F8F302383F31188854680F30888DA
:100640002047F8BD0000020820000208FFFF010853
:10065000002200200045025800ED00E02DE9F04F97
:1006600093B0B44B2022FF2100900AA89D6800F0AF
:10067000CFFBB14A1378A3B90121B04811700360D0
:10068000302383F3118803680BB101F01BF90023B9
:10069000AB4A4FF47A71A94801F00AF9002383F3B9
:1006A0001188009B13B1A74B009A1A60A64A1378D1
:1006B000032B03D000231370A24A53604FF0000AAB
:1006C000009CD3465646D146012000F083FB24B15E
:1006D0009C4B1B68002B00F02682002000F084FA5F
:1006E0000390039B002BF2DB012000F069FB039BCE
:1006F000213B1F2BE8D801A252F823F07D07000808
:10070000A507000839080008C9060008C90600083E
:10071000C9060008CB0800089B0A0008B5090008B4
:10072000170A00083F0A0008650A0008C906000801
:10073000770A0008C9060008E90A00081D08000831
:10074000C90600082D0B0008890700081D080008CD
:10075000C9060008170A0008C9060008C9060008EB
:10076000C9060008C9060008C9060008C90600082D
:10077000C9060008C9060008390800080220FFF76A
:1007800087FE002840F0F981009B022105A8BAF1FC
:10079000000F08BF1C4641F21233ADF8143000F0D0
:1007A00041FA91E74FF47A7000F01EFA071EEBDB76
:1007B0000220FFF76DFE0028E6D0013F052F00F272
:1007C000DE81DFE807F0030A0D101336052304214C
:1007D00005A8059300F026FA17E004215548F9E72B
:1007E00004215A48F6E704215948F3E74FF01C0862
:1007F000404608F1040800F053FA0421059005A8CA
:1008000000F010FAB8F12C0FF2D101204FF00009DE
:1008100000FA07F747EA0B0B5FFA8BFB00F044FB8B
:1008200026B10BF00B030B2B08BF0024FFF738FE9B
:100830004AE704214748CDE7002EA5D00BF00B0373
:100840000B2BA1D10220FFF723FE074600289BD0E7
:100850000120002600F022FA0220FFF769FE5FFA6D
:1008600086F8404600F02AFA0446B0B103994046A3
:100870000136A1F140025142514100F02FFA002807
:10088000EDD1BA46044641F21213022105A83E46B4
:10089000ADF8143000F0C6F916E725460120FFF741
:1008A00047FE244B9B68AB4207D9284600F0F8F975
:1008B000013040F067810435F3E70025224BBA464A
:1008C0003E461D701F4B5D60A8E7002E3FF45CAFF5
:1008D0000BF00B030B2B7FF457AF0220FFF728FE22
:1008E000322000F081F9B0F10008FFF64DAF18F0AA
:1008F00003077FF449AF0F4A08EB05039268934260
:100900003FF642AFB8F5807F3FF73EAF124BB84598
:10091000019323DD4FF47A7000F066F90390039A97
:10092000002AFFF631AF039A0137019B03F8012B30
:10093000EDE700BF002200204C23002030220020E1
:10094000B90400085023002048220020042200207F
:10095000082200200C2200204C220020C820FFF793
:1009600097FD074600283FF40FAF1F2D11D8C5F1A2
:1009700020020AAB25F0030084494245184428BFF1
:100980004246019200F03AFA019AFF217F4800F0B6
:100990003FFA4FEAA803C8F387027C49284601932F
:1009A00000F03EFA064600283FF46DAF019B05EBD0
:1009B000830533E70220FFF76BFD00283FF4E4AE28
:1009C00000F0AAF900283FF4DFAE0027B846704BCC
:1009D0009B68BB4218D91F2F11D80A9B01330ED038
:1009E00027F0030312AA134453F8203C0593404612
:1009F000042205A9043700F089FA8046E7E7384663
:100A000000F04EF90590F2E7CDF81480042105A816
:100A100000F008F902E70023642104A8049300F021
:100A2000F7F800287FF4B0AE0220FFF731FD002870
:100A30003FF4AAAE049800F065F90590E6E70023BC
:100A4000642104A8049300F0E3F800287FF49CAE2E
:100A50000220FFF71DFD00283FF496AE049800F039
:100A600053F9EAE70220FFF713FD00283FF48CAEAC
:100A700000F062F9E1E70220FFF70AFD00283FF4E9
:100A800083AE05A9142000F05DF907460421049007
:100A900004A800F0C7F83946B9E7322000F0A4F8FE
:100AA000071EFFF671AEBB077FF46EAE384A07EB48
:100AB0000903926893423FF667AE0220FFF7E8FC15
:100AC00000283FF461AE27F003074F44B9453FF4D7
:100AD000A5AE484609F1040900F0E2F804210590AA
:100AE00005A800F09FF8F1E74FF47A70FFF7D0FC0B
:100AF00000283FF449AE00F00FF9002844D00A9BCB
:100B000001330BD008220AA9002000F089F900283F
:100B10003AD02022FF210AA800F07AF9FFF7C0FCA2
:100B20001C4800F017FE13B0BDE8F08F002E3FF414
:100B30002BAE0BF00B030B2B7FF426AE00236421AE
:100B400005A8059300F064F8074600287FF41CAE62
:100B50000220FFF79DFC804600283FF415AEFFF70A
:100B60009FFC41F2883000F0F5FD059800F0B4F9E3
:100B700046463C4600F098F9A6E506464EE64FF09C
:100B8000000901E6BA467EE637467CE64C220020A4
:100B900000220020A0860100104B70B51B780C4687
:100BA0000133DBB2012B12D80D4B1D684FF47A7361
:100BB0002968A2FB033222460E6A01462846B04746
:100BC000844204D1074B002201201A7070BD4FF4FB
:100BD000FA7000F0BFFD0020F8E700BF10220020EF
:100BE000142200209C230020002307B50246012187
:100BF0000DF107008DF80730FFF7CEFF20B19DF80B
:100C0000070003B05DF804FB4FF0FF30F9E7000088
:100C10000A46042108B5FFF7BFFF80F00100C0B20B
:100C2000404208BD074B0A4630B41978064B53F8CA
:100C30002140014623682046DD69044BAC4630BCA8
:100C4000604700BF9C23002014220020A0860100E2
:100C500070B5104C0025104E00F03CFF208030682D
:100C6000238883420CD800252088013800F02EFF0D
:100C700023880544013BB5F5802F2380F4D370BD54
:100C800000F024FF336805440133B5F5003F3360BD
:100C9000E5D3E8E79E2300205823002000F0F8BFAA
:100CA00000F1006000F500300068704700F100605E
:100CB000920000F5003000F06FBF0000054B1A688D
:100CC000054B1B889B1A834202D9104400F0FEBEDC
:100CD00000207047582300209E23002038B504468A
:100CE000074D29B128682044BDE8384000F006BF10
:100CF0002868204400F0F0FE0028F3D038BD00BF83
:100D0000582300200020704700F1FF5000F58F109D
:100D1000D0F8000870470000064991F8243033B13C
:100D200000230822086A81F82430FFF7BFBF0120A2
:100D3000704700BF5C230020014B1868704700BF5C
:100D40000010005C1B4B0246F0B518681A4BC0F34C
:100D50000B06000C1F885C68BE4293F9085003D054
:100D60009F89BE4203D10C335C6893F90850042676
:100D7000124B1F880433874208BF13F9025C013EFF
:100D8000F7D1013A013C0B460A44934207D214F9C9
:100D9000016F581C2EB1034600F8016CF5E71846A8
:100DA00005E02C2482421C7001D9981C5D70401A09
:100DB000F0BD00BF0010005C182200205027000882
:100DC000022803D1024B4FF080629A61704700BF46
:100DD000000C0258022803D1024B4FF480629A6142
:100DE000704700BF000C0258022804D1024A536920
:100DF00083F4806353617047000C0258002310B5E0
:100E0000934203D0CC5CC4540133F9E710BD000019
:100E100002440346934202D003F8011BFAE77047ED
:100E20002DE9F8431F4D14460746884695F82420BF
:100E300052BBDFF870909CB395F824302BB9202278
:100E4000FF2148462F62FFF7E3FF95F82400414653
:100E5000C0F1080205EB8000A24228BF2246D6B2AC
:100E60009200FFF7CBFF95F82430A41B17441E44D3
:100E70009044E4B2F6B2082E85F82460DBD1FFF787
:100E80004BFF0028D7D108E02B6A03EB8203834293
:100E9000CFD0FFF741FF0028CBD10020BDE8F88379
:100EA0000120FBE75C230020024B1A78024B1A70EA
:100EB000704700BF9C23002010220020034B0449F0
:100EC0000B60044B186800F01BBB00BF80841E0041
:100ED0008423002014220020094B1822002110B581
:100EE00004461846FFF794FF064A074B014612785E
:100EF000046053F82200BDE8104000F001BB00BFC1
:100F0000842300209C2300201422002030B50A44B2
:100F1000084D91420DD011F8013B5840082340F391
:100F20000004013B2C4013F0FF0384EA5000F6D18B
:100F3000EFE730BD2083B8ED0268436811430160DC
:100F400003B1184770470000024A136843F0C0031A
:100F50001360704700780040024A136843F0C003F2
:100F600013607047007C004037B51A4C1A4D20467C
:100F700000F0BAFA04F11400009400234FF4007258
:100F8000164900F077F94FF40072154904F1380062
:100F90000094144B00F0F0F9134BC4E91735134CCF
:100FA000204600F0A1FA04F1140000234FF400726F
:100FB0000F49009400F05EF90E4B4FF400720E4999
:100FC00004F13800009400F0D7F90C4BC4E9173550
:100FD00003B030BDA023002000E1F50578240020F7
:100FE00078280020490F0008007800400C240020D9
:100FF00078260020590F0008782A0020007C004045
:10100000037C30B5274C002918BF0C46012B0CD1AE
:10101000254B984236D1254B9A6C42F080429A6417
:101020001A6F42F080421A671B6F2268036EC16D0F
:1010300003EB52038466B3FBF2F36268150442BF0C
:1010400023F0070503F0070343EA4503CB60A368D9
:1010500043F040034B60E36843F001038B6042F4CC
:10106000967343F001030B604FF0FF330B625105A1
:1010700005D512F0102211D0B2F1805F10D080F8A7
:10108000643030BD0A4B9842CFD1084B9A6C42F085
:1010900000429A641A6F42F00042C4E77F23EEE7F1
:1010A0003F23ECE760270008A023002000450258FA
:1010B0000C2400202DE9F047C66D05463768F46919
:1010C000210734621AD014F0080118BF4FF4807160
:1010D000E20748BF41F02001A3074FF0300348BFAB
:1010E00041F04001600748BF41F0800183F311885F
:1010F000281DFFF721FF002383F31188E2050AD59D
:10110000302383F311884FF48061281DFFF714FF0B
:10111000002383F311884FF030094FF0000A14F0D8
:10112000200838D13B0616D54FF0300905F1380AB2
:10113000200610D589F31188504600F051F9002897
:1011400036DA0821281DFFF7F7FE27F08003336009
:10115000002383F31188790614D5620612D5302353
:1011600083F31188D5E913239A4208D12B6C33B14C
:1011700027F040071021281DFFF7DEFE376000230F
:1011800083F31188E30618D5AA6E1369ABB15069D1
:10119000BDE8F047184789F31188736A284695F827
:1011A0006410194000F0BAF98AF31188F469B6E7BF
:1011B000B06288F31188F469BAE7BDE8F0870000EF
:1011C000F8B51546826804460B46AA4200D28568E7
:1011D000A1692669761AB5420BD218462A46FFF74E
:1011E0000DFEA3692B44A3612846A3685B1BA36083
:1011F000F8BD0CD9AF1B18463246FFF7FFFD3A4643
:10120000E1683044FFF7FAFDE3683B44EBE718463A
:101210002A46FFF7F3FDE368E5E7000083689342A1
:10122000F7B50446154600D28568D4E90460361A3D
:10123000B5420BD22A46FFF7E1FD63692B44636197
:101240002846A3685B1BA36003B0F0BD0DD93246EE
:10125000AF1B0191FFF7D2FD01993A46E068314496
:10126000FFF7CCFDE3683B44E9E72A46FFF7C6FDFC
:10127000E368E4E710B50A440024C361029B84607C
:10128000C16002610362C0E90000C0E9051110BD40
:1012900008B5D0E90532934201D1826882B98268EB
:1012A000013282605A1C426119700021D0E9043277
:1012B0009A4224BFC368436100F068FA002008BD69
:1012C0004FF0FF30FBE7000070B5302304460E46B8
:1012D00083F31188A568A5B1A368A269013BA36047
:1012E000531CA36115782269934224BFE368A3616C
:1012F000E3690BB120469847002383F31188284601
:1013000007E03146204600F031FA0028E2DA85F3A2
:10131000118870BD2DE9F74F04460E4617469846D2
:10132000D0F81C904FF0300A8AF311884FF0000B70
:10133000154665B12A4631462046FFF741FF034670
:1013400060B94146204600F011FA0028F1D0002390
:1013500083F31188781B03B0BDE8F08FB9F1000F5B
:1013600003D001902046C847019B8BF31188ED1AEA
:101370001E448AF31188DCE7C160C361009B826070
:101380000362C0E905111144C0E900000161704722
:10139000F8B504460D461646302383F31188A76836
:1013A000A7B1A368013BA36063695A1C62611D7009
:1013B000D4E904329A4224BFE3686361E3690BB164
:1013C00020469847002080F3118807E031462046E8
:1013D00000F0CCF90028E2DA87F31188F8BD0000AC
:1013E000D0E9052310B59A4201D182687AB98268A2
:1013F0000021013282605A1C82611C7803699A4282
:1014000024BFC368836100F0C1F9204610BD4FF0CE
:10141000FF30FBE72DE9F74F04460E461746984686
:10142000D0F81C904FF0300A8AF311884FF0000B6F
:10143000154665B12A4631462046FFF7EFFE0346C2
:1014400060B94146204600F091F90028F1D0002310
:1014500083F31188781B03B0BDE8F08FB9F1000F5A
:1014600003D001902046C847019B8BF31188ED1AE9
:101470001E448AF31188DCE7026843681143016067
:1014800003B11847704700001430FFF743BF000056
:101490004FF0FF331430FFF73DBF00003830FFF747
:1014A000B9BF00004FF0FF333830FFF7B3BF000083
:1014B0001430FFF709BF00004FF0FF311430FFF781
:1014C00003BF00003830FFF763BF00004FF0FF326A
:1014D0003830FFF75DBF0000012914BF6FF0130023
:1014E00000207047FFF740BD044B036000234360BA
:1014F000C0E9023301230374704700BF7827000856
:1015000010B53023044683F31188FFF779FD0223D9
:101510000020237480F3118810BD000038B5C36922
:1015200004460D461BB904210844FFF7A5FF2946D0
:1015300004F11400FFF7ACFE002806DA201D4FF47A
:101540000061BDE83840FFF797BF38BD00238268CF
:10155000037503691B6899689142FBD25A6803605E
:101560004260106058607047002382680375036909
:101570001B6899689142FBD85A680360426010600A
:101580005860704708B50846302383F311880B7DF7
:10159000032B05D0042B0DD02BB983F3118808BD84
:1015A0008B6900221A604FF0FF338361FFF7CEFF93
:1015B0000023F2E7D1E9003213605A60F3E700003C
:1015C000FFF7C4BF054BD9680875186802685360F7
:1015D0001A600122D8600275FEF716BF782C002031
:1015E0000C4B30B5DD684B1C87B004460FD02B4642
:1015F000094A684600F05CF92046FFF7E3FF009BCC
:1016000013B1684600F05EF9A86907B030BDFFF776
:10161000D9FFF9E7782C002085150008044B1A68DB
:10162000DB6890689B68984294BF00200120704757
:10163000782C0020084B10B51C68D86822685360CD
:101640001A600122DC602275FFF78EFF01462046FA
:10165000BDE81040FEF7D8BE782C0020044B1A6875
:10166000DB6892689B689A4201D9FFF7E3BF704735
:10167000782C002038B5074C01230025064907487F
:101680002370656000F00CFC0223237085F3118841
:1016900038BD00BFE02E0020A4270008782C0020D1
:1016A00000F046B9EFF3118020B9EFF30583302243
:1016B00082F311887047000010B530B9EFF305844C
:1016C000C4F3080414B180F3118810BDFFF7C6FFFE
:1016D00084F31188F9E700008B6002230861084653
:1016E0008B8270478368A3F1840243F8142C02694B
:1016F00043F8442C426943F8402C094A43F8242C0F
:10170000C268A3F1200043F8182C022203F80C2C25
:10171000002203F80B2C034A43F8102C704700BF3B
:1017200021040008782C002008B5FFF7DBFFBDE896
:101730000840FFF745BF0000024BDB6898610F20AF
:10174000FFF740BF782C0020302383F31188FFF788
:10175000F3BF000008B50146302383F31188082049
:10176000FFF73EFF002383F3118808BD064BDB68BB
:1017700039B1426818605A60136043600420FFF773
:101780002FBF4FF0FF307047782C0020036898423D
:1017900006D01A680260506018469961FFF710BFC2
:1017A00070470000036810B59C68A2420CD85C68C2
:1017B0008A600B604C602160596099688A1A9A604F
:1017C0004FF0FF33836010BD121B1B68ECE7000075
:1017D0000A2938BF0A2170B504460D460A26601949
:1017E00000F056FB00F03EFB041BA54203D8751C1D
:1017F00004462E46F3E70A2E04D90120BDE87040C6
:1018000000F08EBB70BD0000F8B5144B0D460A2ADF
:101810004FF00A07D96103F11001826038BF0A2234
:10182000416019691446016048601861A81800F009
:101830001FFB00F017FB431B0646A34206D37C1C8C
:1018400028192746354600F023FBF2E70A2F04D972
:101850000120BDE8F84000F063BBF8BD782C002003
:10186000F8B506460D4600F0FDFA0F4A134653F848
:10187000107F9F4206D12A4601463046BDE8F84017
:10188000FFF7C2BFD169BB68441A2C1928BF2C4688
:10189000A34202D92946FFF79BFF2246314603485F
:1018A000BDE8F840FFF77EBF782C0020882C002090
:1018B000C0E90323002310B45DF8044B4361FFF734
:1018C000CFBF000010B5194C236998420DD0816834
:1018D000D0E9003213605A609A680A449A60002383
:1018E00003604FF0FF33A36110BD0268234643F845
:1018F000102F53600022026022699A4203D1BDE892
:10190000104000F0BFBA936881680B44936000F008
:10191000A9FA2269E1699268441AA242E4D9114401
:10192000BDE81040091AFFF753BF00BF782C002014
:101930002DE9F047DFF8BC8008F110072C4ED8F8ED
:10194000105000F08FFAD8F81C40AA68031B9A4286
:101950003ED814444FF00009D5E90032C8F81C40C5
:1019600013605A60C5F80090D8F81030B34201D126
:1019700000F088FA89F31188D5E9033128469847A1
:10198000302383F311886B69002BD8D000F06AFAFA
:101990006A69A0EB040982464A450DD2022000F094
:1019A000BFFA0022D8F81030B34208D15146284679
:1019B000BDE8F047FFF728BF121A2244F2E712EB06
:1019C00009092946384638BF4A46FFF7EBFEB5E716
:1019D000D8F81030B34208D01444C8F81C00211ABB
:1019E000A960BDE8F047FFF7F3BEBDE8F08700BF90
:1019F000882C0020782C002000207047FEE7000093
:101A0000704700004FF0FF3070470000BFF34F8F6A
:101A1000044B1A695107FCD1D3F810215207F8D1B1
:101A2000704700BF0020005208B50D4B1B78ABB9C2
:101A3000FFF7ECFF0B4BDA68D10704D50A4A5A606E
:101A400002F188325A60D3F80C21D20706D5064A33
:101A5000C3F8042102F18832C3F8042108BD00BF95
:101A6000E82E0020002000522301674508B5114BE5
:101A70001B78F3B9104B1A69510703D5DA6842F0A5
:101A80004002DA60D3F81021520705D5D3F80C21B3
:101A900042F04002C3F80C21FFF7B8FF064BDA68AA
:101AA00042F00102DA60D3F80C2142F00102C3F8DF
:101AB0000C2108BDE82E0020002000520F289ABFFC
:101AC00000F5806040040020704700004FF40030B3
:101AD00070470000102070470F2808B50BD8FFF79B
:101AE000EDFF00F500330268013204D10430834277
:101AF000F9D1012008BD0020FCE700000F2870B5D7
:101B0000054645D8FFF7CEFD224CFFF77FFF06467E
:101B1000FFF78AFF4FF0FF33072D6361C4F81431DC
:101B200020D82361FFF772FF2B0243F02403E36008
:101B3000E36843F08003E36023695A07FCD4284636
:101B4000FFF764FF4FF40031FFF7B8FF00F002F930
:101B50003046FFF78BFFFFF7AFFD2846BDE870402A
:101B6000FFF7BABFC4F81031FFF750FFA5F1080323
:101B70001B0243F02403C4F80C31D4F80C3143F0B9
:101B80008003C4F80C31D4F810315B07FBD4D6E7DE
:101B9000002070BD002000522DE9F84F40EA0203FA
:101BA00005460C461746D80602D00020BDE8F88F3F
:101BB00027F01F07DFF8D4B0FFF736FF2744BC42F9
:101BC00003D10120FFF752FFF0E7202229462046EB
:101BD00000F0A0FD10B920352034F0E72B4605F1C8
:101BE00020021E68711CE0D104339A42F9D1FFF73C
:101BF00059FD05F17843234AB3F5801F224B28BFD6
:101C00009A4603F1040338BF9046A2F1080228BFA8
:101C10009846A3F108033ABF9146DA469946FFF782
:101C2000F5FEC8F80060A5EB040CD9F8002004F11B
:101C30001C0142F00202C9F80020221FDAF80060FD
:101C400016F00506FAD152F8043F8A424CF80230E9
:101C5000F4D1BFF34F8FFFF7D9FE4FF0FF32C8F832
:101C60000020D9F8002022F00202C9F80020FFF776
:101C700023FD20222146284600F04CFD0028AAD052
:101C800030469FE7142000521021005210200052CD
:101C900010B5084C237828B11BB9FFF7C5FE012306
:101CA000237010BD002BFCD02070BDE81040FFF762
:101CB000DDBE00BFE82E00200244074BD2B210B5B3
:101CC000904200D110BD441C00B253F8200041F8EE
:101CD000040BE0B2F4E700BF504000580E4B30B5A3
:101CE0001C6F240405D41C6F1C671C6F44F4004453
:101CF0001C670A4C02442368D2B243F48073236009
:101D0000074B904200D130BD441C51F8045B00B237
:101D100043F82050E0B2F4E700440258004802586B
:101D20005040005807B5012201A90020FFF7C4FF69
:101D3000019803B05DF804FB13B50446FFF7F2FF0A
:101D4000A04205D0012201A900200194FFF7C6FF9F
:101D500002B010BD0144BFF34F8F064B884204D33D
:101D6000BFF34F8FBFF36F8F7047C3F85C02203013
:101D7000F4E700BF00ED00E0034B1A681AB9034A0C
:101D8000D2F8D0241A607047EC2E00200040025890
:101D900008B5FFF7F1FF024B1868C0F3806008BD7B
:101DA000EC2E002070B5BFF34F8FBFF36F8F1A4A30
:101DB0000021C2F85012BFF34F8FBFF36F8F5369EA
:101DC00043F400335361BFF34F8FBFF36F8FC2F8FB
:101DD0008410BFF34F8FD2F8803043F6E074C3F322
:101DE000C900C3F34E335B0103EA0406014646EA29
:101DF00081750139C2F86052F9D2203B13F1200FEE
:101E0000F2D1BFF34F8F536943F480335361BFF373
:101E10004F8FBFF36F8F70BD00ED00E0FEE7000055
:101E20000A4B0B480B4A90420BD30B4BC11EDA1CDA
:101E3000121A22F003028B4238BF00220021FEF763
:101E4000E7BF53F8041B40F8041BECE72029000807
:101E5000702F0020702F0020702F0020704700008E
:101E600000F07CB9014B586A704700BF000C00407D
:101E7000034B002258631A610222DA60704700BFE8
:101E8000000C0040014B0022DA607047000C00405B
:101E9000014B5863704700BF000C0040FEE7000094
:101EA00070B51B4B0025044686B058600E4685620F
:101EB000016300F001F904F11003A560E562C4E9D3
:101EC00004334FF0FF33C4E90044C4E90635FFF79B
:101ED000C9FF2B46024604F134012046C4E9082319
:101EE00080230C4A2565FFF7F7FB01230A4AE060CF
:101EF00000920375684672680192B268CDE90223C8
:101F0000064BCDE90435FFF70FFC06B070BD00BFEE
:101F1000E02E0020B0270008B52700089D1E00080D
:101F2000024AD36A1843D062704700BF782C002061
:101F30004B6843608B688360CB68C3600B69436107
:101F40004B6903628B6943620B6803607047000052
:101F500008B53A4B40F2FF713948D3F888200A435C
:101F6000C3F88820D3F8882022F4FF6222F0070209
:101F7000C3F88820D3F88830324B1A6C0A431A64AD
:101F80009A6E0A439A66304A9B6E1146FFF7D0FF5D
:101F900000F5806002F11C01FFF7CAFF00F58060C8
:101FA00002F13801FFF7C4FF00F5806002F154012F
:101FB000FFF7BEFF00F5806002F17001FFF7B8FF88
:101FC00000F5806002F18C01FFF7B2FF00F5806040
:101FD00002F1A801FFF7ACFF00F5806002F1C40137
:101FE000FFF7A6FF00F5806002F1E001FFF7A0FF18
:101FF00000F5806002F1FC01FFF79AFF02F58C7199
:1020000000F58060FFF794FF00F066F90F4BD3F8FE
:10201000902242F00102C3F89022D3F8942242F0B9
:102020000102C3F894220522C3F898204FF06052B1
:10203000C3F89C20064AC3F8A02008BD00440258FB
:102040000000025800450258BC27000800ED00E0DF
:102050001F00080308B500F041FBFFF70BFB0B4B1B
:10206000DA6B42F04002DA635A6E22F040025A669E
:102070005B6E074B1A6842F008021A601A6842F059
:1020800004021A60BDE80840FFF776BE004502581A
:102090000018024870470000EFF3098305496833D0
:1020A0004A6B22F001024A6383F30988002383F319
:1020B0001188704700EF00E0302080F3118862B68D
:1020C0000D4B0E4AD96821F4E0610904090C0A435A
:1020D0000B49DA60D3F8FC2042F08072C3F8FC2090
:1020E000084AC2F8B01F116841F0010111602022B6
:1020F000DA7783F82200704700ED00E00003FA056C
:1021000055CEACC5001000E0302310B583F3118824
:102110000E4B5B6813F4006314D0F1EE103AEFF34A
:1021200009844FF08073683CE361094BDB6B2366E5
:1021300084F30988FFF772FA10B1064BA36110BD52
:10214000054BFBE783F31188F9E700BF00ED00E0E2
:1021500000EF00E033040008360400080E4B9A6CD0
:1021600042F008029A641A6F42F008021A670B4A9A
:102170001B6FD36B43F00803D363C722084B9A62EB
:102180004FF0FF32DA6200229A615A63DA605A60D5
:1021900001225A611A607047004502580010005C25
:1021A000000C0040094A08B51169D3680B40D9B248
:1021B0009B076FEA0101116107D5302383F3118872
:1021C000FFF76EFA002383F3118808BD000C00406E
:1021D000044BDA6B0243DA635A6E104358665B6E47
:1021E000704700BF004502583A4B4FF0FF31D3F81B
:1021F000802062F00042C3F88020D3F8802002F0F3
:102200000042C3F88020D3F88020D3F88420C3F89C
:102210008410D3F884200022C3F88420D3F88400EB
:10222000D86F40F0FF4040F4FF0040F4DF4040F042
:102230007F00D867D86F20F0FF4020F4FF0020F423
:10224000DF4020F07F00D867D86FD3F888006FEAAE
:1022500040506FEA5050C3F88800D3F88800C0F3AC
:102260000A00C3F88800D3F88800D3F89000C3F8B8
:102270009010D3F89000C3F89020D3F89000D3F8D2
:102280009400C3F89410D3F89400C3F89420D3F8C2
:102290009400D3F89800C3F89810D3F89800C3F8C6
:1022A0009820D3F89800D3F88C00C3F88C10D3F89A
:1022B0008C00C3F88C20D3F88C00D3F89C00C3F8B2
:1022C0009C10D3F89C10C3F89C20D3F89C3000F0ED
:1022D000BFB900BF0044025808B50122504BC3F8F3
:1022E0000821504B5A6D42F002025A65DA6F42F0F3
:1022F0000202DA670422DB6F4B4BDA605A68910402
:10230000FCD54A4A1A6001229A60494ADA600022E2
:102310001A614FF440429A61434B9A699204FCD58A
:102320001A6842F480721A60424B1A6F12F4407FAE
:1023300004D04FF480321A6700221A671A6842F0FC
:1023400001021A603B4B1A685007FCD500221A6143
:102350001A6912F03802FBD1012119604FF0804157
:1023600059605A67344ADA62344A1A611A6842F488
:1023700080321A602F4B1A689103FCD51A6842F418
:1023800080521A601A689204FCD52D4A2D499A622F
:1023900000225A63196301F57C01DA6301F5E771E4
:1023A00099635A64284A1A64284ADA621A6842F021
:1023B000A8521A601F4B1A6802F02852B2F1285F27
:1023C000F9D148229A614FF48862DA6140221A6298
:1023D0001F4ADA641F4A1A651F4A5A651F4A9A65DE
:1023E00032231F4A1360136803F00F03022BFAD144
:1023F000104A136943F003031361136903F03803B0
:10240000182BFAD14FF00050FFF7E2FE4FF080405A
:10241000FFF7DEFE4FF00040BDE80840FFF7D8BEF2
:1024200000800051004502580048025800C000F0EA
:1024300004000001004402580000FF0100889008D9
:102440003220600063020901470E0508DD0BBF0161
:1024500020000020000001100910E0000001011020
:10246000002000524FF0B04208B5D2F8883003F097
:102470000103C2F8883023B1044A13680BB15068D5
:102480009847BDE80840FFF73FBE00BFF02E002090
:102490004FF0B04208B5D2F8883003F00203C2F81A
:1024A000883023B1044A93680BB1D0689847BDE8DF
:1024B0000840FFF729BE00BFF02E00204FF0B042C9
:1024C00008B5D2F8883003F00403C2F8883023B18D
:1024D000044A13690BB150699847BDE80840FFF7FB
:1024E00013BE00BFF02E00204FF0B04208B5D2F866
:1024F000883003F00803C2F8883023B1044A936996
:102500000BB1D0699847BDE80840FFF7FDBD00BF9B
:10251000F02E00204FF0B04208B5D2F8883003F01A
:102520001003C2F8883023B1044A136A0BB1506A11
:102530009847BDE80840FFF7E7BD00BFF02E002038
:102540004FF0B04310B5D3F8884004F47872C3F864
:102550008820A30604D5124A936A0BB1D06A984723
:10256000600604D50E4A136B0BB1506B98472106D9
:1025700004D50B4A936B0BB1D06B9847E20504D599
:10258000074A136C0BB1506C9847A30504D5044A55
:10259000936C0BB1D06C9847BDE81040FFF7B4BD09
:1025A000F02E00204FF0B04310B5D3F8884004F46B
:1025B0007C42C3F88820620504D5164A136D0BB11E
:1025C000506D9847230504D5124A936D0BB1D06D19
:1025D0009847E00404D50F4A136E0BB1506E98472C
:1025E000A10404D50B4A936E0BB1D06E98476204D8
:1025F00004D5084A136F0BB1506F9847230404D5D4
:10260000044A936F0BB1D06F9847BDE81040FFF7B5
:102610007BBD00BFF02E002008B50348FEF74AFD41
:10262000BDE80840FFF770BDA023002008B50348AF
:10263000FEF740FDBDE80840FFF766BD0C24002012
:1026400008B5FFF7AFFDBDE80840FFF75DBD00002E
:10265000062108B5084600F02BF80621072000F0F7
:1026600027F80621082000F023F80621092000F0B1
:102670001FF806210A2000F01BF80621172000F0A1
:1026800017F80621282000F013F809217A2000F01D
:102690000FF80721322000F00BF80C21522000F037
:1026A00007F80C215320BDE8084000F001B80000F5
:1026B000090100F16043012203F56143C9B283F8C7
:1026C000001300F01F039A4043099B0003F160438D
:1026D00003F56143C3F880211A60704708B5FFF71E
:1026E00083FD00F009F8FEF7FDFEFFF7D3FCBDE81F
:1026F0000840FFF7B5BB00000023054A1946013327
:10270000102BC2E9001102F10802F8D1704700BF96
:10271000F02E002010B501390244904201D1002072
:1027200005E0037811F8014FA34201D0181B10BD3A
:102730000130F2E753544D333248373F3F3F0053A7
:10274000544D3332483734332F37353300000000CF
:1027500001105A00031059000120580003205600B0
:1027600000960000000000000000000000000000D3
:10277000000000000000000000000000A514000898
:1027800091140008CD140008B9140008C5140008FD
:10279000B11400089D14000889140008D914000819
:1027A00063300000A0270008D02C0020E02E00207D
:1027B0006D61696E0069646C6500000000000028AE
:1027C00000000000AAAAAAAA00000024FFFF00003F
:1027D00000000000000000000000000000000000F9
:1027E000AAAAAAAA00000000FFFF00000000000043
:1027F000000000000000000000000000AAAAAAAA31
:1028000000000000FFFF00000000000000000000CA
:102810000000100000000000AAAAAAAA0000000000
:10282000FFFF000000000000000000000A8002001E
:1028300000000000AAAAAAAA05400100FFFF0000AC
:102840008800007007000000000000000000000089
:10285000AAAAAAAA00000000FFFF000000000000D2
:10286000000000000000000000000000AAAAAAAAC0
:1028700000000000FFFF000000000000000000005A
:102880000000000000000000AAAAAAAA00000000A0
:10289000FFFF00000000000000000000000000003A
:1028A00000000000AAAAAAAA00000000FFFF000082
:1028B0000000000000000000000000000000000018
:1028C000AAAAAAAA00000000FFFF00000000000062
:1028D000000000000000000000000000AAAAAAAA50
:1028E00000000000FFFF00000000000000000000EA
:1028F0002E0400000000000000001A00000000008C
:10290000FF000000A0230020000000003427000882
:102910003F000000500400003F2700083F00000077
:10292000FFFFFFFFFFFFFFFFFFFFFFFFFFFFFFFFB7
:10293000FFFFFFFFFFFFFFFFFFFFFFFFFFFFFFFFA7
:10294000FFFFFFFFFFFFFFFFFFFFFFFFFFFFFFFF97
:10295000FFFFFFFFFFFFFFFFFFFFFFFFFFFFFFFF87
:020000040801F1
:020000040802F0
:1000000000060030BD0D02080D010E085103020864
:1000100095000E088D000E0891000E08BF0D020815
:10002000BF0D0208BF0D0208BF0D020841B912083A
:10003000BF0D0208BF0D0208BF0D0208BF0D020868
:10004000BF0D0208BF0D0208BF0D0208BF0D020858
:10005000BF0D0208BF0D02080DFD120839FD120880
:1000600065FD120891FD1208BDFD1208FDC11208C0
:1000700025C2120851C212087DC21208A9C2120874
:10008000D1C21208FDC212082DBE1208A5CE0D085D
:10009000CDCE0D08B9CE0D08E1CE0D08E9FD120850
:1000A000BF0D020839FF1208BF0D02084DFF1208EC
:1000B00051FF1208BF0D0208BF0D0208BF0D020854
:1000C000BF0D0208BF0D0208BF0D0208BF0D0208D8
:1000D000ADC81208BF0D0208C1FE1208D5FE1208F5
:1000E0004DFE1208BF0D0208BF0D0208BF0D020829
:1000F000BF0D0208BF0D0208BF0D020829C3120878
:10010000BF0D0208BF0D020865FF1208BF0D0208EF
:10011000E9FE1208BF0D0208BF0D0208BF0D02085C
:1001200055C312087DC31208A9C31208D5C312080B
:1001300001C41208BF0D0208BF0D0208BF0D02085E
:10014000BF0D0208BF0D0208BF0D0208BF0D020857
:1001500029C4120855C4120881C41208FDFE1208F1
:10016000BF0D0208BF0D0208BF0D0208BF0D020837
:10017000BF0D0208BF0D0208BF0D0208BF0D020827
:10018000BF0D0208BF0D020811FF120825FF12085B
:10019000C1C81208BF0D0208BF0D0208BF0D02083A
:1001A000BF0D0208BF0D0208BF0D0208BF0D0208F7
:1001B000BF0D0208BF0D0208BF0D0208BF0D0208E7
:1001C000BF0D0208BF0D0208BF0D0208BF0D0208D7
:1001D000BF0D0208BF0D0208BF0D0208BF0D0208C7
:1001E000BF0D0208BF0D0208BF0D0208BF0D0208B7
:1001F000BF0D0208BF0D0208BF0D0208BF0D0208A7
:10020000BF0D0208BF0D0208BF0D0208BF0D020896
:10021000BF0D0208BF0D0208BF0D0208BF0D020886
:10022000BF0D0208BF0D0208BF0D0208BF0D020876
:10023000BF0D0208BF0D0208BF0D02084DBE120817
:10024000BF0D0208D5BF1208FDBF120829C0120851
:1002500055C0120881C01208ADC01208D9C01208DA
:1002600005C11208BF0D0208BF0D0208BF0D02082C
:10027000BF0D0208BF0D0208BF0D0208BF0D020826
:10028000BF0D0208BF0D0208BF0D0208BF0D020816
:10029000BF0D0208BF0D0208BF0D0208BF0D020806
:1002A000BF0D0208BF0D0208BF0D0208BF0D0208F6
:1002B000BF0D0208BF0D0208BF0D0208BF0D0208E6
:1002C000BF0D0208BF0D0208BF0D0208BF0D0208D6
:1002D000BF0D0208BF0D0208BF0D0208BF0D0208C6
:1002E000A139020825720208A517030895340408ED
:1002F000C5030508B5F605083D5B08080D6108084B
:100300002DD10808FD260908CD2E09082932090833
:1003100005C6090821E20A08C9300B08F5CE0D0808
:10032000E1D50D0851FB0D08DD070E08A9840E0864
:10033000F5CC0E0841350F083D990F08D16511081D
:1003400021BC1108651912080D4B1208D150120872
:10035000EFF30383EFF30982EFF30881DFF814D0A2
:100360002DE9FE4F684600F053FEBDE8FE4F8D4676
:1003700070470000FC2F0030F1EE101AA0EC200AAC
:1003800001607047A0EC108A704700BF81F0004107
:1003900002E000BF83F0004330B54FEA41044FEA6A
:1003A000430594EA050F08BF90EA020F1FBF54EA05
:1003B000000C55EA020C7FEA645C7FEA655C00F0A1
:1003C000E2804FEA5454D4EB5555B8BF6D420CDD72
:1003D0002C4480EA020281EA030382EA000083EAF5
:1003E000010180EA020281EA0303362D88BF30BD95
:1003F00011F0004F4FEA01314FF4801C4CEA1131EB
:1004000002D0404261EB410113F0004F4FEA033349
:100410004CEA133302D0524263EB430394EA050FD4
:1004200000F0A780A4F10104D5F1200E0DDB02FA43
:100430000EFC22FA05F2801841F1000103FA0EF2D7
:10044000801843FA05F359410EE0A5F120050EF19D
:10045000200E012A03FA0EFC28BF4CF0020C43FACE
:1004600005F3C01851EBE37101F0004507D54FF0DB
:10047000000EDCF1000C7EEB00006EEB0101B1F52B
:10048000801F1BD3B1F5001F0CD349085FEA300071
:100490004FEA3C0C04F101044FEA445212F5800F7C
:1004A00080F09A80BCF1004F08BF5FEA500C50F119
:1004B000000041EB045141EA050130BD5FEA4C0CFC
:1004C000404141EB0101013C28BFB1F5801FE9D259
:1004D00091F0000F04BF01460020B1FA81F308BF7C
:1004E0002033A3F10B03B3F120020CDA0C3208DD48
:1004F00002F1140CC2F10C0201FA0CF021FA02F123
:100500000CE002F11402D8BFC2F1200C01FA02F192
:1005100020FA0CFCDCBF41EA0C019040E41AA2BFB7
:1005200001EB0451294330BD6FEA04041F3C1CDA7F
:100530000C340EDC04F11404C4F1200220FA04F09F
:1005400001FA02F340EA030021FA04F345EA030149
:1005500030BDC4F10C04C4F1200220FA02F001FA0B
:1005600004F340EA0300294630BD21FA04F029468D
:1005700030BD94F0000F83F4801306BF81F4801126
:100580000134013D4EE77FEA645C18BF7FEA655C99
:1005900029D094EA050F08BF90EA020F05D054EA6B
:1005A000000C04BF1946104630BD91EA030F1EBF70
:1005B0000021002030BD5FEA545C05D14000494174
:1005C00028BF41F0004130BD14F580043CBF01F567
:1005D000801130BD01F0004545F0FE4141F470014D
:1005E0004FF0000030BD7FEA645C1ABF1946104628
:1005F0007FEA655C1CBF0B46024650EA013406BF29
:1006000052EA033591EA030F41F4002130BD00BFE7
:1006100090F0000F04BF0021704730B54FF48064A4
:1006200004F132044FF000054FF0000150E700BF25
:1006300090F0000F04BF0021704730B54FF4806484
:1006400004F1320410F0004548BF40424FF0000171
:100650003EE700BF42004FEAE2014FEA31014FEAB4
:1006600002701FBF12F07F4393F07F4F81F0605103
:10067000704732F07F4208BF704793F07F4F04BF4E
:1006800041F40021704730B54FF4607401F000452B
:1006900021F000411CE700BF50EA010208BF70478B
:1006A00030B54FF000050AE050EA010208BF70477C
:1006B00030B511F0004502D5404261EB41014FF4E5
:1006C000806404F132045FEA915C3FF4D8AE4FF0ED
:1006D00003025FEADC0C18BF03325FEADC0C18BFD0
:1006E000033202EBDC02C2F1200300FA03FC20FA21
:1006F00002F001FA03FE40EA0E0021FA02F114446E
:10070000BDE600BF80F0004002E000BF81F0004184
:1007100042001FBF5FEA410392EA030F7FEA226CA7
:100720007FEA236C6AD04FEA1262D2EB1363C1BF37
:10073000D218414048404140B8BF5B42192B88BFA6
:10074000704710F0004F40F4000020F07F4018BFC9
:10075000404211F0004F41F4000121F07F4118BFE9
:10076000494292EA030F3FD0A2F1010241FA03FC91
:1007700010EB0C00C3F1200301FA03F100F0004379
:1007800002D5494260EB4000B0F5000F13D3B0F141
:10079000807F06D340084FEA310102F10102FE2AB0
:1007A00051D2B1F1004F40EBC25008BF20F0010020
:1007B00040EA03007047490040EB0000013A28BFBF
:1007C000B0F5000FEDD2B0FA80FCACF1080CB2EB42
:1007D0000C0200FA0CF0AABF00EBC25052421843C0
:1007E000BCBFD0401843704792F0000F81F4000165
:1007F00006BF80F400000132013BB5E74FEA410338
:100800007FEA226C18BF7FEA236C21D092EA030FA3
:1008100004D092F0000F08BF0846704790EA010F1D
:100820001CBF0020704712F07F4F04D1400028BF4A
:1008300040F00040704712F100723CBF00F500002C
:10084000704700F0004343F0FE4040F40000704762
:100850007FEA226216BF08467FEA2363014642020E
:1008600006BF5FEA412390EA010F40F48000704721
:100870004FF0000304E000BF10F0004348BF4042C7
:100880005FEA000C08BF704743F0964301464FF003
:1008900000001CE050EA010208BF70474FF000035F
:1008A0000AE000BF50EA010208BF704711F00043A0
:1008B00002D5404261EB41015FEA010C02BF844670
:1008C0000146002043F0B64308BFA3F18053A3F5CF
:1008D0000003BCFA8CF2083AA3EBC25310DB01FA16
:1008E00002FC634400FA02FCC2F12002BCF1004F9A
:1008F00020FA02F243EB020008BF20F0010070472B
:1009000002F1200201FA02FCC2F1200250EA4C007E
:1009100021FA02F243EB020008BF20EADC707047C4
:100920007BB972B90029BEBF00204FF0004106E03C
:1009300008BF00281CBF6FF000414FF0FF3000F0EF
:100940003BBAADF1080C6DE904CE002909DB002BA0
:100950001ADB00F0C9F8DDF804E0DDE9022304B099
:100960007047404261EB4101002B1BDB00F0BCF8FB
:10097000DDF804E0DDE9022304B0404261EB41010F
:10098000524263EB43037047524263EB430300F070
:10099000ABF8DDF804E0DDE9022304B0404261EB8E
:1009A00041017047524263EB430300F09DF8DDF8CC
:1009B00004E0DDE9022304B0524263EB43037047D5
:1009C00053B94AB9002908BF00281CBF4FF0FF31B6
:1009D0004FF0FF3000F0F0B9ADF1080C6DE904CE36
:1009E00000F082F8DDF804E0DDE9022304B070478E
:1009F000430803F05533C01A830803F0333300F083
:100A00003330184400EB101000F00F3000EB0020E2
:100A100000EB0040000E704780EA104080EA102092
:100A200080EA101046F6961300F00F0043FA00F02B
:100A300000F00100704700BF08B502460B4643ECCA
:100A4000172BB5EEC07BF1EE10FA03D4BDE80840D9
:100A500000F02AB8B1EE477B51EC170B00F024F8F8
:100A6000404261EB410108BD9FED0B6B07EE900A20
:100A70009FED0B5BB7EEE77A27EE066BBCEEC66B1D
:100A8000B8EE464BA4EE457BFCEEC77B16EE101A83
:100A900017EE900A704700BF000000000000F03D14
:100AA000000000000000F0419FED0B6B41EC170BC4
:100AB0009FED0B5B27EE066BBCEEC66BB8EE464BAC
:100AC000A4EE457BFCEEC77B16EE101A17EE900ADB
:100AD000704700BFAFF30080000000000000F03D51
:100AE000000000000000F0412DE9F047089D044699
:100AF0008E46002B4DD18A42944669D9B2FA82F2D1
:100B000052B101FA02F3C2F1200120FA01F10CFA0C
:100B100002FC41EA030E94404FEA1C48210CBEFB44
:100B2000F8F61FFA8CF708FB16E341EA034306FBCD
:100B300007F199420AD91CEB030306F1FF3080F05C
:100B40001F81994240F21C81023E63445B1AA4B2A9
:100B5000B3FBF8F008FB103344EA034400FB07F74B
:100B6000A7420AD91CEB040400F1FF3380F00A818C
:100B7000A74240F207816444023840EA0640E41B81
:100B800000261DB1D4400023C5E900433146BDE82D
:100B9000F0878B4209D9002D00F0EF800026C5E9CF
:100BA000000130463146BDE8F087B3FA83F6002EE7
:100BB0004AD18B4202D3824200F2F980841A61EB5F
:100BC000030301209E46002DE0D0C5E9004EDDE77D
:100BD00002B9FFDEB2FA82F2002A40F09280A1EB65
:100BE0000C014FEA1C471FFA8CFE0126200CB1FBBA
:100BF000F7F307FB131140EA01410EFB03F08842B3
:100C000008D91CEB010103F1FF3802D2884200F23F
:100C1000CB804346091AA4B2B1FBF7F007FB1011D1
:100C200044EA01440EFB00FEA64508D91CEB04046F
:100C300000F1FF3102D2A64500F2BB800846A4EBCA
:100C40000E0440EA03409CE7C6F12007B34022FAB5
:100C500007FC4CEA030C20FA07F401FA06F31C43E4
:100C6000F9404FEA1C4900FA06F3B1FBF9F8200CF1
:100C70001FFA8CFE09FB181140EA014108FB0EF037
:100C8000884202FA06F20BD91CEB010108F1FF3A87
:100C900080F08880884240F28580A8F10208614493
:100CA000091AA4B2B1FBF9F009FB101144EA0141A1
:100CB00000FB0EFE8E4508D91CEB010100F1FF344C
:100CC0006CD28E456AD90238614440EA0840A0FBE4
:100CD0000294A1EB0E01A142C846A64656D353D0BA
:100CE0005DB1B3EB080261EB0E0101FA07F722FADE
:100CF00006F3F1401F43C5E9007100263146BDE807
:100D0000F087C2F12003D8400CFA02FC21FA03F369
:100D1000914001434FEA1C471FFA8CFEB3FBF7F0EA
:100D200007FB10360B0C43EA064300FB0EF69E420F
:100D300004FA02F408D91CEB030300F1FF382FD2A8
:100D40009E422DD9023863449B1B89B2B3FBF7F650
:100D500007FB163341EA034106FB0EF38B4208D929
:100D60001CEB010106F1FF3816D28B4214D9023E6A
:100D70006144C91A46EA004638E72E46284605E788
:100D80000646E3E61846F8E64B45A9D2B9EB020859
:100D900064EB0C0E0138A3E74646EAE7204694E7E9
:100DA0004046D1E7D0467BE7023B614432E730461C
:100DB00009E76444023842E7704700BF02E000F0F0
:100DC00000F8FEE772B6384880F30888374880F3A9
:100DD000098837483749086040F20000CCF200002B
:100DE0004EF63471CEF200010860BFF34F8FBFF3AF
:100DF0006F8F40F20000C0F2F0004EF68851CEF244
:100E000000010860BFF34F8FBFF36F8F4FF00000FA
:100E1000E1EE100A4EF63C71CEF2000108600620A9
:100E200080F31488BFF36F8F0EF164FC0EF106FCA3
:100E30000EF13AFD4FF055301F491B4A91423CBF1D
:100E400041F8040BFAE71D49184A91423CBF41F8AA
:100E5000040BFAE71A491B4A1B4B9A423EBF51F852
:100E6000040B42F8040BF8E700201849184A914295
:100E70003CBF41F8040BFAE70EF11EFC0EF196FDA3
:100E8000144C154DAC4203DA54F8041B8847F9E7BB
:100E900002F0D6FC114C124DAC4203DA54F8041B9C
:100EA0008847F9E70EF106BC00060030002200304A
:100EB0000000020808ED00E00000003000060030ED
:100EC000F05C160800220030082E0030082E00309A
:100ED00038E50130E002020850030208500302081E
:100EE000500302082DE9F04F2DED108AC1F80CD007
:100EF000D0F80CD0BDEC108ABDE8F08F002383F34E
:100F000011882846A04700200DF1F8FBFEE70DF1FF
:100F10007FFA00DFFEE7000001F0FF01102A2BDB63
:100F200010F0070F08D010F8013B013A8B422DD08A
:100F300010F0070F42B3F6D1F0B441EA012141EAC3
:100F4000014122F007047FF000070023F0E8025679
:100F5000083C85EA010586EA010685FA47F5A3FA09
:100F600087F586FA47F6A5FA87F68EB9EED1F0BC7A
:100F700001F0FF0102F0070232B110F8013B013A23
:100F800083EA010313B1F8D100207047013870479C
:100F9000002D06BF35460338073815F0010F07D17D
:100FA000013015F4807F02BF013015F4C03F0130DD
:100FB000F0BC0138704700BF10F8012B11F8013B5D
:100FC000012A28BF9A42F7D0D01A7047034613F877
:100FD000012B002AFBD1181A0138704710B50446BE
:100FE00020461CB154F80C3B013300D110BD08223F
:100FF000012100F067FB54F80C0C54F8082C14F88D
:10100000041C121AB2FBF1F200F05CFBE8E70000EE
:10101000C26AD0E9003112F0040F2DE9F04118BF87
:101020000B46A6B00021594C042601270291CDE9B8
:101030000003D0064CBF03F1200203F168020392C3
:10104000DA690399D2099B6902F004021B880A43FA
:1010500003F47F4303924FF0E022A3F53E41D2F820
:10106000882D02F4A002B2F5A00F04BF0122029263
:101070004B424B410493464D03A82C6000F020FAEC
:1010800004220121434800F01DFB0422012102A893
:1010900000F018FB10220121019800F013FB0098CA
:1010A000202201210C3000F00DFB019804220121C7
:1010B000103000F007FB0422012103A800F002FB1E
:1010C00001980C220121143000F0FCFA0C220121BD
:1010D000009800F0F7FA029BDA071FD5009BDB6A45
:1010E000DB064ED415A8FFF74DF9DDF804C00DF16D
:1010F000140E0CF120030CF160081868083353F843
:10110000041C7246434503C29646F6D1DCF86030B3
:1011100025938422012105A800F0D4FA00F0BEF83E
:10112000FFF75CFF4FF0E023D3F8003D03F470239A
:10113000B3F5402F0ED0184B05A88DF81C60059311
:1011400014338DF8287006934FF0FF33CDE9083340
:10115000FFF744FF2B68A34206D0104B0422012165
:1011600005A8059300F0AEFA00F020FA002882D01E
:10117000049B1BB1019A93690233936126B0BDE8C9
:10118000F08105A8FFF7F8F8C3E700BFED55CEAC36
:10119000082E00309079130828ED00E0ACCE55ED14
:1011A00037B50E4D2A78202A15D10D4C0D482368ED
:1011B0000D49184401920DF14FFD23680021019A59
:1011C000203309482970236012F126FE03B0BDE8E0
:1011D00030400EF1FDB903B030BD00BFFC2F003030
:1011E0002430003000691608FE2F003008B5522068
:1011F0000CF16CFA124BD3F8902042F08042C3F805
:101200009020D3F8902022F08042C3F89020D3F8A9
:1012100090300C4B9A6C42F080429A641A6F42F004
:1012200080421A676D221B6F074BDA604FF0FF3266
:101230001A620D221A600122044B1A7008BD00BF09
:101240000044025800450258007800403430003015
:10125000014B1868704700BFFCFF1B08014B024898
:10126000C01A70470069160800001C080048704743
:101270000069160807490022074B5B1A9A4201D3FE
:101280000120704751F8040B013001D10432F5E719
:10129000002070470069160800001C085A4B2DE911
:1012A000F74F1F680224594B07F56A57DFF8809102
:1012B0001B781837DFF87C81554D1F44DFF878A183
:1012C0000CF1CAFFA9EB080B06460EB13A2C41D926
:1012D000A9EB0803B3EB070C24D4DFF860E1661C2C
:1012E0004C4A0C21F6B2AEEB0200614360456FDD63
:1012F000681801276A50624407721F464260DB1B70
:1013000077D445490234454FE4B2CA1B9A424FF0A4
:101310000C0206FB02F266DDA91801203B44AF5027
:1013200008724B603B2C66D80C2301225C432B19BE
:101330001A724FF0FF322A515A60394B1B782BB189
:10134000384B1B682B60384B1B686B60304803B010
:10135000BDE8F08F336AF06953450ABF334BF31A87
:10136000A3EB0A0380B101930DF158FE019B58B124
:1013700022460C2101344A430121E4B2A81801722B
:10138000F169A9500D3141600C2001211F4400FB7F
:1013900004FC5F4505EB0C0245F80C6006F13C0CC3
:1013A0001172C2F804C004EB010204F10204D2B2CB
:1013B000E4B200FB02F205EB02000172316AA950AF
:1013C00019444160AED230460CF156FF06467CE728
:1013D00005EB010C4FF0010807446A508CF80880B7
:1013E000CCF804E08BE7AB180120AF5018725960BD
:1013F00098E7344696E7012385F8CC324FF0FF3367
:10140000C5E9B13399E700BF24300030FC2F00302C
:1014100004220030082E00300000043038E501308E
:101420000022003028300030203000300022003010
:1014300000001C08006916080006003038E501307D
:101440000C4B1B7810B50BB9FFF7D0FE00230A49EF
:101450000A48CA699206FCD54A6A1C5CD2B2944218
:1014600005D10133DBB20E2BF3D1002010BD0023D8
:10147000EFE700BF34300030007800409479130863
:1014800038B5084B04461B780BB9FFF7AFFEE4B242
:10149000054DAC62EB695B0600D538BD0EF198F8DE
:1014A000F8E700BF343000300078004010B5441E2B
:1014B00014F8010F00B910BDFFF7E2FFF8E70000D4
:1014C00070B502680446EFF30581D9205369C9B2AB
:1014D000BEF0E2FD294B1B78A3B1294B94E8030031
:1014E00083E803002748FFF7E1FF6368B3B12648AC
:1014F000FFF7DCFF2548FFF7D9FFFFF7A1FF2448DE
:10150000FFF7D4FF234D2B783BB124681CB1204654
:101510000DF184FD20B900232B7070BD1E48E7E754
:1015200020461E4E0DF18EFD00F2145084421FD253
:1015300020460DF187FD30602046194E0DF196FDD5
:1015400004F5E053834217D920460DF18FFD30603A
:101550000023144A1360144A1370FFF78BFE00280F
:10156000D9D00EF135F80120BDE870400DF1F0BB87
:10157000A4F214533360DFE73360E9E7FD2F003056
:101580002C300030A4791308A9791308BA7913080C
:10159000A495140800220030B479130828300030D4
:1015A0002030003024300030FC2F0030284B1A78D7
:1015B00070B542B12748FFF779FF274B58680038CC
:1015C00018BF012070BD254A107800283CD0244E59
:1015D000244C33682448254D1A1D21782D1A0A44BD
:1015E000AA4205D3224A4FF0FF31D1612022227056
:1015F0002278D2B103F120018D4205D81F2A9FBF66
:101600001B4AD361202222702022194918440DF16F
:1016100023FB3268237800211548134420222170CF
:10162000336012F1F9FB0DF1D3FF33689D4207D906
:101630000F4920220F48CB610DF10EFB0DF1C8FFC1
:1016400000200DF185FBB8E701221A70BAE700BF50
:10165000FD2F0030007A13082C30003000220030BB
:1016600024300030FC2F00300069160800001C08F0
:10167000FE2F0030E0FF1B082DE9F84307460E4619
:101680000024DFF83890DFF83880B44201D1BDE89B
:10169000F88324B1230702D14846FFF707FF3D5DD9
:1016A00001342B0905F00F0518F80300FFF7E8FED9
:1016B00018F80500FFF7E4FEE7E700BFA49514085B
:1016C000107A1308474B1B782DE9F74F07460E4653
:1016D00090465BB1022925D0042938D0012902D1D6
:1016E0001146FFF7C9FF4048FFF7E0FE3F4B1B786C
:1016F000002B4ED03E4A00253E4BA2EB030938E0BA
:1017000037F81430ADF8043024B1620702D128460E
:10171000FFF7CCFE0134022101A8FFF7ADFFA04581
:10172000EED1E0E70024304DF9E757F8243001937B
:1017300024B1A30702D12846FFF7B8FE04210134E3
:101740000DEB0100FFF798FFA045EED1CBE7002499
:10175000254DF9E7FFF724FD022E1DD0042E2CD0D5
:10176000012E06D12378795D5A1C2270224AD15469
:101770000135A8450DD0214B214C1B68227804333C
:1017800013444B45E6D31C4B4FF0FF32DA61202364
:10179000237003B0BDE8F08F2378DFF85CA05A1CFB
:1017A00022703A780AF80320FFF7FAFC23785A1CD3
:1017B000227000220AF80320DAE74FF0000ADFF86F
:1017C00038B022783B78511C23FA0AF30AF1080A50
:1017D00021700BF80230FFF7E3FCBAF1200FF0D1D3
:1017E000C6E700BFFD2F0030A4951408002200308A
:1017F00000001C0800691608FE2F0030243000305D
:10180000FC2F00307FB5039140210546B0F004FC69
:10181000039A18B90124204604B070BD134E0392F8
:1018200096F97235002BF5D078F0E0FF437A039AF1
:1018300053B978F0DBFF847A039A2CB90C4B402122
:101840002846B0F0F1FBE6E70A4BB6F97415D3F879
:10185000B43DB3F906309942DCDD074B4021284600
:1018600000240093054BB0F0DFFBD4E73860003074
:10187000247A130838700030437A1308317A130839
:101880002DE9F0410D4690B020210446B0F0C4FB94
:10189000002800F0AE80584E96F97235BBB106F5BF
:1018A0008052B6F97435D2F8B42DB2F90A1003F1AA
:1018B0000A02914203DD40F28D32934207DC4F4B26
:1018C0002A4620212046B0F0AFFB00208EE096F99A
:1018D0006135022B05D14A4B2A4620212046B0F023
:1018E000A3FBB6F8343541F65832A3F57A739BB2B0
:1018F00093420FD8434F06F29C52D7F8843C92EDA6
:10190000007AD3ED097AB4EEE77AF1EE10FA03DD4E
:101910003D4BD5E73D4BD3E706F5B462D3ED0B7AEB
:1019200092ED007AB4EEE77AF1EE10FAF0DCB6F957
:101930006E35002B01DC364BC2E7A7F5005898F84E
:1019400004210D2A04D84FF42153D340DA0713D4CD
:10195000304811F097FA012806D1D7F88C0CA8F07E
:101960005BFD58B1012812D02B4B93F8F91111F0FF
:10197000100121D0294BA3E7294BA1E7294B009364
:10198000294B2A4620212046B0F04EFB9DE798F8CF
:10199000703EDB070ED51921244864F0FFFD48B1E5
:1019A000D6F84C651921214864F01EFE8642DBDD25
:1019B0001F4BE4E71F4BE2E72E2204A8039112F12C
:1019C0002BFA322303AA1C49D7F8880CA6F0D8FEBC
:1019D00018B903AB0093194BD3E7322303AA184974
:1019E000D7F8840CA5F02EF80028F2D010B0BDE88E
:1019F000F0810120FAE700BF386000304C7A13080C
:101A00005F7A130838900030977A1308877A1308A2
:101A1000B17A13089CA8003038800030407B13084E
:101A2000C67A13080B7B1308E67A1308B840003017
:101A30002A7B13081B7B1308557B1308597B13085B
:101A40006B7B130870B58EB00E4600212E22054622
:101A500002A8019112F1E0F9322201A909488CF0A3
:101A60005BFE044640B99DF9043043B9064B074A72
:101A700031462846B0F092FD20460EB070BD01AB55
:101A8000F5E700BFBC7B0030707B1308EADC13086D
:101A900007B50448AAF03EFA00F0010003B05DF873
:101AA00004FB00BFA09C00302DE9F043DFF87891E3
:101AB000044699B00D46D9F8E00103681B699847C0
:101AC000804619F0FFFE002107462E220CA80B913C
:101AD00012F1A2F932230BAA4146384619F0B6F9A1
:101AE000064648B90BAB434A29462046B0F056FD9E
:101AF000304619B0BDE8F0833F488AF08DFEB8F15A
:101B0000000F0BD0A9F5A04015F0C2FA80B93B4AEE
:101B1000294620460026B0F041FDE9E710F0060F07
:101B2000E6D0A9F5A04015F0B3FA08B9344AEFE7BA
:101B300003A9384617F0CEFF28B19DF80D305B069B
:101B400001D5304AE4E7DFF8E4800023D8ED007ADD
:101B5000F5EEC07AF1EE10FA35DD0DF120090893AB
:101B6000099305AA0A9307AB04A93846019306AB6B
:101B7000CDF8009019F090FC48463AF085FDD8ED7C
:101B8000007AB4EEE70AF1EE10FA01DB1E4ABFE775
:101B90009DED057AF4EEC77AF1EE10FA01D81B4AF2
:101BA000B6E79DED047AF4EEC77AF1EE10FA01D8AB
:101BB000174AADE79DED067AF4EEC77AF1EE10FA1A
:101BC00001D8144AA4E707F22C41134805F0C0FEDF
:101BD000074608B1114A9BE711490F4805F0B8FEC6
:101BE000002885D00F4A294620463E46B0F0D6FC54
:101BF0007EE700BF887B13081C620030917B1308CE
:101C0000A87B1308CE7B1308DC7B1308F17B130839
:101C1000077C13081D7C130838300030317C130812
:101C2000909C00304E7C130838800030C86500302E
:101C300008B5064B93F8F9319B0704D5044AB0F078
:101C4000ADFC002008BD0120FCE700BF388000305B
:101C5000707C130870B50E468EB020210546B0F09A
:101C6000DBF918B9012420460EB070BDB1F062FD59
:101C700004460028F6D000212E2202A8019112F17C
:101C8000CBF82046322201A9B1F01CFD0446002801
:101C9000E8D101AB024A31462846B0F07FFCE2E7CA
:101CA000EADC130870B50C4C05460E46D4F8E0018A
:101CB00003685B69984710B10124204670BDA4F504
:101CC000A04015F0F7F904460028F5D1034A314643
:101CD0002846B0F063FCF0E738800030807C1308C1
:101CE0002DE9704E424E8FB082468B46D6F80432B4
:101CF00093F8D14084B978F079FD202179F050FE35
:101D0000A8B178F073FD1F2179F04AFE40B1394A3D
:101D100059465046B0F042FC20460FB0BDE8708EE8
:101D200078F064FDA52179F03BFE0028EFD196F80C
:101D3000D63103F01403142B01D12F4AE8E72F4BBF
:101D40001D780DB12E4AE3E759465046B1F094FA9A
:101D500004460028E0D02E22294602A8019512F15F
:101D60005BF8D6F8040201AA322103681B68984781
:101D7000044630B901AB234A59465046B0F00EFC38
:101D8000CAE7DAF808303BB9DAF80030594650466D
:101D90005B6B98470446BFE759465046FFF770FD16
:101DA000814659465046FFF74DFE09EA0000594664
:101DB000C4B25046FFF73CFF594604405046FFF777
:101DC00049FF594604405046FFF71CFD5946044060
:101DD0005046FFF767FF594604405046B0F0F6FC06
:101DE000594604405046B1F05FFA044094E700BF02
:101DF00038800030947C1308AE7C130870BA003031
:101E00000EF61308C67C130808B5FFF769FF054AEC
:101E100092F8D41160F3041182F8D411024A90713F
:101E200008BD00BF3880003065AF0030F7B505460B
:101E30000F46B0F02DF9044678B102212846B0F0E3
:101E4000EBF8064648B11548AAF064F8C205C0F39D
:101E50000723C0F3002403D53446204603B0F0BD69
:101E60009B07F9D50D48AAF063F80D4B03F62C43F8
:101E7000D3ED007AF8EEE77A30EE670ADFED097A03
:101E8000B0EEC00AB4EEE70AF1EE10FAE4DD064B5C
:101E90003A4602212846B0F0C7F8DEE7A09C0030A1
:101EA000389000300000C842D47C1308F8B50446CE
:101EB0000F46B0F0BBFA102105462046B0F0ACF852
:101EC00058B12046FFF7E4FD064630B93546044BCD
:101ED0003A4610212046B0F0A7F82846F8BD00BFCA
:101EE000E87C130870B505460E46B0F017FB0446B3
:101EF00078B180212846B0F08FF850B1074B93F8A5
:101F0000593743B10024064B324680212846B0F0B1
:101F10008BF8204670BD0446FBE700BF38800030D8
:101F2000FC7C130838B50D4D0446D5F88C0CA8F090
:101F300073FA012810D0D5F88C0CA8F06DFA02289D
:101F400004D02046BDE83840B0F018B8044810F07E
:101F500099FF0128F5D138BD0020FCE7389000300A
:101F60009CA80030F0B5134C85B006460F4604F52A
:101F7000804304F5A044D3F8AC2D0092D3F8B02DE3
:101F80000192D3F8B42DD3F8B83D02926A46039378
:101F9000B1F000F9054639463046B0F0FDF994F845
:101FA000D431284060F3C303C3F3C00084F8D431B4
:101FB00005B0F0BD383000302DE9F843DFF8AC90C3
:101FC000064626480F468AF027FC0446D9F8E00169
:101FD000DFF89C8003681B699847054630B914F008
:101FE000060F03D1D9F81432022B09D139463046F5
:101FF000B0F074F8054618B9002488F807400AE0E4
:1020000039463046FFF750FD04460028F4D02DB97C
:10201000012388F807302046BDE8F88308213046C0
:10202000AFF0FAFF0028F3D00D4826F05BFE002841
:10203000EED00C4BB02193F8B02501FB023203F532
:102040004053B2F8BE23B3F962359A42E0DD064B45
:102050003A4608213046AFF0E7FFCDE71C6200307A
:102060000833003038300030107D130838800030DD
:1020700065AF003070B588B005460E46B0F0B6FAD0
:10208000044688B320212846AFF0C6FF60B31B4B3F
:1020900093F87C2D42B393F85C3D9B0724D507AAA7
:1020A00006A9174886F03CFDF0B19DED077ADFEDFB
:1020B000157AB4EEE77AF1EE10FA15D8B7EEC77AD2
:1020C0000024202128468DED027BDDED067AFDEE11
:1020D000E77A08A3D3E90023CDED007ACDE9042304
:1020E000094B3246AFF0A0FF204608B070BD00BFDC
:1020F000AFF30080000000403333E33F38900030FE
:10210000586700309A99193F207D13082DE9F34153
:102110000F46054619F0D6FB804617F037FF0446F8
:1021200040B9684A01212846B0F038FA204602B08A
:10213000BDE8F081404619F083FB78B924F04CFEED
:1021400090F84113044624F00FF97C23C0B203FB3E
:10215000004494F83D400CB95B4AE3E75B4E3946D6
:10216000D6F8E00103689B699847044658B9D6F849
:10217000E00103689B6B9847554A034601212846B6
:10218000B0F00CFAD2E7AB68002BCFD01021284674
:10219000AFF042FF20B3D8EDED7A98EDEC0A20EED7
:1021A000270A0EF125FFDFED4B7AA6F5005320EE4E
:1021B000270ADFED497AB3F9343520EE270A07EE16
:1021C000903AF8EEE77AB4EEE70AF1EE10FA07DD9E
:1021D000424B012210212846AFF026FF0024A5E73C
:1021E00020212846AFF018FF38B196F8F931DB0608
:1021F00003D53B4B01222021EDE740212846AFF0DB
:102200000BFF002833D0012F1CD0042F1AD0354CDF
:10221000D4F8B43DA4F58040B3F9083000EE103A8C
:10222000B8EEC00A00F068FBB5EEC00AF1EE10FA95
:102230002BDD2D4B01224021284600932B4BAFF084
:10224000F3FECBE7D6F8E00103681B689847042843
:102250000DD0D6F8E00103681B689847142806D013
:10226000D6F8E00103681B6898470328CFD1204BBC
:102270001B68586D03681B6A98470128014619D1ED
:102280001C4A2846B0F08AF9A8E7D6F8E0010368AE
:102290005B69984730B1D4F8B43DB3F90830002BEE
:1022A000E5DDC6E7D6F8E00103681B6898470B2810
:1022B000DDD1F0E73946284602B0BDE8F041B0F084
:1022C000CFBC00BF4C7D13085D7D13083880003003
:1022D000717D1308E02E65420000C842857D130819
:1022E000407B130838700030437A13088D7D130843
:1022F00008AD0030997D130870B505460E46FFF70E
:10230000D3FB084B04463146D8712846FFF7CAFC78
:1023100000283146284608BF0024B0F02DFF204099
:1023200070BD00BF65AF00302DE9F041514F3B78E3
:10233000002B40F09C80504C0126D4F804523E7093
:1023400095F8D1501DB13B702846BDE8F081B1F041
:1023500065F8054630B9494A3870137843F00103EF
:102360001370F1E76CF0B0FF31466CF03BF9A4F567
:10237000A04007F0DBFA424B1E710B26013E5DF0D8
:1023800003FD5DF09FFC16F0FF06F7D13D4800F01D
:1023900099FE19F097FAD0F87423C4F82C2290F81B
:1023A0003C34DA0753D418F027FE6CF08DFF3C2143
:1023B0006CF0D2FE0023C4F8EC310021314800F06B
:1023C00009FF304814F064FE01462F48AEF028FAA9
:1023D0002E4B2F4E01211B68586D03681B689847D0
:1023E00096F8B83DD4F804026FF3410386F8B83D7F
:1023F00003681B6A98470121D4F80402AAF052FD31
:102400006CF062FF8046D4F8E00103681B689847CF
:10241000A6F540530146404693F8F4226CF0A2FA28
:10242000A6F5C04007F074FA69F064FE69F0B8F9E7
:1024300000233B70BDF0A0FEB4F8D631C6F8980C6E
:1024400023F4087343F02003A4F8D6317CE79B07FC
:10245000B3D431460B4805F0F9FA0E48A9F068FDEF
:10246000DFED0D7A20EE270A84ED7B0AA5E7002533
:102470006AE700BF353000303880003084AF00306C
:1024800065AF003038300030447A003008AD00309D
:1024900038900030A09C00300AD7233C2DE9F0434F
:1024A000374D87B0D5F8043293F8D130002B64D083
:1024B00052B1012908D195F9D431002B04DB002455
:1024C000204607B0BDE8F083B1F04EF8044600287E
:1024D000F5D019F0F7F9074624F07EFC804638461F
:1024E00017F0A0FCD8B198F92430022B17D10026A0
:1024F0004FF00009F1B203AA3846CDF80C900191D3
:10250000CDF81090CDF8149018F0A8FA019918B1F0
:1025100003AA404624F086F80136032EEAD1194B6F
:10252000D5F8E001984224D10BF032FE0121164883
:1025300007F000FC0121144807F038FB0021D5F812
:102540000402AAF0AFFC11483CF00CFE6CF0BCFE9B
:1025500000216CF047F80E4B00211B68586D036892
:102560001B68984795F8D6316FF3451385F8D63137
:10257000A6E718460BF010FED8E70124A0E700BF3D
:102580003880003038A400303830003040A10030AE
:1025900008AD003001488AF007BA00BF1C62003065
:1025A00000F5A04008B590F8D431C3F340128A4238
:1025B0000BD061F3451380F8D43131B16CF084FE57
:1025C0000F21BDE808406CF0C7BD08BD70B500F52F
:1025D000A04605460C46D6F814328B4212D001298B
:1025E00011D0022916D059B96CF06EFE1B216CF087
:1025F000B3FD0D4A05F59F40062140306EF0BAFE4E
:10260000C6F8144270BD6CF05FFE1A216CF0A4FD98
:10261000064AEFE7012100F0DDFD6CF055FE1D21BB
:102620006CF09AFD024AE5E7F47D1308097E130871
:10263000047E130800F5A04210B592F8F9310C465B
:1026400003F00101A14209D064F3000382F8F931DB
:10265000DB0704D406F034FD024B9C7210BD06F07B
:1026600017FFF9E765AF003000F5A04090F8F931A9
:1026700061F3410380F8F931014B1973704700BFD2
:1026800065AF003010B5044678F0B0F8202179F03D
:1026900087F904F5A043003893F8D62118BF01202C
:1026A00060F3820283F8D62110BD000010B5044605
:1026B00069F020FD436F04F5A04204F5C040D2F854
:1026C0000422D360D0F8842C5364D0F8882CC2F84C
:1026D0004832D0F8840C0368BDE810405B6C1847A2
:1026E000F8B500F5A04504462DED028BD5F804326F
:1026F00093F8D130002B7ED095F9D431002B7ADBC2
:1027000000F5E04393F83430002B74D1D5F8E001A4
:1027100003685B69984700286DD1384BD3F8E00116
:1027200003681B6898470B2865D004F5C0479FEDE8
:10273000347AD7F8883CD3EDAA7AF0EEE77AF4EE53
:10274000C77AF1EE10FA56D5D5F8040244306EF08F
:1027500055F90346B7EE001A9C20DFED2A0A93EDE7
:10276000000A34F093F8B5EEC00AF1EE10FA42DD3B
:1027700004F5D8406830A9F0E7FBB0EEC00ADFED01
:10278000227AB4EEE70AF1EE10FA34D504F5805659
:10279000D7F8840CD6F8043F07EE903A0368B8EEF9
:1027A000E78ADB6F9847DFED197A38EE400AB0EE22
:1027B000C00AB4EEE70AF1EE10FA1CD5D6F8083FCD
:1027C00040F2E63203F2F313934214D8D5F8040230
:1027D0009FED0F0AACF018F8D5F8043204F5A150BB
:1027E0009FED0B0AD3ED0C0A0830BDEC028BBDE85F
:1027F000F84096F069BDBDEC028BF8BD3880003022
:102800000000003400000000000070420000FA43A5
:102810000AD7233C00F5A04008B5D0F804020368AD
:102820009B689847F6EE007A20EE270AB5EEC00ABC
:10283000F1EE10FA48BF9FED010A08BD000000004C
:1028400038B500F5C0450446B7EE001A6F2004F510
:10285000A044DFED110A2DED028BD5F8843C93EDF9
:102860002E0A34F013F8D4F80402B0EE408AD5F8FA
:10287000885C036805F5B8759B68984738EE400A90
:10288000DFED067A2846BDEC028B20EE270ABDE874
:10289000384092F04FBF00BF0000000000007A44B3
:1028A00000F5DC50D2ED007A91ED006AD0EDF45ADB
:1028B000D0EDF76A26EEE77A67EEA57AA6EE257ADE
:1028C000E6EE267A81ED007AC2ED007A70470000CC
:1028D00000F58043B3F9DC3A43B900F54050B0F954
:1028E0006E050028B8BF404280B2704783EAE370AB
:1028F000A0EBE370F8E7000000F5A04330B52DED44
:10290000028B93F8F91183B0044611F0010105D050
:102910009FED2C0A03B0BDEC028B30BD93F8D5318E
:1029200001915B07F4D5DFED288A04F54055DFED12
:10293000250A4C20B0EE681A33F0A8FF4FF4C87295
:102940000199B0EE408AB5F9760534F007F8A5F89C
:102950007605204613F0CCFFB5F9763507EE900AE0
:10296000B8EEE77A07EE903AF8EEE77A77EE676A24
:10297000B4EEE68AF1EE10FA0DD5204638EE668AFE
:10298000FFF7A6FF07EE900AB8EEE70A20EE088AE6
:1029900088EE260ABEE777EE877AB4EEE78AF1EE94
:1029A00010FAB5DDB5F96E3538EE678A78EEE77A5C
:1029B00000EE103AB8EEC00A20EE088A88EE270A28
:1029C000A8E700BF0000000000007A440020704724
:1029D000002070477047000000F5A040D0F8E001EB
:1029E00003681B6818470000034808603B2111700A
:1029F00008221A60704700BF8084130800F5A040C9
:102A000010B5D0F8E0010C4603685B6D984707EEFF
:102A1000900A9FED057A0120F8EE677A67EE877AD3
:102A2000C4ED007A10BD00BF0AD7233C00F5A040DA
:102A300010B5D0F8E0010C4603681B6D984707EE0F
:102A4000900A9FED057A0120F8EEE77A67EE877A23
:102A5000C4ED007A10BD00BF0AD7233C00F5A040AA
:102A600010B5D0F8E0010C4603689B6D9847DFED88
:102A7000047A012020EE270A84ED000A10BD00BF71
:102A80000AD7233C95F0D0BA7DF012BDB0F036BE27
:102A900089F032B904F0F4BB83F048B87AF0AAB8F0
:102AA00069F074BA31F03ABD6BF002BF1CF004BF9C
:102AB0007AF0B8BC77F046BB75F000B913F076BB7E
:102AC00014F040B907F0F0BA15F008BA06F04CBBA4
:102AD00006F0A2B805F0C6BF5DF0F4B813F0F8BC7C
:102AE0001BF08EBB7FF00CB989F068BD11F038B8CF
:102AF000FFF7F6BD13F0A0BCAEF0B0BA86F02EB86A
:102B000013F058BF03F01EBC13F01EBC13F096BBAD
:102B100077F0ECBD5EF02ABF28F0CEB802F0F2BE2E
:102B20007AF090BC14F05AB807F074BA04F0B0BF51
:102B300007F0C2BB06F028B806F0F0BF13F0C6BA23
:102B4000FFF7B4BD32F04AB906F024BD0AF09EBECC
:102B50000BF054B80AF0E8BF0A4A0B4692F9D421A8
:102B6000002A05DA00228A604A600A600120704764
:102B700000F5C040D0F8842C543207CA83E807001F
:102B8000F4E700BF38800030634B70B5044640F86E
:102B9000043B7DF0ADFD002504F1100004F5545612
:102BA0001CF0D2FC04F160001FF05CF904F5087021
:102BB00068F08AFF04F5347025F0D2FF04F5CB608D
:102BC0001AF098FE04F2FC7023F030FA04F5346039
:102BD00031F0AEFA04F57B607DF04AFB04F58450D9
:102BE00063F002FC04F59950043610307AF094FA40
:102BF00004F59B500C301DF00FFD04F5A15008307A
:102C000097F0DCF904F5D55018309FF0F9FE04F583
:102C1000D650143069F004FB04F5D95008307EF02A
:102C200015FF04F5805304F5DA503C4A83F8385B0D
:102C300004F5D9530830183313605CF0FBFE04F53B
:102C4000DC502946183016F07DFC04F50950203080
:102C500094F000F804F509502C3082F077FF04F569
:102C60000A50183094F0DAFC04F528501C309BF020
:102C700023FA04F52C5034309AF0D0FA04F52D5094
:102C80001C309DF0D7FA04F52F5018309FF070F8E3
:102C900004F530503C309FF09BFC04F5325004307A
:102CA00092F05EFF04F53450103015F03FFB04F550
:102CB00039503830A1F056F804F5475018490C3017
:102CC00062F0AEF904F54750243089F011FD04F5A7
:102CD0004A501C30A0F000FF04F5405383F8F45232
:102CE00004F54C550435284610356DF0D7FDAE423D
:102CF000F9D104F554500B4D1030A0F087FF2B682C
:102D000013B10948BDF006FA2046084962F088F977
:102D100020462C6070BD00BF68CE1408ECBF0030A8
:102D2000D025150864B00030187E130850CD140863
:102D300010B513F057FD77F059FD0368BDE810405A
:102D40005B681847FFF7F4BF10B5044606F046FF6E
:102D5000204614F0C7F9204604F072FC2046BDE876
:102D6000104004F0D3BD0000FFF7EEBF70B500F5D2
:102D7000A4450446303528461CF05EF924F02CF8B2
:102D800090F9213093B390F840337BB304F5A0431E
:102D900004F2FC76D3F8040244306DF02FFE0346B3
:102DA000B7EE001A9C20DFED120A93ED000A33F013
:102DB0006DFD94F9303828460021012B04F6542487
:102DC00008BF86ED0E0A1BF031FFDFED0A7A94EDA5
:102DD000287A304620EE270ADFED077AA7EE270A89
:102DE00084ED280ABDE8704023F0AABC70BD00BF86
:102DF00000000000CDCCCC3D6666663FFFF7B6BF55
:102E000010B50121044614F0A9F960B1114BD3F8B3
:102E1000E00103689B6A984728B9204602F04EFCFF
:102E2000204602F085FC4FF40011204614F096F97C
:102E300018B132F047FF31F08FF84FF4802120466F
:102E400014F08CF928B132F03DFFBDE8104030F0AD
:102E500091BF10BD38800030FFF7D2BF38B50221D6
:102E6000044614F07BF970B10121204614F076F984
:102E700048B9534BD3F8E00103689B6A984710B9EF
:102E8000204602F01BFC0121204614F067F948B9E6
:102E90004B4BD3F8E00103689B6A984710B9204672
:102EA00002F046FC0121204614F058F910B92046E2
:102EB00002F098FC4FF40031204614F04FF930B185
:102EC00004F5A043D3F804020368DB6B9847402164
:102ED000204614F043F968B104F59B453C3528467B
:102EE0006AF0D4FC04F5805393F9303313B12846CB
:102EF0006AF0ACFE4FF48061204614F02FF920B147
:102F000004F59B403C306AF059FD2021204614F026
:102F100025F968B104F5A045D5F8E00103681B69FF
:102F2000984780B304F5C043D3F8880CA4F0A2FC02
:102F30008021204614F012F990B332F0C3FE30F035
:102F40003DFF1021204614F009F978B104F5C04383
:102F5000D3F8840CA1F0CEFB04F55C50203085F052
:102F600019FF04F559502430AEF0EAF84FF6FF711E
:102F7000204614F0F3F810B304F59540BDE838404E
:102F80004030B0F0C9BB20460EF0F0FC0028C9D19B
:102F9000D5F8E00103685B6998470028C2D0C7E70D
:102FA0004FF48021204614F0D9F80028C5D14FF401
:102FB0000021204614F0D2F80028BED1C1E738BD68
:102FC00038800030FFF74ABF10B50121044614F0E5
:102FD000C5F810B1204602F005FC8021204614F00F
:102FE000BDF848B14FF48021204614F0B7F818B965
:102FF00032F068FE30F0BEFE4FF40011204614F0AF
:10300000ADF830B104F5A150BDE81040083096F09D
:10301000F3B910BDFFF7D8BF10B5044606F08CFB1E
:10302000204606F0D5F9204606F0CEFB204606F0F5
:10303000E9FC204614F0BCFF2046BDE8104004F037
:10304000FBB80000FFF7E8BF70B504464FF6FF710C
:1030500014F084F804F5A04528B1D5F8D42107214F
:10306000204602F0F1FBD5F8043293F8D1309BB939
:103070002046FFF707FBD5F8040204F5804304F56A
:103080004052016892F88A258E6993F80411B0477E
:10309000D5F80402ABF084FB78F032FF204614F040
:1030A00085FF95F8D43104F5C044044ADB43C3F3EB
:1030B000C01384F8513F537170BD00BF65AF00303D
:1030C000FFF7C2BF70B500F5805600F5A044054675
:1030D00006F69833D3F8B823C4F81822D3F8C433CB
:1030E000C4F81C32D6F80C0F00F58C40503033F089
:1030F0009BFBD4F81832C4F820024FF6FF71C4F8D5
:1031000024322846D4F81C32C4F8283214F026F8A9
:1031100038B1D6F80C2F28460921BDE8704002F0DE
:1031200069BB70BD00F5A04330B5D3F81442002C44
:103130004ED093F8D521D1074AD56FF30002012C68
:1031400083F8D52100F5804208BFD3ED875A00F5FA
:10315000DC50D2F8AC1DD2F8B05DB1F9084018BF10
:10316000D3ED8A5A07EE104AB5F9084008BFD3EDEF
:10317000867A06EE904AB8EEC77A16BFD3ED897A02
:10318000F8EEE66AF8EEE66A25EEE66AA7EE276A4A
:1031900067EEA67AD0EDF46AE7EE257A90EDF77A3D
:1031A00027EE877AA6EE267ABDEEC77A17EE103A9A
:1031B0000B8190EDF47AD2F8B03D67EE877A90ED0E
:1031C000F77AE6EE477AFDEEE77A17EE902A1A8153
:1031D00030BD000038B5054600F5A0442DED028B4A
:1031E00071B1284613F04CF9D4F8203240F2E6329F
:1031F0001B1A03F2F31393420CD8BDEC028B38BDBB
:10320000D4F81432022BF8D113F01AF9B0F57A7F02
:10321000E7D2F2E7C4F8200200F58C406423503076
:1032200090FBF3F300EE103A9FED0A7BB8EEC00B73
:1032300020EE070BB7EEC08BB0EE480A0CF102FF90
:1032400084ED890AB0EE480A0DF13EFD84ED8A0A4C
:10325000D3E700BF000000A046DF913F00F5DC503F
:103260000121183017F022BAFFF7F8BF10B5044655
:1032700013F044FB1021204613F070FF98B1204654
:1032800002F072F94FF40011204613F067FF50B9B5
:1032900032F018FD30F060FE04F5A150BDE810409A
:1032A000083096F0A9B810BDFFF7E0BF70B504462E
:1032B00006F036FF214B4FF6FF76254604F17C00E1
:1032C00045F83C3B1E4B6465C4E916341D4BC4E90C
:1032D00018341D4BA3661FF0CBFC04F198001FF0BF
:1032E000C7FC04F1B4001FF0C3FC184B04F1D0007C
:1032F000A4F8CC60C4F8C8301FF0BAFC144B1549D0
:1033000028461D6061F08CFE04F52470A4F87460FA
:10331000A4F890601FF0ACFC04F52B701FF0A8FC23
:1033200004F532701FF0A4FC0023204684F8DC3240
:10333000C4F80033012384F8043370BD98E2130805
:103340004D2B0208512B0208552B02080000FFFFED
:103350002CAF0030B466140810B5044606F0E0FE49
:103360000A4B04F1400023600123A3871FF080FC77
:1033700004F150001FF07CFC04F160001FF078FCA9
:1033800004F170001FF074FC204610BD84ED13089A
:103390002DE9F04304462DED028B85B004F58046FF
:1033A000FFF7F2FB944B04F5565004F59E4523605D
:1033B00002AF2830303502F01DFC04F5565104F5FB
:1033C0009B4004F5A04804313C3008F148086BF0FC
:1033D0004FF804F5555304F59C4038337C30C6F85B
:1033E000683E062386F86C3E6DF058FA04F59D4061
:1033F00024306DF053FA04F59D40503079F02CFAEA
:103400002846AEF0C5FD7D4B281D3946C6F8303F35
:10341000012304F59F458DF8083062F0FFFB04F5A9
:103420009E40643568305EF045FA754BC6F8C03F83
:103430002846143572F01CF9A845F9D104F5A045C9
:103440001E2340F2CC60C5F86C310023A5F8703122
:1034500020F030F8C5F8680104F5A2407430B9F0E6
:10346000CBFD04F5A3403830B9F0C6FD654A1368BA
:103470001BB904F59F434033136004F5F148624BD8
:1034800004F5A340B7EE008A08F17008C6F8C03F03
:1034900065300026C5F8E08104F5DB49ABF04CFF50
:1034A0005A4B04F5A4404FF40071039309F16409E9
:1034B000574B303085ED868A85ED898A04F5C04505
:1034C0000294009397E80C001BF08EF904F5AE40CF
:1034D0005C30B1F0ABF904F5D840B0EE480A3030BA
:1034E0006DF0F2FA04F5D840B0EE480A48306DF0BD
:1034F000DDF904F5D84058301FF0BAFB05F66843F3
:1035000004F5D9404FF400411E605E6020309E609B
:1035100005F674431E605E609E6004F5DC5318334C
:10352000C5F8803C002385F89D3C1CF011F904F59A
:10353000D940703079F060FF04F5DA405C308BF0F0
:103540006BFB04F5DB40143062F08EFC314B04F56C
:10355000DB40C5F8943D283088F0D2FF04F5DB400D
:103560002D4B44302D49186061F05AFDFF232C4942
:10357000484685F8F43D85F8FC3D61F051FD294B46
:103580001F6817B12848BCF0C5FD04F5DC40C3F83E
:10359000009004F5DD490430A5F00CFC04F5DD4095
:1035A00009F170096830A5F0C3FA484691F0EAF9CC
:1035B00004F5DF4049464430ABF0D8FE1B4B1C48B5
:1035C0004FF0140CC5F8C43F04F5E04506232A4625
:1035D0002B76184B243218603B469FB201330CFB0C
:1035E0000701097C0029F8D1134B1F80134B1F687A
:1035F00057B31348C7E700BF2C891308B07D1308E1
:1036000034EC140830BA003084891308492B0208BE
:103610001C891308F07D1308F4BF0030FC04150862
:10362000042415088CC000302C7E13087CDA1308A3
:1036300080D013081CB0003018B00030D8AF003074
:103640004D7E1308CDCC4C3D04F5E0401FED030A40
:103650001A6004F5E84938306DF028F904F5E040C7
:10366000503006F05DFD634B04F5E1402B651030F2
:1036700006F056FD604B04F5E140C5F890304C3043
:10368000FFF714FE484606F04BFD5C4B09F13C0089
:10369000C5F80034B5F026FE594B04F5EB40C5F8EB
:1036A0003C34283006F03CFD564B04F5EB40C5F8A1
:1036B000A8356C3006F034FD534B04F5EC4085F82A
:1036C0002876C5F8EC352C3006F02AFD4F4B04F572
:1036D000EC40C5F82C36683006F022FD4C4B04F562
:1036E000ED40C5F8683605F2A4633C301E605E60AC
:1036F0009E6006F015FD474B04F5EE40C5F8F876E0
:10370000C5F8BC36043006F00BFD434B04F5EE4023
:10371000C5F84077C5F80437483006F001FD3F4B47
:1037200004F5EF40C5F84837103006F0F9FC3C4B83
:1037300004F5EF40C5F89037503006F0F1FC394BF6
:1037400004F5F040C5F8D03705F6480364301E6034
:103750005E60FFF701FE404606F0E2FC324B04F5E6
:10376000F240C5F8F0382C3010F03AFB04F5F34085
:103770004C3006F0D5FC2D4B04F5F440C5F8087A22
:10378000C5F8CC39103006F0CBFC294B04F5F440D9
:10379000A5F84C7AC5F8103A603006F0C1FC254B0C
:1037A00004F5F540C5F89C7AC5F8603A2430FFF777
:1037B000D3FD214B04F5F640C5F8A43A012334307B
:1037C00085F82D3B05F54C650BF07EFC04F5F840C3
:1037D000083011F063FC04F5F94006F0A1FC174B2A
:1037E000204645F8403C2E606E6005B0BDEC028B73
:1037F000BDE8F083F4DE130894DF130838E3130800
:10380000C4E3130808E51308A4E5130840E6130809
:10381000D4E6130814E91308B0E91308E0EA130822
:1038200074EB130810EC1308BCEE13086CE41308D7
:1038300078F2130854EA13081CEE130838F313083F
:1038400038B5054B0A4601461C68236820461D68AA
:10385000024BA847002038BD08AD0030383000309A
:1038600038B5037904463BB905682DB128462FF0D9
:1038700007FC28461FF01AFE204638BD314B70B5B4
:103880000360044600F545502C301FF0DFF804F5C6
:10389000005393F8302C42B9D3F82C5C2DB1284654
:1038A0002FF0EEFB28461FF001FE04F5D55004F57D
:1038B000815504F6D476183014359FF0B5F804F528
:1038C000B1501C30FFF7CCFF04F5B1501430FFF7B6
:1038D000C7FF04F5B1500C30FFF7C2FF04F5995053
:1038E000103079F031FCB54204D0183D28462FF055
:1038F000D3F9F8E7144B04F55860C4F8403BFFF7E0
:10390000AFFF04F67850FFF7ABFF04F55760FFF701
:10391000A7FF04F624406CF057FD04F53A606CF004
:1039200053FD0A4BC4F8AC3094F8943143B9D4F841
:1039300090512DB128462FF0A3FB28461FF0B6FD6D
:10394000204670BD68CE14089C571408080E140851
:1039500038B5114B0446036000F5C04393F8B82F07
:1039600042B9D3F8B45F2DB128462FF089FB284621
:103970001FF09CFD04F58043084AC3F8C02F04F5EE
:10398000A043D3F8680108B11FF096FD2046FFF769
:1039900075FF204638BD00BF2C89130834EC14088D
:1039A00010B5B9F00DFE064C064B18602046FFF727
:1039B000EFFC2046044A0549BDE810400CF13CBB31
:1039C0003830003008AD0030685C013051390208F1
:1039D0000120704790F888308B4286BF00EB810051
:1039E000D0F88C000020704790F888308B4286BF5A
:1039F00000EB8100D0F88C0000207047FA2070475F
:103A0000014B93F83A05704738600030034BD3F808
:103A10001402431E58425841704700BF388000309E
:103A2000034BD3F81402831E58425841704700BF1D
:103A300038800030034BD3F8040208B1A9F00CBB66
:103A400001487047388000307089130870B581696B
:103A50000446C26941F4E053534D836142F4E0539C
:103A6000C361036A43F4E050206295F8D501400732
:103A700010D541F48E3142F48E32A161E26195F8A5
:103A8000D521510706D595F8F921D2075CBF43F43B
:103A90008E332362A36943F4C043A361D5F8E001E8
:103AA00003681B6898470238192816D8DFE800F029
:103AB000740D0D0D0D0D150D1515157415740D0DD9
:103AC0000D0D740D74151515150DD4E9072342F469
:103AD000C04243F4C043E2612362344885F07AF87F
:103AE00018B1A36943F08063A361304885F01EF8E4
:103AF00018B1E36943F08063E3612C4885F072F804
:103B000018B9236A43F080632362294B1E6846B1CB
:103B10001921304662F042FD18B1A36943F4807365
:103B2000A361244B93F8703EDB070DD5E36943F4A2
:103B30008073E36146B11921304662F067FD18B128
:103B4000236A43F4807323621B4B93F9042E8AB1DA
:103B5000D4E9061242F0800241F08001E261A161E5
:103B600093F9042E32B193F8DC3E1BB1236A43F083
:103B700080032362A36943F08043A361E36943F0B8
:103B80008043E361D5F8043293F8C9301BB9236A46
:103B900043F08043236270BDE36943F40053E36163
:103BA000236A43F4005397E73880003058670030A9
:103BB00028B00030387000303890003013B54FF422
:103BC000F470CDE900211FF06BFC044628B1DDE95B
:103BD000002175F035F8024B2360204602B010BD7D
:103BE000CC8B1308002070477047000003207047FB
:103BF00010B5154CD4F8E00103681B6898470728F6
:103C00001CD8032834BF10231823D4F8042243F00F
:103C1000400022B192F8D1200AB143F0C00040F038
:103C2000010010BD0B280DD8DFE800F006060C06D9
:103C30000C060C060C0C0C061823E6E71038C3B271
:103C40000B2BEFD91023E0E738800030014B93F8BD
:103C50003C05704738600030034B93F9F80000389A
:103C600018BF0120704700BF38700030014B93F936
:103C70003E057047386000307047000038B5C578A1
:103C80000B4604463522352D4FF00001184628BF5B
:103C9000352510F1C1F804F10C012A46BDE8384081
:103CA00010F170B81FB5184C94F8661E04F55160F9
:103CB00014F036FD78B194F8661E04F5516014F0E6
:103CC0009DFF40B194F8661E04F5516004B0BDE854
:103CD000104014F0DBBF002301930293039317F00D
:103CE000F1FD01A916F06EF820B101A838F0CCFC66
:103CF00004B010BD27F01EF8B02290F8E03202FBAD
:103D0000030090ED370AF3E73850003008B50D4B4B
:103D1000D3F80402A8B144306CF070FE0346B7EE4D
:103D2000001A9C2093ED000ADFED070A32F0AEFD89
:103D3000DFED067A20EE270ABDEEC00A10EE103A3B
:103D400018B208BD38800030000000000000C842F2
:103D50002DE9F04FDFF8DC808DB00446344F0425A8
:103D600008F5405617F8019BB8F9943509F1FF3A68
:103D700043FA0AF3D90744D5207C6EF0F7FA83465C
:103D8000207C6FF031FA00F121039B4505D2207CA5
:103D90000DB0BDE8F04F6DF00DBDBAF1030F30D896
:103DA000DFE80AF002363B40D6F8840C03689B68D3
:103DB000984700F18C03D3F800B0D3F804A0D3F8EF
:103DC0000CC018695969D3F818E0DA691B6ACDF894
:103DD00029206222CDF82530212307900891C221A5
:103DE000207CCDF80CB0CDF810A0CDF814E0CDF8C3
:103DF00018C08DF82490CDE90032192303AA6EF083
:103E000033FB013D15F0FF05ACD10DB0BDE8F08FDF
:103E1000D6F8840C0368DB68CAE7D6F8840C03681C
:103E20001B69C5E7D6F8883C03F5FE73C3E700BFFE
:103E3000B88C13083860003007B50190AFF07AFCF9
:103E400028B1019903B05DF804EBAFF035BC03B0C5
:103E50005DF804FB014809F08FB900BF04A10030F0
:103E60000B4B70B5D3F8FC3005460E461446DB0705
:103E700003D511460748ABF037FE21460648B0F09F
:103E80003DF8224631462846BDE8704073F0F2BD49
:103E900038700030FC9F0030207B003010B588B0B7
:103EA000044670F0BFFE0C4BD3F8040238B90B4A3D
:103EB0000621204608B0BDE8104070F09DBD69465F
:103EC0001E22A9F0CDF86B46054A0621204670F067
:103ED00093FD08B010BD00BF38800030BC891308C6
:103EE000EADC1308034A92F8A83D013382F8A83DA2
:103EF0006FF038BE387000300148A5F08BB900BFB4
:103F00003C9E003007B5084601911EF085FF38B190
:103F10000448019902F0B2FF002003B05DF804FBF1
:103F20000420FAE70CAD0030014803F08FBD00BF5C
:103F300038300030014803F037BD00BF3830003062
:103F400070B58B8B06460C46CD2B15D10D4D95F8D3
:103F5000511D05F54F6079F085FA68B195F8511D4E
:103F600005F54F6079F086FA30B9DFED070A94ED78
:103F7000020A064802F062FF21463046BDE8704062
:103F80006FF00ABE38900030000000000CAD003029
:103F900008B56FF09FFD40F41C6040F00D0008BDB7
:103FA00000B5002389B0029303930493059306930D
:103FB000079317F087FC02A915F004FFB0B117F0C2
:103FC00081FC15F0E7FE05A88DED050ACDED060A8A
:103FD0008DED071A38F058FBF1EE047A20EE270A2F
:103FE000FCEEC07ACDED017A9DF8040009B05DF8D1
:103FF00004FB000010B504461FF058FA204610BD1F
:1040000010B50C4C94F9D431002B0FDBD4F8E0013F
:1040100003685B6C984758B9D4F8E00103681B6CDF
:10402000984700280CBF0220032010BD0120FCE7A8
:104030000420FAE73880003008B5134B93F8D50117
:1040400010F020001ED0D3F8E00103685B6D9847A4
:1040500007EE900AF2EE046AB8EE677ADFED0B7AAB
:1040600027EE277ADFED0A7AB4EEE77AF1EE10FA5E
:1040700058BFB0EE677AC7EE267AFCEEE77A17EE05
:10408000903A98B208BD00BF388000300AD7233C70
:1040900000FF7F4737B5F7EE000A91ED050A019260
:1040A00004460D4632F08CFA019A30B1214606489A
:1040B00003B0BDE8304003F0FDBC2946204603B004
:1040C000BDE8304072F0AABC383000302DE9F34131
:1040D000B1F9043006460C461546002B35DB1C4F63
:1040E0004FF000089FED1B0A4FF47A73CDE90028CA
:1040F000B1F90220D7F8AC1D73F0E6FF01239FED64
:10410000150A3046B4F90020D7F8B01DCDE90053A8
:104110004FF47A7373F0D8FF9FED0F0A4346B4F95A
:104120000420D7F8B41D3046CDE9005873F0CCFF19
:104130009FED080A4FF47A73B4F90620D7F8B81D3A
:104140003046CDE9005873F0BFFF02B0BDE8F08102
:10415000387000300000FA4400007A4408B5094B7A
:1041600093F8D50110F020000AD0D3F8E0010368DD
:104170001B6D984732F058FBC82390FBF3F0C0B298
:1041800008BD00BF3880003000B5002389B002931D
:104190000393049317F096FB02A915F013FED8B110
:1041A00017F090FB15F0F6FDF0EE607AF1EE400AA4
:1041B000B1EE670A0CF184FFDFED097A20EE270AE1
:1041C00032F0B4FAF6EE007A20EE270AFCEEC07A5E
:1041D000CDED017A9DF8040009B05DF804FB00BF45
:1041E000E02E6542124B07B593F8D50110F0200080
:1041F0001AD003F58053D3F8880C00F52B7038F0F3
:1042000043FADFED0C7A20EE270ADFED0B7AB4EEED
:10421000E70AF1EE10FA58BFB0EE670AFCEEC07A7A
:10422000CDED017A9DF8040003B05DF804FB00BFFA
:1042300038800030CDCC4C3D00007F43044B1878D3
:1042400020B9044B93F8D601C0F38010704700BF2B
:104250007CAE003038800030084B93F8592752B9B3
:1042600093F8F921920606D193F9D431002BACBF13
:104270000420032070470520704700BF38800030BD
:1042800008B5074B93F98835032B03D0BDE80840E8
:1042900070F0CABB034A022170F0AEFB042008BDD7
:1042A00038600030D4891308094BD3F8FC209207FA
:1042B00001D46FF0E5B903F50053DFED067A03F69C
:1042C0005C4393ED000AB8EEC00A20EE270A70475F
:1042D000387000300AD7233C10B594B0044603A8C8
:1042E0001EF0C6FC1C4B03A9D3F8E0010368DB6C8D
:1042F000984778B3002103A81EF052FD50B3247CE8
:10430000BBF03AFF059B9622DDED047A5721089316
:10431000069BF8EEE77A9FED117A0993002367EE8A
:10432000877A07900B9320460C930D930E930F936F
:104330001093119312934FF6F853CDED0A7AADF81E
:104340004C3000238DF84E303323CDE9003207AADC
:104350006EF08AF814B010BD388000300AD7233CC4
:1043600030B5844C05462DED0A8BD4F8E00199B0A8
:1043700003685B6A9847002867D004F50054D4F8B6
:104380004037062B00F2E180DFE803F00404046309
:10439000A0C35F00784840F6F8540CF0C5FD9FEDCF
:1043A000778A9FED770AF0EE489AB0EE48AAF0EED1
:1043B000488AF0EE48AAB0EE48BA90ED027B90ED44
:1043C000005BF7EEC76BB7EEC55B90ED047B0BA807
:1043D0008DED0B5ACDED0C6AB7EEC77B8DED0D7AE6
:1043E00037F034FDB0EE40CAF0EE60BAB0EE419A5C
:1043F0002D7CBBF0C1FE00238C22B1EE499A0B90BC
:104400001593F1EE688A16930123B1EE488A55217F
:104410008DF85E30332328468DED0CCACDED0DBAF4
:104420008DED0E9A8DED0FBACDED10AACDED118A5E
:104430008DED12AACDED139A8DED148AADF85C4086
:10444000CDE900320BAA6EF00FF819B0BDEC0A8B63
:1044500030BD49484FF440640CF066FD9FED480ABA
:1044600090ED027B90ED005BF7EEC76BB7EEC55B9E
:1044700090ED047B0BA88DED0B5ACDED0C6AB7EED9
:10448000C77B8DED0D7A37F0E1FC3B48F0EE60BA6A
:10449000B0EE419AB0EE40CA0CF04AFD9FED380AEA
:1044A00037F0D4FC3448B0EE40BAF0EE60AAF0EE3B
:1044B000418A0CF041FD9FED320A37F0C7FCF0EE67
:1044C000609AB0EE40AAB0EE418A91E72A4840F6E1
:1044D00007440CF02DFD9FED2A0A37F0B7FC264863
:1044E000B0EE40BA9FED259AF0EE60AAF0EE418A58
:1044F0000CF022FD9FED220AF0EE49BA37F0A6FC3F
:10450000B0EE49CAB0EE40AAF0EE609AB0EE418A31
:104510006EE7194840F63F44DFED188A0CF00CFDB9
:104520009FED170A37F092FCF0EE68AAB0EE40AAB1
:10453000F0EE609AB0EE418AB0EE68BAB0EE689ADA
:10454000F0EE68BAB0EE68CA52E79FED0C8A00241C
:10455000F0EE489AB0EE48AAF0EE488AF0EE48AA8B
:10456000B0EE48BAB0EE489AF0EE48BAB0EE48CA9B
:104570003EE700BF388000303CA70030000000005C
:104580000AD7233C2DE9F041414D04462DED088B1F
:1045900095F8D5318CB0990675D505F58057DFEDC6
:1045A0003D8A9FED3D0AD7F8840C483037F04EFC29
:1045B0008DED041A21EE281AD5F8E061CDED030A3D
:1045C00020EEA8AA8DED020A3046BDEEC11A94F87D
:1045D000108060EE28AA11EE103A1DB233681B6DF0
:1045E000984707EE900A3046F8EEE77A67EEA87A29
:1045F000FDEEE77A17EE903A1CB233685B6D984790
:1046000007EE900AD7F8883CB8EE678ADFED237A88
:10461000986828EE288A93EDA69BB4EEE78AF1EE1F
:1046200010FA58BFB0EE678AA7F082FC3368B0EE8C
:1046300040BA30469B6D9847B7EECBBABCEEC88AFD
:104640000023B72220EE280A39EE4B9B089318EE80
:10465000103A3E214046CDED05AAB7EEC99BADF814
:104660002C301A238DED06AA8DED090A29EE289A21
:10467000ADF82850ADF82A40CDE9003205AA8DEDFD
:10468000079A6DF0F1FE0CB0BDEC088BBDE8F0812F
:10469000388000300AD7233C9F0CB34500FF7F478A
:1046A0001B4B2DE9F04F2DED028BD3F8843C8DB0E0
:1046B000047CD3F860805F6E9E6EDD6E93ED1C8A85
:1046C000D3F874B0D3F878A0D3F8B890BBF054FD09
:1046D00000231622029053218DF82C3025232046EA
:1046E0008DED078ACDF820B0CDF824A0CDF8289024
:1046F000CDF80C80049705960695CDE9003202AA04
:104700006DF0B2FE0DB0BDEC028BBDE8F08F00BFC6
:104710003890003070B58A7A06464B7A0C4643EAE8
:104720000223CA7A43EA02439D2B1BD1104D95F810
:10473000511D05F54F6078F095FE98B195F8511D23
:1047400005F54F6078F096FE60B9D4ED057A9FEDDF
:10475000090AF8EEE77ADFED080A084827EE800A32
:1047600002F06CFB21463046BDE870406FF012B994
:10477000389000300AD7233C000000000CAD003018
:1047800010B52DED048B84B017F09CF804466846F4
:104790001EF06EFA6946204615F0A6FA134B93F800
:1047A000D50110F020001DD003F58053DDED017A16
:1047B000D3F8883CB8EEE79A986893EDA68BA7F0FB
:1047C000B7FBB7EEC00ADFED0A7A38EE408BB7EEE2
:1047D000C88B38EE098A28EE278ABDEEC88A18EE03
:1047E000103A18B204B0BDEC048B10BD3880003014
:1047F0000AD7233C054BD3F804322BB193F8D000F1
:10480000002808BF0220704702207047388000301F
:1048100008B5034BD3F8E00103681B68984708BD4F
:1048200038800030024B93F8D501C0F34010704738
:104830003880003070B52C4E05460C46D6F8E001A5
:104840002DED028B036886B091ED018A5B6A984773
:1048500050B9BDEEC88A18EE103ADB0704D4022026
:1048600006B0BDEC028B70BDD4E9040133F0CCFA84
:104870000028F4D002A81EF0FBF902AA214628461F
:1048800073F00AFB0028EAD0184902A81EF0D0FAFB
:1048900003460028E3D1DFED160A0246009002A984
:1048A000B0EE600A13480CF037F9D8B1D6F8E00141
:1048B00003685B6A9847044608B10020D0E70222EB
:1048C00004210D4806F02EF860B1DFED090A2346F9
:1048D000224602A9B0EE600A064800940CF01CF9CA
:1048E0000028EAD10420BBE738800030909C0030DB
:1048F000000000003CA700303830003010B5D1ED8A
:10490000007A0446FCEEE77A17EE903A13F0FF03C4
:104910000FD10F4BD3F8E00103681B6F984708B124
:10492000002010BD0B4A2046062170F065F80420D7
:10493000F7E7012B09D1064BD3F8E00103685B6F61
:1049400098470028ECD1044AEDE70220E9E700BFD0
:1049500038800030F8891308088A13088A8B82B0DF
:10496000C02A1DD0C12A1ED0202A1FD1D1ED007A25
:10497000F5EEC07AF1EE10FA1BDD9FED0F7AF4EE42
:10498000C77AF1EE10FA14D8FCEEE77A0B4A002051
:10499000CDED017A9DF80430A2F8EA3A02B07047F2
:1049A00002B0FFF747BF02B0FFF7A8BF02B073F035
:1049B0006BBB0320F2E700BF00007F43387000307C
:1049C00010B5002304462DED028B8CB003930493A5
:1049D000059316F077FF03A915F0F4F950B316F01C
:1049E00071FF15F0D7F9F0EE607A8DED060ACDED86
:1049F000070AF1EE400AB1EE670A247C8DED081A31
:104A00000CF15EFB06A8B0EE408A37F03DFE089B35
:104A1000DFED0A7A01220B930C2328EE278AA821C6
:104A200020468DED0A0ACDE9003209AA8DED098AEA
:104A30006DF01AFD0CB0BDEC028B10BDE02E65428E
:104A40002729F7B506460D4611D00AD819290ED0E8
:104A500024290ED02946304603B0BDE8F04073F05B
:104A6000D3BD372912D0A1F13903012BF2D801248B
:104A700005E00C216CF0B0FE044618B90024204675
:104A800003B0F0BD3046FFF79BFFF8E726216CF03E
:104A9000A3FE04460028F1D0317C104890F0B8F80D
:104AA0000F4B1F68002FEAD0262130466CF094FE91
:104AB00004460028E3D000230DF1060229463046C3
:104AC000ADF8063071F030F90028D8D0BDF80620D6
:104AD0003846317C8DF056FAD1E700BF289F003070
:104AE00088C0003070B52DED028B8B8B90B00446E2
:104AF0000E46C12B00F0208260D8542B00F0C980F4
:104B000017D8162B09D8102B0AD9113B052B07D81B
:104B1000DFE803F0DA0606E0E3BF202B00F0E080D8
:104B20003146204610B0BDEC028BBDE8704074F0F9
:104B30004BBDB22B00F0F98039D8552B00F0CD8059
:104B4000732BEDD1D1ED007AF5EEC07AF1EE10FACB
:104B5000C0F2E5809FEDBA7AF4EEC77AF1EE10FA72
:104B600000F2DD8091ED030A9FEDB68AF0EEC07A87
:104B7000F4EEC87AF1EE10FA40F1CA80D6ED037A6D
:104B8000D6ED010AF4EEC87AD6ED027A96ED000A67
:104B9000FDEEE77AAC48F1EE10FACDED037AACBF4A
:104BA000012200229DF90C1002F0D8F88AE0BD2BFA
:104BB000B6D10221A54807F0D3F882E04AF21142AB
:104BC000934200F0288141D8B3F5967F00F0D2805F
:104BD00027D8D02B00F0E380D12BA1D1D1ED017AE1
:104BE000FCEEE77ACDED037AD1ED007AFCEEE77AC0
:104BF000CDED047AD1ED047A9DF81020FCEEE77A31
:104C0000CDED057A9DF8143000939DF80C30D1ED70
:104C1000030A91ED020A01468D4811F0BDF90446E0
:104C20007EE040F6D81293427FF47AAFD1ED017A5C
:104C3000FCEEE77ACDED037A9DF80C30012B40F0C5
:104C4000E880002183488DF073FB3BE04AF2134279
:104C5000934200F030814AF26862934200F0B580DE
:104C60004AF2124293427FF45BAF7B4D95F8F941D3
:104C700014F0010426D1D5F8043293F8D130002B7A
:104C800040F0FC800122A5F1D0001146FDF74CFB5D
:104C900046E0D6ED027A9FED6B7AF0EEE77A96ED7C
:104CA000060A6D4BF4EEC77ADFED6C7AD3F8E001BB
:104CB00020EE270AF1EE10FA4CBF0121002112F07C
:104CC00087FD60B300242BE002220521604805F037
:104CD00029FEF6E702220621F8E702220921F5E77C
:104CE000D1ED007AF5EEC07AF1EE10FA17DD9FED06
:104CF0005C7AF4EEC77AF1EE10FA10D8FCEEE77A9F
:104D0000584ACDED037A9DF80C30A2F8EA3AD9E77B
:104D1000F7EE000A31F054FC00287FF42FAF042492
:104D2000204610B0BDEC028B70BD91ED010AB5EECE
:104D3000C00AF1EE10FAF2DD9FED487AD1ED007A6B
:104D400020EE070A9FED487A434BF4EEC77AD3F87A
:104D5000E001F1EE10FA036802DD5B6E9847B0E700
:104D60009FED427AF4EEC77AF1EE10FACCBF1B6EDB
:104D7000DB6DF3E702220321354805F0D3FD00285F
:104D8000CDD033480121FDF70BFC394890F80C31A8
:104D9000012B97D000F584703AF04AFC92E7D1EDF0
:104DA000007AFCEEE77A17EE903A99B2012904D026
:104DB000022906D00029B2D100212E487DF0D6F973
:104DC00080E7234803F07CFC7CE72B48AEF006FC30
:104DD0000028A4D0D6ED017AFCEEE77ACDED037A77
:104DE0009DF80C40012C08D0022C0CD0002C96D140
:104DF0001C4B002283F8CC2A92E796ED020A1E484B
:104E0000AEF02EFC5EE796ED030A1B48AEF03CFCCC
:104E100058E7012116E7104890F8F931DB073FF514
:104E200051AF02220521A0F5A04005F07BFD00282E
:104E30007FF448AF02220648114605F073FD41E7B2
:104E40000000B443000000340CAD003004A1003079
:104E5000383000301C9E0030388000300000C842DE
:104E600000007F43387000309A9939403333F33F64
:104E700038A00030FC9D0030F87A003095F9D4312C
:104E80000222002B12DA0521304805F04BFD0028E4
:104E90003FF418AF96ED000A0121DFED2D7AD5F829
:104EA000E00120EE270A12F093FC39E70921274898
:104EB00005F038FD34E7274D95F8F94114F0010469
:104EC0007FF400AFD5F8043293F8D130002B3FF4D3
:104ED000F9AE95F9D431002B06DA01220821A5F1AB
:104EE000D000FDF7DBFA1BE7D1ED007A9FED1A7ACF
:104EF000F0EEE77AF4EEC77AF1EE10FA0CD5022262
:104F00001121124805F00EFD002893D040F6C4117F
:104F1000124809F0A7FA03E7D5F8E00103681B6817
:104F2000984704283FF4CEAED5F8E00103681B682B
:104F300098471428E3D1C5E607A93046032271F04B
:104F40004BFF07A92046FFF7D9FC68E63830003050
:104F50000000C8423880003000000034E0A5003076
:104F6000F6EE007A08B591ED007AB4EEE77AF1EE4C
:104F700010FA06DD012205210348FDF78FFA002013
:104F800008BD0420FCE700BF687F00302DE9F04732
:104F90002DED028B8A7AA2B04B7A05460C4643EA85
:104FA0000223CA7A43EA0243562B00F0D8810DD877
:104FB000522B21D0542B00F0AF802146284622B03E
:104FC000BDEC028BBDE8F04774F0E0BC872B11D834
:104FD000852B6CD86D2BF0D10821BB4812F0BEF8A0
:104FE00021460246284622B0BDEC028BBDE8F047C0
:104FF0006FF098BEA62BEEE7CD782722002114A8EB
:10500000272D28BF27250EF107FF04F10C0114A856
:105010002A460EF1B7FEAD4BD3F8E00103685B6A98
:105020009847002843D09DF876506A063FD44FF049
:105030007E53002410932B0613941294119429D5B7
:1050400010A835F0B3FFA2480BF0A4FA9DED1C0A9E
:105050000646002830D0B7EE001A40F28D40FFEE31
:10506000000A31F013FCEF070C940D940CAA58BF02
:10507000199B10A90E9458BF0C93AC075CBF1A9BE8
:105080000D93680792485CBF1B9B0E9333460BF051
:1050900089FA0CE0159B10A81093169B1193179B8F
:1050A0001293189B139335F087FF0028CBD122B0C1
:1050B000BDEC028BBDE8F087DFED8A0AB7EE001A7F
:1050C0004FF4926031F0E2FBF6EE000AB0EE408A57
:1050D00031F076FAE8B9B6EE000A7E4BD3F88C3C94
:1050E000B4EEC08AF1EE10FA08DD38EE400A30EE78
:1050F000008A93ED070A28EE000AB4E730EE480A6A
:10510000D3ED087AF0EEE77A30EE000A27EEC00A17
:10511000A9E79FED740AA6E7204614A9FEF7AEFDA5
:105120006A4BD3F8E00103685B6A98470028BED059
:105130009DF88420012A07D0D31F022B04D9012116
:1051400063480BF0C5F9B2E7BDF88030990503F06C
:10515000070703F0380803F4E07603F4806503F4EE
:10516000006401D5002EA2D04FF00009CDF82490A4
:10517000CDF82890CDF82C903FBB9FED576A083AA8
:105180009DED167ADDED177A012ADDED156A27EE21
:10519000067A67EEC67A66EE866A8DED0A7ACDEDFE
:1051A0000B7ACDED096A04D80AAA09A94648FDF789
:1051B00077FB9DF88430073B022B06D84748A6F0C2
:1051C000B3FE014609A836F061FECDF83090CDF867
:1051D0003490CDF83890B8F1000F1DD19DF884308F
:1051E0009FED3D6A9DED197A083BDDED1A7ADDED04
:1051F000186A27EE067A67EEC67A012B66EE866A93
:105200008DED0D7ACDED0E7ACDED0C6A04D80DAA98
:105210000CA92D48FDF744FBCDF84090CDF8449003
:10522000CDF84890EEB99DF884309FED2B6A9DED46
:105230001C7A083BDDED1D7ADDED1B6A27EE067A50
:1052400067EEC67A012B66EE866A8DED117ACDED9A
:10525000127ACDED106A04D811AA10A91A48FDF7E8
:105260001FFB002D40D1DFED1E7A9DED1E0A9DF83B
:10527000843020EE270ADFED187A083B012B20EE60
:10528000270A8CBF0023012394BBDFED157ADDEDE7
:105290001F0A60EEA70ADFED107A60EEA70A57BB7F
:1052A000B8F1000F4BD1B4FA84F4B5FA85F5029346
:1052B0000CAA640910AB6D0909A901940095044872
:1052C0000BF02AFDF3E600BF3830003038800030A4
:1052D0003CA70030389000300000C842A09C00304D
:1052E000E02E65420000000000231FED020ACBE71C
:1052F0005FED040AD3E7B8F1000F0FD10122B4FA31
:1053000084F40CA96409CDE90132B5FA85F310AA39
:1053100000945B098F480BF09FFAC8E6002E7FF4DB
:105320000EAF012210A9CDE90032B4FA84F3B5FA28
:1053300085F25B09520987480BF024FAB7E6002E84
:105340003FF4FDAEB5FA85F209A982485209CDE9CC
:105350000037B4FA84F35B090BF0FCFAA7E62046A9
:1053600014A9FEF78BFC7C4BD3F8E00103685B6A61
:10537000984700283FF49BAEBDF88040A30504F495
:10538000E07702D5002F3FF492AE0CAE04F0070890
:1053900030461DF06DFCB8F1000F25D1DDE9150197
:1053A00032F032FD00283FF4CAAE09AA9DF88410FD
:1053B000284672F05BFD00283FF4C1AEDDED177AA0
:1053C00010AD9FED667A099B284667EE877A0093B9
:1053D000FDEEE77ADDE9151217EE903A1DF068FC54
:1053E00095E80F0086E80F00002514F0380A0695AE
:1053F0000795089513D19FED596A9DED197ADDED5A
:105400001A7ADDED186A27EE067A67EEC67A66EE3E
:10541000866A8DED077ACDED087ACDED066A09959D
:105420000A950B959FB99FED4D6A9DED1C7ADDEDB8
:105430001D7ADDED1B6A27EE067A67EEC67A66EE08
:10544000866A8DED0A7ACDED0B7ACDED096A14F4FA
:10545000806905BFDFED427A9DED1E0A9FED410A8E
:1054600020EE270A04BFDFED3D7A20EE270A14F470
:10547000006405BFDFED3A7ADDED1F0ADFED390A82
:1054800060EEA70A04BFDFED357A60EEA70AB8F137
:10549000000F31D1BAF1000F4CD13046CDED050AE5
:1054A0008DED040A1DF014FC03289DED040ADDEDCA
:1054B000050A3FF444AE10A93046CDED050A8DED46
:1054C000040A1095119512951DF064FD00283FF413
:1054D00036AEB4FA84F4B9FA89F3DDED050A06AA0A
:1054E00064099DED040A5B0910A9CDF804A000949D
:1054F00018480BF087FCDAE5BAF1000F0CD1012354
:10550000B4FA84F409AA06A96409CDE901A3B9FA99
:1055100089F300945B09FDE6002F7FF410AE0123B0
:10552000B9FA89F209A95209CDE90073B4FA84F3F2
:105530005B0900E7002F3FF402AEB4FA84F3B9FA36
:1055400089F23146CDF800805B09024852090BF020
:10555000E3FAACE53CA70030388000300000C842D8
:10556000E02E6542000000002DE9F04300F5A04662
:105570000446002704F5C0492DED028BD6F8E00162
:1055800091B0DFED4B8A03685B699847002840F0D3
:105590008A80D9F8883C93EDA67BB7EEC77BD3ED24
:1055A000AD7AFDEEE77A27EE288A17EE903A1DB223
:1055B00004F59D4801A908F14008404611F074FC2B
:1055C00018B969F081FE3B4B01933722002102A8F4
:1055D0000EF122FCA3238DF8083095238DF80930B5
:1055E000BAF0D2FDD9F8843CCDF80B00D6F804020D
:1055F000D3F8B820D3F8BC304430CDF80F10CDF834
:105600001320CDF817306BF0F9F90346B7EE001A06
:10561000DFED290A9C2093ED000A31F037F9D6F826
:10562000040210EE103A04F5D846CDF81B30683667
:1056300003689B68984710EE103A3046CDF81F304B
:1056400018EE103ACDF82330A6F072FC20EE280AAE
:10565000404610EE103ACDF82730D9F82C3CCDF862
:105660002B30019BCDF82F3011F044FC10EE103A96
:105670003046CDF83770CDF83330ADF83B50A6F05A
:1056800063FCBDEEC00A04F59B40372202A93C3002
:1056900010EE103AADF83D3068F0BCFF11B0BDEC33
:1056A000028BBDE8F083002508EE107A80E700BF8A
:1056B0000AD7233C2292CA7F0000000070B500F593
:1056C000C04604468AB09FED190AD6F8840C01AD95
:1056D000483036F0BBFB0AAACDED080A04AB8DEDCD
:1056E000091A8DED070A12E9070085E807009DED0C
:1056F000030A83E8070031F057F804F5DC50294627
:105700008DED030A183013F0B9FC04F5A04104F53F
:105710008044D6F8883CD6F8842CD1F80412D4F80A
:105720002C0F13F0FFFD0AB070BD00BF9F0CB345F6
:1057300070B54FF48051054611F010FD00284FD090
:1057400005F5C04605F59B44D6F8840C3C34036847
:105750009B689847642100F18C02204668F030FD78
:10576000D6F8840C0368DB689847652100F18C0249
:10577000204668F025FDD6F8840C03681B6998471D
:10578000662100F18C02204668F01AFDD6F8882CBC
:105790006721204602F5FE7268F012FD202128469E
:1057A00011F0DCFCE0B105F5A043D3F8E00103689B
:1057B0001B69984778B1D6F8882C20466921903229
:1057C00068F0FEFCD6F8882C20466A21B832BDE885
:1057D000704068F0F5BC28460CF0C8F80028EAD103
:1057E00070BD000008B516F06DF8BDE8084016F071
:1057F00017B800007FB50E464FF6FF7104461546F8
:1058000011F0ACFCE8B11022002168460EF104FB57
:10581000A3238DF8003095238DF8013003238DF8F4
:105820000230BAF0B1FCCDF8030004F59B40CDF88E
:105830000710102269463C308DF80B60039568F024
:1058400069FF04B070BD00007FB50E464FF6FF71D2
:105850000446154611F082FCE8B11022002168468A
:105860000EF1DAFAA3238DF8003095238DF801307C
:1058700004238DF80230BAF087FCCDF8030004F55C
:105880009B40CDF80710102269463C308DF80B6024
:10589000039568F03FFF04B070BD000030B52DEDFA
:1058A000048B87B004460D46182200216846B0EEEE
:1058B000409AF0EE608AB0EE418A0EF1ADFAA32371
:1058C0008DF8003095238DF8013006238DF80230D5
:1058D000BAF05AFCCDF8030004F59B40CDF8071050
:1058E000182269463C308DF80B508DED039ACDEDB2
:1058F000048A8DED058A68F08DFE07B0BDEC048B3F
:1059000030BD000010B54FF48011044611F026FCA4
:1059100030B104F5DC50BDE81040183013F0A0BCE5
:1059200010BD00002DE9F04F2DED028B8DB08046AB
:105930002F2200216846F0EE408AB0EE608A11EE18
:1059400010BA11EE90AA12EE109A12EE907A13EE9F
:10595000106A13EE905A14EE104A0EF15DFAA3236A
:105960008DF8003095238DF8013009238DF8023031
:10597000BAF00AFC18EE903ACDF8030008F59B4007
:10598000CDF80710CDF80B302F2218EE103A6946EB
:105990003C30CDF813B0CDF80F30CDF817A0CDF8CE
:1059A0001B90CDF81F70CDF82360CDF82750CDF8AF
:1059B0002B4068F02FFE0DB0BDEC028BBDE8F08FE0
:1059C00030B52DED088B8BB004460D462822002102
:1059D0006846B0EE40BAF0EE60AAB0EE41AAF0EE32
:1059E000619AB0EE429AF0EE628AB0EE438A0EF10E
:1059F00013FAA3238DF8003095238DF801300A2384
:105A00008DF80230BAF0C0FBCDF8030004F59B40DE
:105A1000CDF80710282269463C308DF80B508DEDEB
:105A200003BACDED04AA8DED05AACDED069A8DED54
:105A3000079ACDED088A8DED098A68F0EBFD0BB071
:105A4000BDEC088B30BD00002DE9F0438FB014464B
:105A5000054689463122002101A89846DDE91676DF
:105A60000EF1DAF9A3238DF8043095238DF8053073
:105A700008238DF80630BAF087FB23683122CDF871
:105A8000070005F59B40049363683C30CDF80B108C
:105A900001A90593A3688DF80F9006933B688DF8D4
:105AA0001C80CDF81D307B68CDF82130BB68CDF867
:105AB00025303368CDF829307368CDF82D30B368C0
:105AC000CDF8313068F0A6FD0FB0BDE8F0830000DE
:105AD00070B52DED068B8CB0144605460E462C2273
:105AE000002101A8B0EE409AF0EE608AB0EE418A43
:105AF000B0EE61AAF0EE429A0EF18EF9A3238DF872
:105B0000043095238DF805300B238DF80630BAF05C
:105B10003BFBDFED1A7A2C2294ED007ACDF80700DA
:105B200005F59B4027EE277ACDF80B1029EE279A32
:105B300001A968EEA78A3C308DED077A28EE278A06
:105B400094ED017A8DF80F6027EE277A8DED049A97
:105B5000CDED058A8DED068A8DED087A94ED027AF9
:105B60008DED0AAA67EE277ACDED0B9ACDED097A75
:105B700068F050FD0CB0BDEC068B70BDE02E6542A8
:105B800030B5044689B0144B1E2204F59B45694686
:105B9000D3F804023C35A7F063FA6A460F49284659
:105BA00068F0BCFE04F5A043D3F8E00103681B686D
:105BB000984704F540530146284693F8F42268F0CC
:105BC000D1FE04F5DC50183016F0F4F804F534700A
:105BD00023F0F4FD09B030BD38800030EADC130852
:105BE00000F59B40AC2202493C3069F01FBA00BF6F
:105BF000ECB31308484B70B50446436008304FF4CB
:105C0000386592F093F904F1600086F027F80023DC
:105C1000424A04F1BC00C4F88830C4F88C30C4F89F
:105C20009030C4F8B0303E4BC4F8A8204FF080420A
:105C3000C4F8B4303B4BC4F8AC20C4F8B830AAF078
:105C4000FBFF04F5BC7082F0F9FD04F5366074F0DA
:105C500085FC354E354BC4F8603B601974F0ECFDA3
:105C600066512C35B5F5646FF7D104F5646004F521
:105C7000805676F023FB04F5A35000212C4D043010
:105C8000AAF0D8FB04F5A8501830ADF097FCC6F880
:105C9000385504F5AA50AEF05FF8A5F5DF6304F5BA
:105CA000AE50C6F8D0351C3088F00AFDA5F5027359
:105CB000D4359FED201AC6F8303704F5BA50DFED21
:105CC0001E0A9FED1E0AC6F83C579EF0AFFC9FEDE2
:105CD000191A04F5BA509FED1A0AF0EE410A18306D
:105CE0009EF0A4FC9FED131A04F5BB509FED140A1F
:105CF000F0EE410A10309EF099FC04F5BD501C30C6
:105D0000A2F08EFD20460F495FF08AF920460E4929
:105D10005FF086F9204670BDE83F00300000C841C2
:105D20000AD7233C0000E04048DA13085CDA130885
:105D30006CAB0030000000009A99993E0000B4431B
:105D400000804A4300CD130810D0130870B5ADF59C
:105D50000E7D4B4DD0224B4906465AA80EF112F843
:105D60000EAC0FCD0FC40FCD0FC40FCD0FC495E8EF
:105D70000F0084E80F0000245AABB7EE000A0021A0
:105D8000181910345EF0F4FCD02CF5D13E4B02AC67
:105D90000FCB84E80F0001A920465EF09DFC90B176
:105DA0009DF90430F0EE007ADFED386AB7EE000AB4
:105DB00007EE103AE068B8EEC77AE7EE267A80EE92
:105DC000270A5FF0BFFC00240EAB00211819103425
:105DD000B7EE000A5EF0CCFC402CF5D190222C49A5
:105DE00036A80DF1CFFF0022092136A85EF050FD44
:105DF00096F9046CD6B9274D1EAC0FCD0FC40FCD4C
:105E00000FC40FCD0FC495E80F0084E80F00324691
:105E100004211EA85EF03CFD9FED1F0A1F485FF0A5
:105E200091FCB7EE000A1E485FF08CFC1D4C06ADDD
:105E30009FED1D0A0FCC0FC594E80F0085E80F00F9
:105E4000002106A85EF094FC00219FED170A284669
:105E50005EF08EFC04F11001002460221EA80DF1FA
:105E600091FF1EABB7EE000A0021181910345EF046
:105E70007FFC602CF5D175F0ABFF0DF50E7D70BD8C
:105E800094731308C4721308D4731308CDCCCC3D9B
:105E9000E47313087474130800000000A8CB1308FF
:105EA000B7CB1308B47413080000344210B5B4B073
:105EB0000024D022074968460DF164FF0DEB040071
:105EC0001034B7EE000A00215EF052FCD02CF5D160
:105ED00034B010BD347513082DE9F04790B01D2083
:105EE0000DF1060176F03AF9002800F09E809DF849
:105EF00006301121604A0BA80133DBB28DF8063061
:105F0000B7F094F800220DF107010BA85EF08AF9B2
:105F10009DF80630594A112105460BA8B7F086F8BE
:105F200000220DF107010BA85EF07CF99DF8063008
:105F3000534A112106460BA8B7F078F800220DF15C
:105F400007010BA85EF06EF99DF806304D4A11214D
:105F500003F03F0307460BA8B7F068F800220DF1E5
:105F600007010BA85EF05EF98046002D5DD0002E83
:105F70005BD0002F59D0002857D028465EF05CFB3C
:105F8000002852D130465EF057FB00284DD13846EC
:105F90005EF052FB002848D140465EF04DFB0028E1
:105FA00043D1394C0DF10C0C0DF11C0994E80F0094
:105FB00010348CE80F0094E80F0089E80F0002A964
:105FC00060465EF089FB98B3BDF8084002A94846D8
:105FD0005EF082FB00284AD0BDF8083054BB23B3E2
:105FE00040F2E2449C420FFA84FA0FFA83F927D870
:105FF0000DF10A013046ADF80A905FF07FFE0DF119
:106000000A012846ADF80AA05FF078FE0DF10A01FA
:106010003846ADF80AA05FF071FE00230DF10A01C9
:106020004046ADF80A305FF083FE10B0BDE8F0875F
:106030000024CBE740F2D662002B08BF1346D1E71D
:106040000DF10A013046ADF80AA05FF057FE0DF1E0
:106050000A012846ADF80A905FF050FE0DF10A01E2
:106060003846ADF80A905FF049FE0123D6E7002CD0
:10607000DBD040F2D663B5E7C8CB1308D4CB130806
:10608000E0CB1308EDCB1308047613087FB5314B32
:10609000044600211E6804F55455706D38350368B8
:1060A0001B68984728465FF08FF828B104F54053E5
:1060B000B3F93835782B15D0306C274903681B6845
:1060C000984776F0ABFA5DF077FB78230DF10E017F
:1060D0002846ADF80E305FF011FE306C1F490368A2
:1060E0001B68984778230DF10E012846ADF80E3055
:1060F0005FF0E0FDBAF034F805465EF039FE0022AC
:106100000C2117485EF0C4FB2046FFF7E5FE04F5BE
:10611000555002210C305EF021FC0023012204F5D1
:10612000475145202431CDE900320E4A5EF0C4FBD0
:10613000346C23681E68BAF013F80B49421B2046E2
:10614000B0475FF071F9094A138843F001031380E7
:1061500004B070BD08AD003000CC130824CC130887
:1061600040CC13086C1C15082BCC13080CB0003065
:106170000F299DBF2C2303FB010020300020704716
:10618000014B93F97F05704738600030044BB3F83A
:106190004435DB075ABF0069C0F340100020704748
:1061A00038600030014BD3F8B80D704738700030BC
:1061B000054A92F8F93192F8F82103F001031343EC
:1061C0000CBF0120002070473880003038B50C1E0D
:1061D0002EDB184DE3B295F86C2E9A4228D3D5F8F1
:1061E000683E0122A5F58040195D04F09BFBF8B1E3
:1061F00074F0FCFA032175F0D3FBC8B974F0F6FA19
:106200000D2175F0CDFB98B9A5F58052A5F580401C
:1062100092F96435E340DB0756BF92F97E150221FF
:10622000E140BDE8384058BF01F00101FCF7CEB9AC
:1062300038BD00BF38700030022910B5044606D1C1
:10624000014601220948BDE8104004F06BBB084B31
:10625000D3F8E00103681B689847844205D174F0C5
:10626000C5FABDE8104074F07DBA10BD383000307A
:106270003880003029B1022907D1044BC3F8D81166
:106280007047024B0122C3F8D82170473880003094
:1062900031B1022907D1044B012283F8DC21704778
:1062A000014B83F8DC1170473880003000F58043E3
:1062B000DFED186A9FED187A012110B5D3F8B02DE3
:1062C0000446D3F8AC3D00F5DC50B2F90820B3F930
:1062D0000830183007EE902AF8EEE77AC7EEA60AE3
:1062E00007EE903AF8EEE77A87EEA60A60EE870AA4
:1062F00020EE070A15F09AFB68F0E6FF262168F009
:106300002BFF04F59F40054A06214030BDE81040B0
:106310006BF030B80000C84235FA8E3C3CD8130808
:1063200000F5C042002300F59F40062182F89C3C06
:10633000024A40301372024A6BF01CB865AF00305D
:1063400048D8130870B500F5C045044695F89C1C64
:10635000002957D02C4B2D4AD3F8E001904204D1AC
:10636000D3F8043293F8D13023B92046BDE8704009
:10637000FFF7D6BF264E012204F5A04395F89D0CE9
:10638000327293F9D431D0BB002B3BDB85F89D2CC6
:10639000013904F58043DFED1F6A04F5DC50C9B212
:1063A0009FED1D7A183085F89C1CB1FA81F1D3F865
:1063B000B02DD3F8AC3D4909B2F90820B3F9083043
:1063C00007EE902AF8EEE77AC7EEA60A07EE903AB3
:1063D000F8EEE77A87EEA60A60EE870A20EE070A53
:1063E00015F024FB95F89C3C63B904F59F4033728B
:1063F0000A4A06214030BDE870406AF0BBBF002B5E
:10640000C6DAB2E770BD00BF3880003028A900307E
:1064100065AF003000007A4535FA8E3C5CD8130831
:106420006D2900F3E380012901DC75F0CDB88B1EE6
:106430006B2BFAD80FF2040C5CF823F037660208D5
:106440003166020837660208376602082B640208C4
:10645000376602082B6402082B64020831660208C2
:106460002B640208376602083166020831660208AA
:106470002B6402083766020837660208376602088E
:106480002B6402082B640208316602083766020892
:10649000316602082B640208316602083166020880
:1064A0002B6402082B6402082B6402082B64020888
:1064B0002B64020831660208376602082B64020862
:1064C0002B6402082B640208376602082B6402085A
:1064D000316602082B6402082B6402083766020842
:1064E0003166020831660208376602082B6402082A
:1064F0003766020837660208376602082B6402080E
:106500002B640208376602082B6402082B64020819
:106510003766020837660208376602082B640208ED
:106520002B64020837660208376602082B640208EB
:106530002B6402082B6402082B6402082B640208F7
:106540002B640208376602083766020837660208BD
:106550003766020837660208376602082B640208AD
:1065600031660208316602082B6402082B640208B7
:106570002B6402082B6402082B6402082B640208B7
:1065800037660208316602082B6402082B64020891
:106590002B6402082B6402082B6402082B64020897
:1065A0002B6402082B6402082B6402082B64020887
:1065B0002B6402082B6402082B6402082B64020877
:1065C000376602082B6402082B6402082B64020859
:1065D0002B6402082B6402082B6402082B64020857
:1065E0002B6402082B64020831660208A1F19703AC
:1065F0000A2B3FF61AAF0A2B3FF617AF0FF2040C27
:106600005CF823F037660208376602082B6402083C
:10661000376602082B6402082B6402082B64020808
:106620002B640208316602083166020837660208E8
:10663000002374F09BBF7047632970B514468AB07D
:1066400000F3D280012905DC22460AB0BDE8704083
:1066500074F0BCBC8B1E612BF6D801A252F823F05B
:106660002D68020841680208616802086B68020828
:10667000496602089F6802084966020849660208DE
:106680005369020849660208496602084F68020811
:1066900085690208496602084D690208C169020855
:1066A000C76902084966020849660208DF690208EC
:1066B000ED690208FB69020849660208216A0208BE
:1066C000336A0208496602084966020849660208F8
:1066D0004966020849660208456A02085F6A0208BC
:1066E000496602084966020849660208656A0208A6
:1066F000496602086B6A0208496602084966020890
:10670000856A0208316802088B6A0208316802084B
:106710004966020849660208496602084966020895
:106720004966020849660208FB6A020849660208CF
:1067300049660208CD690208D3690208D9690208CE
:106740004966020849660208AB6A0208B16A020893
:106750004966020849660208496602084966020855
:106760004966020849660208E96A0208EF6A0208F7
:10677000F56A0208316B0208376B02083D6B0208AC
:1067800049660208856B0208436B020849660208E5
:106790004966020849660208496602084966020815
:1067A00049660208AB6B0208C96B02084966020819
:1067B00049660208496602084966020849660208F5
:1067C00049660208496602084966020849660208E5
:1067D00049660208496602084966020849660208D5
:1067E00049660208DF6B0208A1F197030A2B3FF606
:1067F0002BAF0A2B3FF628AF01A252F823F000BFBF
:10680000E56B0208EB6B020849660208FF6B0208A1
:106810004966020849660208496602084966020894
:10682000D76B0208236C020831680208022C01D0E1
:10683000012431E001220E21B14804F073F8F7E79A
:10684000211E18BF0121AE48FBF7C0FEF0E7012C66
:1068500004D0022C14BF00210221F4E72146F2E704
:1068600021460620FFF7E8FCE2E7022CE0D1A54D27
:10687000D5F8E0010368DB6A984704460028D7D0C2
:10688000A5F58053D3F8B43DB3F90830002BCFD130
:10689000A5F5A040FFF70AFD20460AB070BD022C06
:1068A000C6D1984E984AD6F8E0119142C0D0D6F899
:1068B000042292F8D120002ABAD006F50054A6F599
:1068C0008056B4F938212AB9D6F8B43DB3F9083066
:1068D000002BADD005AD1C22002103A80DF19CFAC0
:1068E00028461CF0C5F9B4F93831884C93B9162301
:1068F00003A98748ADF80E30D4F85C3C642BB8BFD0
:106900006423069336F01AFD20B168F0DDFC2721E0
:1069100068F022FC04F658430FCB85E80F00D6F848
:10692000B43D03A97A48B3F90830002BCCBF10233B
:106930001523ADF80E3036F001FD00283FF478AF96
:1069400068F0C2FC272168F007FC71E721460320AC
:1069500088E7022C6F4D06D095F8703E6FF3000368
:1069600085F8703E64E71921A5F53E505FF016FEEC
:1069700004460028F0D095F8703E43F0010385F8F6
:10698000703E89E7012C0BD0022C12D0002C7FF432
:106990004FAF614B83F8A44568F096FC2B21D2E7FA
:1069A0005D4B83F8A44568F08FFC2C2168F0D4FB84
:1069B00072E7594B83F8A44568F086FC2D21C2E7A5
:1069C00021460F204EE7214609204BE721460420AF
:1069D00048E72146052045E72146172042E7A01E4B
:1069E000414241414D487BF0C1FB21E7022C7FF43D
:1069F0001FAF434801F064FE1AE7012C06D0022CB9
:106A000009D0002C7FF414AF2146EBE72146434820
:106A10007BF0ACFB40E7012140487BF0A7FBE8E7B7
:106A2000A21E3A4B5442D3F8843C544183F8204090
:106A3000FEE6A31E59425941344BD3F8840C9FF013
:106A40006BFEF5E6013C2F4B012C93F8D6218CBF51
:106A50000024012464F3041283F8D621E8E62146D9
:106A60001120FFE621461220FCE6012234B1022C5F
:106A70007FF4DEAE2A4B83F8CC27D9E6284B83F887
:106A8000CC47D5E621461520ECE6012C08D9022C8E
:106A90007FF4CEAE9FED230A2348ACF0F5FDC7E6A8
:106AA0001C4B002283F8CC2AC2E621461820D9E6E6
:106AB000144BD3F8E0011D4B98427FF4B9AE01901E
:106AC0000EF090FE012C019808D0022C0AD0002C68
:106AD0007FF4AEAE21460EF027FFA9E600210EF0AE
:106AE00099FED9E60121F6E721460020BAE62146C3
:106AF0001020B7E621460220B4E621460120B1E687
:106B0000383000303880003004A100303890003038
:106B100040A100303870003038600030FC9D0030FB
:106B200038A0003000000000F87A003040AC00309F
:106B30002146162096E62146072093E621460B20A3
:106B400090E6022C3D4B0ED1012483F8344068F0CE
:106B5000BBFB4A2168F000FB71F010FC384A0621AB
:106B60006AF008FC98E6002283F8342068F0ACFB59
:106B70004B2168F0F1FA71F001FC324A06216AF00B
:106B8000F9FB55E6012C09D0022C0CD0002C7FF427
:106B90004FAE01212C4810F0C3F949E600212A48E4
:106BA00010F0BEF978E62146F4E7284BD3F8E0016F
:106BB000274B98427FF43CAE022C02D10EF098FF96
:106BC00036E60EF0A5FE33E62146FFF753FB2148DB
:106BD00004F0A0FB2CE62146FFF75AFB28E62146ED
:106BE0001B203FE621461C203CE6022C7FF420AE11
:106BF0001948FCF767FA71F0C1FB184ABEE7214655
:106C000074F088F81648ABF0FBF9044600283FF40E
:106C10000FAE0E4A92F8D73143F0020382F8D73113
:106C20003AE6012234B1022C7FF402AE0D4B83F818
:106C3000902DFDE50B4B83F8904DF9E538A0003021
:106C400074D8130885D81308F87E003038800030D7
:106C500040AC003088A000303830003097D813089E
:106C6000687F00303870003010B504460448A5F045
:106C70005DF904F10801BDE8104031F043B800BFF0
:106C8000A09C003038B5044614482DED028BA5F0C9
:106C900053F9054633F010F91148B0EE408A10F070
:106CA000F7F9B0B1DFED0F7AB4EEE78AF1EE10FA42
:106CB0000FDDD5ED000A95ED010A0AF101FADFEDCD
:106CC0000A7A20EE270ADFED097A20EE270A84ED02
:106CD000080A94ED080ABDEC028B38BDA09C003078
:106CE0003830003000401C46E02E65420000C842AB
:106CF000074B93F96505022805D0032806D0003814
:106D000018BF0120704781F00100704704207047D0
:106D10003860003003688B4212D00429C0E90013A8
:106D200002D007290AD07047064B03F60C73D3ED47
:106D3000007AF8EEE77AC0ED087A704700238362A4
:106D4000704700BF38400030024608B5FFF7D0FF5B
:106D500001461046BDE80840FFF7DCBF70B50446A9
:106D600016460D462DED048BF0EE408A9FED2E9ACF
:106D7000B0EE608ADFED2D9AB9F0FEF9E06116B34E
:106D800068EE898A002DB7EE000AFFEE007A20FE39
:106D9000270A68EE808AC4ED058AB4EEE98A244B9E
:106DA000D3F8840CF1EE10FA30DA9DF01BFD20EEE2
:106DB000090A84ED060A20460321BDEC048BBDE8D8
:106DC0007040FFF7A7BF94ED090A98EE890A2FF0EB
:106DD00001FD002D84ED050A0BDAB4EEE90AF1EEAF
:106DE00010FADADBDFED137A30EE670A84ED050A7C
:106DF000D3E7D2D0DFED107AB4EEE70AF1EE10FA65
:106E0000CBD8DFED0C7A30EE270AEFE79DF0EAFCF5
:106E1000B4EE480AF1EE10FA48BFB0EE408A28EE10
:106E2000098A84ED068AC6E70000C84200000034E3
:106E30003890003000A00C47000000B410B52DEDD4
:106E4000028BF0EE408A0446B0EE608AB9F094F905
:106E5000DFED090A0621E061204668EEA08A68EEAF
:106E6000200AC4ED098AC4ED0A0ABDEC028BBDE814
:106E70001040FFF74FBF00BF0000C84270B54B681D
:106E800006460C46184DB3B98B68A3B9C96891B9C9
:106E90001648FFF759FF95F8511D05F54F6076F03C
:106EA000F5FA04281FD195F8511D05F54F60BDE88E
:106EB000704076F0F5BA95F8511D0D4876F0DAFA83
:106EC00048B906F1080120461CF064F818B1022107
:106ED0000648FFF71FFF224695F8511D0448BDE8FC
:106EE000704076F087BB70BD389000300CAD00303C
:106EF000289D0030072108B5FFF70CFF80ED0A0A36
:106F000008BD000008B50368032B23D1D0ED057A36
:106F10009FED127AF0EEE77AF4EEC77AF1EE10FA0E
:106F20001AD50F4B90ED090A03F60C73D3ED007AD6
:106F3000F8EEE77A37EEC00A2FF04CFCB0EEC00A4C
:106F4000DFED087AB4EEE70AF1EE10FA94BF012003
:106F5000002008BD0120FCE70020FAE70000003413
:106F6000384000300000484330B5036885B004461F
:106F7000023B082B69D8DFE803F0050D3033475D8D
:106F80003B5D5D00FFF770FE84ED090A94ED090A90
:106F900005B030BDB9F0F0F8E369DFED2F0AC31A90
:106FA000E06194ED050AE32007EE903AF8EE677A87
:106FB00067EEA07AD4ED060A20EEA71A67EEE00A83
:106FC0002FF064FCD4ED057A77EEC07AC4ED057A33
:106FD000D4ED097A37EE800AD6E7FFF753FED3E700
:106FE0001E4BD3ED8B7AF8EEE77AC0ED097ACDE748
:106FF0001B4DD5F8940CA2F0B9FE0028C6D0D5F8E8
:10700000943C1B6C6362C1E7B9F0B6F8E3699FED8D
:10701000127AC31AD4ED0A6AE06107EE903AF8EEEC
:10702000677A67EE877A94ED097AA6EEA77A84EDFF
:10703000097AABE70A4B9FED0B0AD3F8840C483072
:1070400034F004FF84ED091AA0E7054BD3F8883C1F
:10705000D3F87C32D6E700BF6F12833A3880003015
:10706000389000309F0CB3450368092B08D8DFE83F
:1070700003F0050A050505050707051000238362CF
:1070800090ED0A0A7047044BD3F8883CD3F880325D
:10709000F5E7C36AF3E700BF38900030F0B52F4D35
:1070A00004460E46D5F8E0012DED028B036889B049
:1070B0009B6F984700283ED005F58057D5F8E00132
:1070C00003F098FA08EE100AD7F8883CD7F8840C39
:1070D000D3ED9D8A0368DB6F9847D7F8883CD5F8D5
:1070E000E00178EEC00A93ED9E1A0368CDED050A23
:1070F0001B6C8DED041A98470390D5F8E0010268E7
:10710000526C9047B8EEC88A9FED150A324600903F
:1071100007A928EE000A039B9DED041AA5F5277028
:10712000DDED050AA1F094FB48B10A212046FFF7E6
:10713000F1FD079BA36209B0BDEC028BF0BD236893
:107140000A2BF8D1002361682046A36211B9FFF72A
:10715000FBFDF0E7FFF7DEFDEDE700BF3880003014
:107160000AD7233C2DE9F04100232B4E04460D465F
:10717000CB6296F8F931294F13F0010F3FD1D6F8C1
:10718000E0010368DB6E9847002838D0D6F8E0812C
:10719000A6F58056D6F8B80D73F046FC404603F0CD
:1071A00071FD85ED0B0AB0EEC00ADFED1D7AB4EE7D
:1071B000E70AF1EE10FA03D409213846FFF7AAFDD9
:1071C000D5ED0B7A2846FDEEE77A17EE903A19B224
:1071D000FFF764FF1148FFF7C7FE104884ED000A6F
:1071E000FFF742FF3B6884ED010A0A2B0FD8DFE866
:1071F00003F00C1111111111110C110C0C003B6852
:10720000092BDDD100210548D8E70223A3602046E1
:10721000BDE8F0810123F9E7388000300CAD003083
:1072200000000034034B01221A6000229A60DA60E9
:107230001A6170470CAD003013B5044601A90FF078
:1072400057FD04F5C04320B9012283F87D2D02B01B
:1072500010BD03F55762DDED017ADFED086AB8EE87
:10726000E77AD2ED007A67EEA67AB4EEE77AF1EE2D
:1072700010FA54BF01220022E7E700BF0000C84215
:1072800010B5044600F5DD4070308DF03BFE04F58E
:10729000DF40BDE810404430A8F0FCBB08B50F2229
:1072A000084803F03FFB60B90F220621054803F0B0
:1072B00039FB30B90F2209210248BDE8084003F02C
:1072C00031BB08BD3830003070B5154E04460D4650
:1072D00096F8F931DA0622D56FF3041386F8F931FE
:1072E000A6F5005667F0F0FF0022142167F054FF66
:1072F00096F8F4320E2B12D1022D0AD0032D0AD0AB
:10730000012D0CD194F854102046BDE87040FFF7D1
:10731000C5BF0621F8E794F854100329F4D070BDD6
:107320003880003010B50E4C49B9D4F8E00103683C
:107330001B689847A0F113035842584110BDD4F878
:10734000E00103681B6898471328EED00E22132132
:10735000A4F5A04003F0E6FA0028E6D1EEE700BF6E
:107360003880003030B50D4689B01146FFF7DAFF9E
:107370000446F0B104A81BF07BFC14F0A3FA04A9A6
:1073800012F0B2FC28B12869059B8342D4BF0020CB
:1073900001209FED127A124B8DED017AD3F88C2CDF
:1073A0008DED027A40B1D369039301A90D4806F02F
:1073B00065FF204609B030BDD2ED087AA3F54051F3
:1073C000D3F85C2CF0EEE77AD1F84C359A42F1EE26
:1073D000677A67FE877ACDED037AE6E70000000062
:1073E0003890003004AA0030F0B50F4685B0114641
:1073F0000646FFF797FF044658B1002501AA394613
:107400003046019502950395A8F050FC044618B942
:107410000024204605B0F0BDDDED017A9FED177A1E
:10742000F0EEE77A0395F4EEC77AF1EE10FA08D59C
:10743000DDED027AF0EEE77AF4EEC77AF1EE10FABB
:10744000E6D401A835F020F901A834F067FD0C4B13
:107450009DED017A01A9D3F88C3CDDED027AD3EDE4
:10746000066A084827EE267A67EEA67A8DED017A3D
:10747000CDED027A06F002FFCBE700BF000000343A
:107480003890003004AA003070B50E46114605460B
:107490002DED028B84B0FFF745FF044680B39FEDCE
:1074A000238A01AA314628468DED018A8DED028A94
:1074B0008DED038AA8F0FAFB044608B31C4B9DED42
:1074C000017AD3F88C2CDDED027AD2ED066A27EE34
:1074D000267A67EEA67A8DED017A9DED037ACDEDE1
:1074E000027AB4EEC87AF1EE10FA0EDDD2ED077A28
:1074F00067EE877A01A90F48CDED037A06F0BEFE4C
:10750000204604B0BDEC028B70BDD2ED087AA3F525
:107510004051D3F85C2CF0EEE77AD1F84C359A4222
:1075200067EE877A67FE887AE4E700BF0000000014
:107530003890003004AA00302DE9F0413D4F144648
:107540000646884697F8F931DA0616D4D7F8E001EE
:1075500043F01003012587F8F93103681B68984749
:1075600086F85400D7F8E00103681B68984709289B
:1075700005D100242046BDE8F0810025F2E7D7F8C8
:10758000E00103681B6898471228F2D0D7F8E001A1
:1075900003681B6898470E28EBD0012C12D8062CE4
:1075A00038D801A353F824F075750208157602083F
:1075B000077602081B76020827760208DD750208A6
:1075C000FD7502081C4801F09BFE0028E7D001224F
:1075D0000A211A48FAF762FF00241BE0002DC9D0E7
:1075E0000E220621144803F09DF900B9002467F02B
:1075F0006BFE2246142167F0CFFDBBE7002DB9D00A
:107600000E220521EEE72A4641463046FFF7AAFE44
:107610000028E1D0002DADD0E9E72A4641463046AA
:10762000FFF7E2FEF4E72A4641463046FFF72CFF1B
:10763000EEE700BF3880003038300030687F00301F
:1076400000F540532DE9F04F00F5DC59054600F5F3
:10765000E04409F118092DED068B93F926368DB01B
:1076600033B100F5A048D8F8043293F8D17077B957
:1076700000212185484614F0DBFC94F82910484687
:107680000DB0BDEC068BBDE8F04F14F0DBBC05F58A
:10769000C04BB8F071FD019009AEDBF8880C9FED8E
:1076A000938A90EDAAAA9FF00BFD002800F0CA80F3
:1076B000DBF8883C03F52B7393E8070086E80700A6
:1076C00030468DED0B8A34F0DFFFB0EE409A05F5C1
:1076D000D84A28460FF0DCFC0AF1680A002800F0BE
:1076E000B4805046A4F028FC07C886E8070030465E
:1076F0008DED0B8A34F0C8FFF0EE409AD8F8E00127
:1077000003681B689847122840F0A880002384F87B
:107710002830D8F8E00103685B69984738B105F56F
:107720008043D3F8B43DB3F90830002B0ADC98F954
:10773000D431002B06DA019B5046E362A4F0F8FB3B
:1077400084ED0C0A94F8283053B1019BE06A181AB2
:1077500041F28833984240F28F80002384F8283029
:10776000DBF8840C9FED620A483034F06FFB06AB07
:107770008DED090ACDED0A0A8DED0B1A9FED5D0A1C
:1077800096E8070003AE83E8070086E80700304666
:1077900034F05CFB2846B0EE408A8DED060AF0EE30
:1077A000608ACDED070A8DED081A0FF071FC0028F4
:1077B00072D0DFED517AF4EEE79AF1EE10FA94BF51
:1077C00001250025DBF8880C9FF07AFC30B1DFED55
:1077D0004A7AB4EEE79AF1EE10FA09D9002D62D197
:1077E000D8F8E00103681B689847022862D0002798
:1077F000DBF8880C9FF0A2FD0546002871D0B5EE9D
:10780000C0AAF1EE10FA6BD5DFED3C7AB4EEE7AA30
:10781000F1EE10FAACBF012600265046A4F094FB0E
:107820005EB9B0EEC00ADFED367AB4EEE70AF1EEEB
:1078300010FA58D8002D08BF002794F8281084F8B3
:10784000297017E7B0EE489A41E728460FF0E6FBAB
:1078500000287FF446AFDFED259A4FE7D8F80432D1
:1078600093F8D130002B3FF454AF98F9D431002B6A
:10787000BFF64FAF01234AE75046A4F059FBD4EDC1
:107880000C7A30EE670ADFED1F7AB4EEE70AF1EE0C
:1078900010FA3FF762AF63E728460FF0BFFB0546DB
:1078A000002886D18EE7DBF8880C9FF009FC0028C1
:1078B00096D19DE7B0EE680A08F1C4FBF0EE408A6D
:1078C000B0EE480A08F1BEFBDFED0F7A20EE280A81
:1078D000B4EEE70AF1EE10FACCBF0127002787E7E4
:1078E00000252E4699E73746A7E700BF00000000B5
:1078F0009F0CB345D30237390000FA420000C8C2DA
:10790000000070420000484255CF7D3F38B5044624
:107910000FF0BEFB04F5DC55183548B920460FF0D2
:107920007DFB014620B92846BDE8384013F072BD02
:1079300004F5A044D4F8E00103681B6C984720B913
:10794000D4F8E00103685B6C98470146EBE7000060
:1079500030B585B005460C4668461BF089F905F53B
:10796000DC506946183013F0D5FBB0B16268019B5A
:107970009FED0B7A9B1A002BB8BF5B4207EE903A43
:10798000F8EEE77A67EE877A9FED067AF4EEC77A2B
:10799000F1EE10FACCBF0120002005B030BD00BFD1
:1079A0000AD7233C00504347F0B5044685B00F4644
:1079B000154604F5DC5668461BF05AF96946183638
:1079C000304613F0A7FB10B9002005B0F0BD3946D2
:1079D0002046FFF7BDFF0028F6D13946304615F0A6
:1079E000C7FA0028F0D0002DEFD004F580542846C7
:1079F00094F8D43F43F0020384F8D43FE5E7000055
:107A000030B5044689B004F5DC5568461BF030F902
:107A100004A818351BF02CF96946284612F064F9C1
:107A200090B104A9284613F075FB68B1059B0022AC
:107A3000694620460193FFF7B7FF28B104F594404B
:107A400001210C30A8F0ECFE09B030BD30B587B094
:107A5000054602A801911BF00BF905F5DC5002A9BF
:107A6000183012F041F9019A18B90024204607B0E5
:107A700030BD02A92846FFF797FF04460028F4D03E
:107A800005F5944001210C30A8F0CAFEEEE7000095
:107A900000F5805292F8D42FD2070AD400F5A04303
:107AA000D3F8043293F8D11009B1FFF7A9BFFFF75B
:107AB000CDBF70472DE9F04F2DED0A8BBDB00446C8
:107AC00024220D4618A800210CF1A6F92422002139
:107AD00021A80CF1A1F9242200212AA80CF19CF97B
:107AE0002422002133A80CF197F904F5A0460023C5
:107AF000CDE90D330F9396F8D53113F0080835D141
:107B000004F5804943F0080399F8A82D079286F8F8
:107B1000D5311FF061F990F9213053B390F840331B
:107B20003BB304F2FC77C24638461EF009FE5FFA0A
:107B30008AF194F81E288A4225D938460AF1010AAA
:107B40001EF012FC7C23C0B203FB004090F839B851
:107B5000BBF1000FEBD1D34A022128466CF04CFF59
:107B600096F8D5316BF3C30386F8D5314FF0010891
:107B70005CE3CD4A022128466CF03EFF96F8D531F1
:107B80006FF3C303F0E704F59E4301213033184639
:107B90000BEE903AFAF7E6F9824648B9C34A022159
:107BA00028466CF029FF96F8D5316AF3C303DBE76A
:107BB00020460EF017FED9F8B43DB3F90890B9F19C
:107BC000000F01D0BA4AD5E796F9D431002B09DB72
:107BD000B84A022128466CF00FFF96F8D53169F3B8
:107BE000C303C1E720469FEDB48A01F09FFE04F570
:107BF000A4434A460CA9303318460CEE103A17F04D
:107C000053F800284FF08F0113AA14BF0223012359
:107C1000ADF854900393F123CDE913390A234FF0C3
:107C20000009CDE9003103234D21287C6AF01CFCBA
:107C3000A24B0122062128465A72A14A6CF0DCFEB2
:107C4000039B06212846022B0CBF9E4A9E4A6CF0DD
:107C5000D3FE04F540534946384683F872951EF02A
:107C600055FF5FFA89F194F81E388B420CD913AA9C
:107C700038468DED138A09F101098DED148A8DEDD9
:107C8000158A1EF0FBFCECE74FF0000A4FF07C0B6E
:107C900038461EF055FD5FFA8AF994F81E284A45C9
:107CA00019D9494638461EF05FFB3CAAC0B20C23E6
:107CB0000AF1010A0BFB004003FB092C00F68C00C3
:107CC000ACF1900C07C88CE807003CAA02EB8909CC
:107CD00009ED2F8ADFE741F288310AA82BF0B2F8CC
:107CE000D6F804029FED749A0368F0EE499A9FED6E
:107CF00077AA1B6A9847D6F8040201210026A5F04E
:107D0000D1F8734BDFED73AA01211B68586D029304
:107D100003681B689847B8F02FFA0590B8F02CFA62
:107D2000069004F58049079A99F8A83D934240F0DF
:107D3000D98094F83D1B38461EF016FB7C23C0B258
:107D400003FB004090F83938002B00F0CB8004F59D
:107D5000A04ADAF8043293F8D1300493002B00F0F3
:107D6000C18041F288310BA82BF06CF8B8F004FA0E
:107D7000059BC01A132840F2D480B8F0FDF9059095
:107D800020460EF02FFD74F09DFBD9F8B43DDAF8D3
:107D90000402B3F9083000EE103AB8EEC00A20EE43
:107DA0000A0AA6F0DFFE74F095FB38461EF0C8FC08
:107DB0001CEE100A17F040F9D9F8B43DA120B7EE37
:107DC000001AB3F90830DFED3C0A00EE103AB8EEC5
:107DD000C00A20EE0A0A2EF059FDB4EEE90A00228C
:107DE0000CA91CEE100AF0EE408AF1EE10FA58BF12
:107DF000F0EE409A16F058FF08B900230C939DED61
:107E00000C8ADFED357AB4EE498AF1EE10FAF4EE21
:107E1000E78A48BFB0EE498AF1EE10FA80F28F800F
:107E20004FF0000A9FED2D9ADFED2D8A5FFA8AFB55
:107E300094F81E385B4540F296814FF00C0918AB60
:107E4000B0EE490A0AF1010A09FB0BF903EB09003C
:107E500033F0FCFF59463846CDED110A8DED121A6C
:107E60008DED100A1EF080FA7C23C0B2B0EE680AD5
:107E700003FB004000F68C0033F0E8FF3CAB13A995
:107E800010A899448DED130ACDED140A8DED151A45
:107E900033F0B0FF09ED240A49ED230A09ED221A57
:107EA000C4E700BF95DA130884DA1308CFF5130886
:107EB000A3DA1308B5DA13080000000065AF00303C
:107EC000C0DA1308D5DA1308437A13086F12833A1D
:107ED00008AD00300000C84200000034A4707D3FAF
:107EE0000AD7233C04F5A049D9F8040203681B6AA9
:107EF00098470021D9F80402A4F0D4FF029B002186
:107F0000586D03681B689847002E40F05F81284633
:107F1000C94A05216CF070FD314638461EF0F6FD69
:107F200070E1029BB0EE498A0521186D03685B6819
:107F300098470BA82AF092FFB0EE489AF1E64FF06E
:107F400000094FF00C0B04F6380A5FFA89F394F835
:107F50001E289A4222D91946384608931EF004FA80
:107F6000089B4FF07C0CC0B209F101090BFB03F137
:107F70003CAB0CFB00A05A185430A2F16C03CDE9C5
:107F8000083218AB194433F04BFF089B099A02EDF5
:107F90001B0AC3ED010A83ED021AD6E7039B4FF0DB
:107FA000000A012B46D14FF00C0B9FEDA4BA9FEDB8
:107FB000A49A94F81E385FFA8AF6B34240F286809B
:107FC0000BFB06F63CABB0EE680A0AF1010A03EBC4
:107FD0000609A9F14803089321AB981933F046FF2D
:107FE000089B09ED120AB0EE4B0AC3ED010A83EDBE
:107FF000021A33AB981933F029FF2AAB8DED100A22
:10800000B0EE490A9819CDED110A8DED121A33F030
:108010001DFF13A910A88DED130ACDED140A8DEDE7
:10802000151A33F0FDFE09ED090A49ED080A09EDBC
:10803000071ABEE7F0EE088A9FED809A9FED80BA9E
:1080400094F81E385FFA8AF94B4564D99DED0C0A05
:10805000B4EEE80AF1EE10FA35DB0C2303FB09F964
:108060003CAB03EB090621AB03EB090033F0FEFE4A
:1080700033AB06ED120AB0EE490A46ED110A03EBE6
:10808000090006ED101A33F0E1FE2AAB8DED100A5F
:10809000B0EE4B0A03EB0900CDED110A8DED121A7B
:1080A00033F0D4FE13A910A88DED130ACDED140AF8
:1080B0008DED151A33F0B4FE06ED090A46ED080AF7
:1080C00006ED071A049E0AF1010AB9E74FF000090C
:1080D0004FF00C0A94F81E385FFA89F6B34241D982
:1080E00033AB09F101090AFB063034F0CDFA1BEE7F
:1080F000900AF0EE408AA9F07FFF07EE900A3CABB1
:10810000B8EE677A03EB8606C8EE877A67EEAA7A3E
:1081100046ED2F7ADEE74FF0000A4FF00C0B94F893
:108120001E385FFA8AF94B451DD933AB0AF1010AB3
:108130000BFB093034F0A8FAC8EE297A1BEE900A3E
:1081400067EE808AA9F058FF07EE900A3CABB8EEC4
:10815000677A03EB8909C8EE877A67EEAA7A49ED58
:108160002F7ADCE7049EB8F007F8069BC01AB0F53A
:10817000FA7F27D9B8F000F804F580430C9AB121B2
:10818000D3F8B43DDDED0D7A1B891392FCEEE77A4E
:10819000339AADF85C30149217EE903A349AADF8F9
:1081A0005E3014231592359A06901692F022CDE98E
:1081B000003213AA287C6AF057F98FF09BFE297CC5
:1081C0008FF050FC0BA82AF049FEB5E600264FF0D0
:1081D0000C0A039938461EF099FCF1B294F81E3847
:1081E0008B4207D933AB384601360AFB01321EF009
:1081F00045FAF2E738461EF053FA124A062128469D
:108200006CF0FAFB104B002520465D7201F080FBFC
:1082100004F5555032305CF0D7FF99F8D5310AA8F3
:1082200065F3C30389F8D5312AF018FE40463DB006
:10823000BDEC0A8BBDE8F08FC18A1508A4707D3FA4
:108240000AD7233CDDDA130865AF0030F0B5534F91
:1082500085B00446D7F8443DDA0700F19D8000F56B
:10826000A045D5F8043293F8C920002A40F0948044
:1082700093F8D130002B00F08C8095F9D431002B8D
:10828000C0F2878000F5E04393F83430002B40F0D3
:10829000838000F5C0469FED420AD6F8840C483032
:1082A00033F0D4FDCDED020A60EEA00ADFED3D7A99
:1082B0008DED010A8DED031AE0EE000AF4EEE70AF7
:1082C000F1EE10FA65DCD6F8843C9FED377AD3EDF9
:1082D0002E7AF4EEC77AF1EE10FA04D5D5F804320E
:1082E0001B7A002B55D0B5EE007AF4EEC77AF1EE8A
:1082F00010FA4ED404F5D8406830A3F025FEDFED27
:108300002B7AB4EEE70AF1EE10FA42D8D6F8843CA4
:108310009FED277AD3ED2D7A67EE877AB3EE0E7A4A
:10832000F4EEC77AF1EE10FA33DA224AB4F95C12AD
:10833000138801339BB2138019B9B4F85A12A4F808
:108340005C12B4F85C12994226D80026168066F0BA
:10835000BBFF0122192166F01FFFD5F80402036854
:10836000DB689847431C04F59F40134A3146403070
:1083700069F000F8D5F80432012283F8C920D7F853
:10838000443D5B0708D50D4805B0BDE8F04083F0DB
:10839000A9BC084B00221A8005B0F0BD387000302F
:1083A0009F0CB3454054094A6666663F000000B41E
:1083B000E02E654246AD0030F4DA13084066003026
:1083C0004A4BF0B52DED048BD3F8443D83B0044601
:1083D0009B0700F1878000F5C0469FED459AD6F8CF
:1083E000840C03681B699847D0ED027AF4EEC97AD1
:1083F000F1EE10FA76DB04F5A04304F5E045D3F87E
:108400000422383592F8C91049B19FED3A0A28463E
:1084100003B0BDEC048BBDE8F04068F0F1BA92F80F
:10842000D120002AF1D093F9D431002BEDDB04F5F3
:10843000E04797F83430002BE7D1D6F8840C036876
:108440001B699847D0ED278AD6F8840C03681B690E
:108450009847D4EDB20A90ED270A284668F04CFA06
:10846000F0EEE87AB0EEC08AF4EEC87AF1EE10FAD7
:1084700004D5B0EE680A284668F0C2FAD6F8840C33
:1084800003681B699847D0ED050AF4EEC90AF1EEBE
:1084900010FA27DBF6EE087A60EEA77AF4EEC87AD7
:1084A000F1EE10FA18D5B7F067FEBB6C42F210720D
:1084B000C31A934216D99FED100A0021B86404F53F
:1084C0009F4028EE000A0D4A4030B7EEC00A8DEDFD
:1084D000000B68F04FFF05E0B0EE680A2EF070F870
:1084E0000028E0D103B0BDEC048BF0BD3870003043
:1084F00000000034000000000000C84210DB130838
:1085000070B500F5A04504465C4E2DED028BD5F804
:1085100004328CB093F8D13043B195F9D431002BAB
:1085200004DB00F5405393F98E352BB900233380DB
:108530000CB0BDEC028B70BD00F5E04393F8343015
:10854000002BF3D195F8DC31002B7DD1D5F8E0017B
:1085500003681B6898470128E8D0D5F8E001036854
:108560001B6898470E28E1D004F5D840303068F0F9
:1085700047FB34F089F8F0EE087AF0EE408AB4EE6A
:10858000E70AF1EE10FAD1DA04F5DC539FED3C8AEC
:10859000D3EDF37A93EDF20A20EE270A08F128FDD5
:1085A000F2EE0E7A20EE080AB4EEE70AF1EE10FAC7
:1085B000BCD904F5C043F3EE0E7AD3F8843C93EDB6
:1085C0002D7A27EE088AB4EEE78AF1EE10FAADD9DB
:1085D00004F5DC50002309A9183009930A930B9382
:1085E00011F066FC002838D13388B4F95C220133DD
:1085F0009BB23380002A3BD0B4F85C22B3EB420F2D
:1086000096DB66F061FE01220C2166F0C5FD0022BA
:108610001C4BB7EEE80AB7EEC88A04F59F4000216C
:108620004030CDE90623184B00228DED040BCDE937
:1086300002238DED008B154A68F09CFE01220C216F
:108640001348F9F72BFF73E7D5F8E00103685B6C7B
:10865000984700287FF47AAF68E709A834F014F847
:10866000F2EE047AB4EEE70AF1EE10FABCDB5DE755
:10867000B4F85A22A4F85C22BEE700BF3CAD00303B
:10868000E02E65420000084000003E4028DB130851
:10869000687F003010B5044600F59E400B21012292
:1086A0003030F9F7FBFE04F5DB40443079F070FD23
:1086B00004F5DB4001216430BDE8104089F038BE8C
:1086C00000F5C04208B592F9C43D6BB300F5A04374
:1086D00093F9D431002B0EDA00F59F40134A06219E
:1086E000403068F047FE66F0EFFD03220F21BDE841
:1086F000084066F051BDB2F9CA3D8BB16421D2F891
:108700005C2C13FB01F39A420ADA00F59F40084AF9
:108710000121403068F02EFE66F0D6FD0222E5E72A
:10872000BDE80840FFF7B6BF08BD00BF5CDB13081B
:108730006EDB1308F8B500F5C045044695F9C43D55
:108740005BB300F5A04695F8D82D00F5DB4700F5A2
:10875000D84096F8D43168304437DB43C3F3C013B4
:1087600063F3C30285F8D82DA3F0EEFBDFED457A65
:10877000384620EE670A79F081FD04F5E04393F86E
:10878000343053B9384679F025FDD6F8043293F8E1
:10879000D1301BB93C4B00221A80F8BD95F8D83D6A
:1087A000DB0706D501220B213848BDE8F840F9F770
:1087B00075BED6F8E00103681B6898470128E9D028
:1087C000D6F8E00103681B6898470E28E2D096F9B6
:1087D000D431002BDEDB2C4E33884BB9B5F9CA3DC2
:1087E00033B1642213FB02F3D5F85C2C9A42D4DB3C
:1087F000384679F05FFDD5F8843C9FED257AD3EDBE
:108800002D7A67EE877AB3EE0E7AF4EEC77AF1EE40
:1088100010FA05D83388002BBFD0013B3380BCE76A
:10882000B4F95C321BB9B4F85A32A4F85C3233881C
:10883000B4F85C22B4F95C0293421649D5F82C2CAA
:108840003CBF013333803388012B01D10A60A4E798
:1088500009688A429EDA18B9B4F85A22A4F85C2250
:10886000B4F85C229A4298D80023338066F02CFD3D
:1088700002220C2166F090FC2046BDE8F840FFF78C
:1088800009BF00BF0AD7233C44AD0030687F0030E9
:10889000E02E654240AD003030B500F556558BB046
:1088A00004460023D5ED047A1035F5EEC07AF1EEDA
:1088B00010FA4ED9079300F5DC50089303AA0993E8
:1088C00006AB04A91830019307AB009305AB12F077
:1088D000E3FD80B3DDED087A04F580449DED077A71
:1088E000D4F8682F87FE277ADDED097A87FE277A8C
:1088F000D5ED007AB4EEE77A9DED047AF1EE10FA48
:10890000ACBF012300231AB194F86C2FD20714D402
:1089100077EEA76AF4EEC76AF1EE10FA0DD80233CB
:10892000DBB29DED037AF4EEC77AF1EE10FA0BD8C4
:10893000181E18BF01200BB030BDF4EEC77AF1EE5F
:1089400010FAEED80133EBE7012B94BF0020012091
:10895000F1E70020EFE7000070B500F5A045044600
:1089600095F8F93143F0040385F8F93166F0ACFC71
:108970000122112166F010FCD5F8043293F8D130B1
:10898000002B43D0D5F8E00103681B6898470928FD
:108990000AD1204608F0EAFF30B104F5EE40BDE808
:1089A0007040483008F0CABF194BD3F8E0010368A3
:1089B0001B69984704F5405340B993F98D35032B53
:1089C00024D10621204608F0BDFF0DE093F98D1556
:1089D0000229F6D195F8F931DB07F2D406222046B8
:1089E00001F0A0FF0028ECD00122D5F8E001094BEE
:1089F0005A7303689B6B9847034604F59F40064AE9
:108A000002214030BDE8704068F0B4BC70BD00BFCA
:108A10003880003065AF003084DB130800F5A042D9
:108A200008B592F8F931590717D56FF3820382F828
:108A3000F9310A4B5A7B42B1002200F59F400221D6
:108A40005A734030064A68F095FC66F03DFC0022FF
:108A50001121BDE8084066F09FBB08BD65AF00303E
:108A6000A8DB1308F0B5054685B005F5DC57684668
:108A70001AF0FEF869461837384612F04BFB80B101
:108A800005F55653384CD3ED047AF5EEC07AF1EE85
:108A900010FA08D80023354A28462380D373FFF7FD
:108AA000BDFF05B0F0BD2846FFF7F6FE0646284696
:108AB0000EF0B4FA10B928460EF08AFA002EA37808
:108AC00018BF00200343DBB2A370002BE9D063780A
:108AD000A8BB83BB23780133DBB2082B237003D1FF
:108AE0004EB3384612F084FE2378092B02D1384663
:108AF00012F06AFE2378092B1DD94FF48573238069
:108B000066F0E2FB0222102166F046FBB7F034FB70
:108B10006368C01A47F23053984209D905F59F405F
:108B2000134A0221403068F025FCB7F025FB606055
:108B30002846FFF711FF62780C4BDA73B1E726780D
:108B4000002EF8D0013EF6B22670002BF3D0002E96
:108B5000F1D1667066F0B8FB3246102166F01CFB5E
:108B60002846FFF75BFFE6E748AD003065AF003011
:108B7000C0DB130800F5A04393F8F9315B0701D57A
:108B8000FFF7EABE70470000F7B500F5DC56044673
:108B900001A9183604F58045304612F0DFF9D5F802
:108BA000A83F074683420CD004F5C043D3F8840C99
:108BB0009CF0E2FAC5F8A87F66F086FB3E2166F0DD
:108BC000CBFA304612F0BAFD95F9AC3F83421FD084
:108BD000304612F0B3FD01301AD004F5C043D3F88B
:108BE000840C9CF0C9FA304612F0A8FD85F8AC0F51
:108BF00066F06AFB95F8AC2F182166F0CDFA04F503
:108C00009F4095F9AC3F0421024A403068F0B2FB26
:108C100003B0F0BDD0DB13082DE9F043054695B055
:108C2000B7F0AAFA002403AB05F5DC5780460BAA7F
:108C30000193183702AB08A93846089400930EAB8D
:108C400009940A940B940C940D940E940F94109420
:108C500012F0FAFBDFED4D7A06469DED0A7AB4EE8E
:108C6000E77AF1EE10FA4BDB9DED0D7AB4EEE77A80
:108C7000F1EE10FAACBF4FF001094FF0000907AB5D
:108C800004AA05A93846019311AB1194009306ABD1
:108C90001294139412F000FC0028384608BF0026F6
:108CA00012F0ECFB044666B1B9F1000F09D0F7EE03
:108CB000007A9DED057AB4EE677AF1EE10FAC8BF3E
:108CC0004C4605F5804696F9DC3C012B1BD174B16E
:108CD00005F5A043D3F8042292F8D1403CB1D3F873
:108CE000E00103685B69984780F00104E4B296F8FC
:108CF000B02F52BB4CB9C6F8B48F15B0BDE8F083A5
:108D00004FF00009BBE70024F1E7D6F8B43FA8EB29
:108D10000300B0F57A7FF0D9012405F5C043C6F809
:108D2000B82F86F8B04FD3F8883C83F8F44266F049
:108D3000CBFA22461D2166F02FFA154A05F59F4011
:108D40000221403068F016FBD7E714B1C6F8B88F9F
:108D5000D3E7D6F8B80F43F69823A8EB0000984263
:108D6000CBD905F5C043C6F8B44F86F8B04FD3F859
:108D7000883C83F8F442C6F8B84F66F0A5FA22465C
:108D80001D2166F009FA034AD8E700BF000000344D
:108D9000E8DB130802DC13080A4B012210B5044675
:108DA0005A72B7F0E9F904F5E042136AC31A142BBA
:108DB00007D9106204F5DA50BDE81040083056F0CB
:108DC00081BF10BD65AF00302DE9F743044600F5C3
:108DD000565000230DF1070104F5A04708308DF827
:108DE00007305CF039FFD7F8040290F9C830026808
:108DF00033F008032CD013693221984704F1100096
:108E000004F59F4816F0F2FB1F4B4FF0000908F1E4
:108E100040081E68706D03681B6A984701281ED1C0
:108E2000B7F0AAF941F28733A0EB090205469A424E
:108E300005D9A946154A0621404668F09BFA204606
:108E4000FFF7AAFF306D032103685B689847E1E7ED
:108E500004F540531269B3F898159047CEE7012105
:108E6000D7F80402A4F01EF8D7F8040203685B6A7E
:108E7000984772F047FF706D012103681B6803B0CB
:108E8000BDE8F043184700BF08AD003020DC1308F0
:108E9000044600F59F40174A06214030164D9FEDCD
:108EA000178A08B568F066FA2046FFF78DFF20465E
:108EB000FFF772FF20460DF095FC2B680321186D1B
:108EC00003685B68984773F0FDFA04F58043D3F8B4
:108ED000B43DB3F9083000EE103A04F5A043B8EE03
:108EE000C00AD3F8040220EE080AA5F03BFE73F096
:108EF000F1FADCE744DC130808AD00306F12833A66
:108F00002DE9F843044600F59F40264A06214030EB
:108F100004F5A045DFF8948041F287392DED028BEE
:108F200068F028FA2046FFF74FFF73F0CBFAB7EE50
:108F3000000AD5F80402A5F015FE73F0CBFAB7F0DD
:108F40001BF90646B7F018F9801BD8F800704845A1
:108F500014D99FED158A73F0B5FAB0EE480AD5F82A
:108F60000402A5F0FFFD73F0B5FA2046FFF714FFE9
:108F7000386D032103685B689847ECE773F0A2FA49
:108F8000B7EE000AD5F80402A5F0ECFD73F0A2FAE2
:108F90002046FFF701FF386D032103685B6898479F
:108FA000D0E700BF74DC13080000000008AD0030FB
:108FB00000F5A043F7B5D3F80432044693F9C8305E
:108FC000032B2AD0652500F5E047354E013D15F00D
:108FD000FF050BD0FB694BB933681421186D03688A
:108FE0005B68984720460DF0FDFBEFE704F59E40D7
:108FF00001213030F8F7B6FF04F5405393F9883576
:1090000068B953B1092B08D08DF8070004F5565004
:109010000DF1070108305CF01FFE03B0F0BD032B1B
:1090200038D8DFE803F00227313404F58043D3F861
:10903000B43DB3F9082040F2B5339A422CDD04F573
:10904000565001250DF1070108308DF807505CF0EE
:1090500003FE04F59F40134A0221403068F08AF96C
:10906000114B5D720E4B1C68206D052103685B6817
:109070009847F9E704F58043D3F8B43DB3F90820E5
:1090800040F2B5339A4207DD2046FFF701FF204644
:10909000FFF736FF092BC0D000238DF80730B5E766
:1090A00008AD003098DC130865AF003000F59F4034
:1090B0000B46024A0421403068F05CB9B8DC130862
:1090C00010B5044666F000F90022052166F064F848
:1090D00004F59F40034A04214030BDE8104068F089
:1090E00049B900BFC4DC13080B4613B54AB100F5FB
:1090F0009F4000920421054A403068F03BF902B0DD
:1091000010BD02B0BDE81040FFF7D0BFDCDC130893
:1091100000F59F40064A0421403008B568F02AF95E
:1091200066F0D2F800220821BDE8084066F034B8A5
:10913000F0DC130838B504460D46B7F01DF804F509
:10914000A0433DB9D3F8F021C3F8F4010AB9C3F83C
:10915000F00138BDD3F8F421801A642884BF0022BE
:10916000C3E97C22F5E7000037B5044600F5D84096
:109170006830A2F0CFFE04F5A042C0F3803592F82B
:10918000D631C3F34001A9421DD065F3410304F574
:109190009F4482F8D63140346DB166F095F80222D2
:1091A0000B2165F0F9FF094A0221204603B0BDE812
:1091B000304068F0DFB866F087F82A460B2165F08A
:1091C000EBFF034AF0E703B030BD00BF08DD130832
:1091D00024DD130838B50A460C460621054601F081
:1091E000A1FB28B921462846BDE8384008F0AABBB3
:1091F000024A137843F00803137038BD84AF00307F
:1092000038B50A460D461521044601F08BFB60B9BE
:1092100004F59F400421084A403068F0ABF8294625
:109220002046BDE8384008F08DBB044A137843F06F
:109230000803137038BD00BF34DD130884AF00305D
:1092400038B50A460D461521044601F06BFB60B99E
:1092500004F59F400421084A403068F08BF8294605
:109260002046BDE83840FFF7B5BF044A137843F005
:109270000803137038BD00BF5CDD130884AF0030F5
:1092800038B50A460D461B21044601F04BFB28B1B8
:10929000094A137843F00803137038BD04F59F4062
:1092A0000421064A403068F065F829462046BDE8AA
:1092B0003840FFF78FBF00BF84AF003072DD130866
:1092C00038B50A460D461121044601F02BFB28B1A2
:1092D000094A137843F00803137038BD04F59F4022
:1092E0000421064A403068F045F829462046BDE88A
:1092F000384008F027BB00BF84AF003084DD13087E
:1093000010B500F5A04494F8D6319A0623D4D4F8C9
:10931000E00103681B689847032808D005D8022895
:109320000ED194F8D401C00914E01B28F9D194F8A7
:10933000D40100F0A000A0F180035842584109E098
:10934000B4F8D40120F4FE4020F07F0080B2003851
:1093500018BF012010BD0120FCE7000038B500F562
:10936000A045044600F59F40184A95F8F9310221BE
:10937000403043F0080385F8F93167F0FBFF65F0F2
:10938000A3FF0122172165F007FF2046FFF7B8FF72
:1093900040B104F59E40012215213030BDE838402F
:1093A000F9F77CB8D5F8E00103681B6898470628F0
:1093B00006D104F5F040BDE83840643009F048BDFE
:1093C00020460B21BDE83840FFF704BF98DD1308A5
:1093D00070B500F5A0450646D5E97C239B1A41F2FD
:1093E0008832934211D9D5F8E00103689B6C984705
:1093F000044695F8F931C3F3C003A34213D034B146
:109400003046BDE87040FFF7A9BF0024F1E765F0E2
:109410005BFF2246172165F0BFFE95F8F93164F332
:10942000C30385F8F93170BD0B46114610B50446EB
:10943000072B07D8DFE803F028041114171A222598
:1094400008F080FA04F58044D4F8E03C9B061BD574
:109450000E48BDE8104082F045BCFFF7BBFEF1E7C7
:10946000FFF7EEFEEEE7FFF7CBFEEBE700F59E40E1
:10947000012214213030F9F711F8E3E7FFF700FF7C
:10948000E0E7FFF71DFFDDE710BD00BF40660030DD
:1094900070B5044665F018FF0122052165F07CFED9
:1094A00004F54053204693F87235072B96BF324A95
:1094B0000125D55CFFF724FF68B1304A20463049CA
:1094C000FFF712FE04F59E40012210213030F8F71C
:1094D000E5FF002514E004F5A046D6F8E001036896
:1094E0005B6C984798B196F8593783B196F958371D
:1094F000012B0CDC234A244901252046FFF7F4FD0B
:10950000294620460322BDE87040FFF78DBFD6F8FC
:10951000E00103685B6C984728B104F58043D3F8F9
:10952000E03C190717D4D6F8E00103681B68984798
:10953000032805D104F58043D3F8E03CDA070DD4C5
:10954000D6F8E00103685B6A984768B90C49204681
:10955000FFF7ACFDD4E70B4A0949CDE70B4A0849B0
:109560002046FFF7C1FDB4E704F58043D3F8E03CA3
:109570005B07EBD5064AF2E780DE1308B8DD130877
:10958000C2DD1308C8DD1308DBDD1308EBDD1308AB
:10959000FBDD130838B50446154665F095FE01223B
:1095A000062165F0F9FD2046FFF7AAFE98B104F503
:1095B0009E400122072100253030F8F76FFF144A42
:1095C00014492046FFF790FD294620460422BDE8B5
:1095D0003840FFF729BF04F5A043EDB2D3F8E0010E
:1095E00003685B6C984768B104F58043D3F8E03CAE
:1095F0001B0707D535B1084A204606490125FFF764
:1096000073FDE1E703492046FFF750FDDCE700BFAB
:10961000B8DD13081ADE1308C8DD1308F8B50446D0
:1096200065F052FE0122082165F0B6FD04F5A04662
:1096300071F00EF804F5405393F86135062B96BF90
:10964000364A0225D55CD6F8043293F8D1705FB95A
:1096500033492046FFF72AFD0025294620460522EA
:10966000BDE8F840FFF7E0BE2046FFF749FE60B1D5
:1096700004F59E40012212213030F8F70FFF294AED
:1096800027492046FFF730FDE6E7D6F8E0010368FA
:109690005B6C984768B196F8593753B196F95837CB
:1096A000012B06DC204A214920460125FFF71CFD3D
:1096B000D3E7D6F8E00104F5804703685B6C984770
:1096C00018B1D7F8E03C190713D4D6F8E0010368C5
:1096D0001B689847032803D1D7F8E03C9A070BD4BE
:1096E000D7F8E03CDB0609D40D492046FFF7DEFC45
:1096F000B3E70D4A0A49D7E70D4AC1E7D6F8E001BA
:109700000368DB69984706460028EDD1094A2046E0
:1097100003493546FFF7E8FC9FE700BF88DE1308E2
:10972000A2C81308B8DD1308C8DD130814DE130837
:1097300022DE130837DE1308F8B500F5405304465F
:1097400093F96135CBB300F5A04500F58047D5F816
:10975000646196B307F63C57B6F00EFDDFED177A5D
:10976000861B97ED000A8D209FED151A20EE270A23
:10977000DFED140A2DF08AF8BCEEC00A10EE103AA4
:109780009E420CD295F8F9319A0716D52046002151
:10979000F8F76AFF2046BDE8F840FFF7B9BC0CD9DE
:1097A00095F8F9319B0708D420460121F8F75CFFB2
:1097B0002046BDE8F840FFF731BFF8BD00007A440D
:1097C0000000804F000000002DE9F341074600F53E
:1097D000D84007F5A0446830A2F09CFBC0F3804855
:1097E0000190B6F0C9FC94F8FC3145460646434565
:1097F0000DD007F59F4084F8FC814030002D41D00A
:109800003B4B3C4AC4F80062022167F0B3FD94F878
:10981000FC3107F5804843B394F8FD312BBBB8F910
:10982000523D4FF4AA709FED340A07EE903A9FED37
:10983000331ADFED330AF8EEE77A27EE800A2DF0CF
:1098400025F8BCEEC00AD4F8000210EE103A361A21
:109850009E420AD9012307F59F402A4A022184F833
:10986000FD314030224B67F085FD98F9513D002BCA
:1098700094F8F9310DDC6FF3451384F8F93102B037
:10988000BDE8F0811A4B204AC4F8008284F8FD81BB
:10989000BAE7C3F34012AA42F1D065F3451384F846
:1098A000F9319B06EBD5194BD3F8E00103681B692E
:1098B00098470028E3D065F007FD01221F2165F0DD
:1098C0006BFC3846FFF71CFD48B107F59E400122AE
:1098D0002121303002B0BDE8F041F8F7DFBD32227F
:1098E00098F8511D384602B0BDE8F041FFF79CBD25
:1098F00050DE13085FDE130800007A440000804F3A
:109900000000000075DE13086ADE1308388000309E
:1099100008B50122034B1A70B6F022FC024B186006
:1099200008BD00BF51AD003054AD0030014B0022E6
:109930001A70704751AD00302DE9F0410446B6F081
:109940000FFC2A4B0546B4F876221988284E91421E
:109950000ED01A80274B18603378A3B100243470DE
:1099600065F0B2FC22461321BDE8F04165F014BC5D
:109970003378214FDBB93B782BB11E4B1F4A1B6854
:10998000C31A934201D8BDE8F0810123337004F576
:10999000A043D3F8040290F8D13013B103681B6AD6
:1099A000984765F091FC0122132165F0F5FB3B78A7
:1099B000002BE8D03378002BE5D00E4A104913680D
:1099C000EB1A8B42DFD904F5A0441560D4F80402E9
:1099D00090F8D130002BD6D00021A3F063FAD4F850
:1099E00004020368BDE8F041DB69184752AD00305E
:1099F00050AD003054AD003051AD003080841E00B9
:109A000040420F002DE9F84300F54758044600F5A1
:109A1000405908F1240804F5A04799F8246240460B
:109A200083F054F9D7F80432054693F8D130002B6F
:109A30006BD0002867D0364B93F9D431002B06DB6E
:109A400004F59F40334A0521403067F093FC99F9B3
:109A5000E76156B197F9D431002B0EDA04F59E4038
:109A600001220F213030F8F719FD65F02DFC2A4650
:109A70000921BDE8F84365F08FBBD7F8E001036822
:109A80005B69984758B197F9D531002B07DA97F8F9
:109A9000F931DA0703D499F82432DB07DED52946F9
:109AA000404683F051F9DFED1C7AB4EEE70AF1EE9F
:109AB00010FA05DD0A220921204600F033FFD4E721
:109AC000023E032E11D801A353F826F0B59A0208DE
:109AD000DD9A0208FB9A0208019B02080A2215215E
:109AE000204600F01FFF0028BFD10A220621204691
:109AF00000F018FF0028B8D1DCE70A221121F6E7B0
:109B00000A221521F3E7002EAFD1BDE8F88300BF8C
:109B10003880003090DE13080000C84270B500F5B0
:109B2000D84500F5804386B00446683593F8B01FE9
:109B30002846A2F0A7F902A819F09AF804F5DC501B
:109B400002A9183010F0D0F804F5C043049A284652
:109B5000C3F8602C059AC3F8642CA2F0DBF98206E6
:109B60001AD5284604F5D845A2F0E2F9FDEEC07AF0
:109B7000583504F58054022217EE901A284617EE45
:109B8000906A19F07BF894F8D43FDB0706D40122E1
:109B90003146284619F072F806B070BD01212846FA
:109BA00019F0FEF80028F2D0F6E7000038B500F50D
:109BB000A0440D4694F8D531C3F380138B420BD0EB
:109BC00021B165F081FB112165F0C6FA94F8D53119
:109BD00065F3861384F8D53138BD0000F0B500F583
:109BE000A046054600F5C0442DED048BD6F804329E
:109BF0008BB093F8D130002B73D096F9D431002B71
:109C00006FDBD6F8E00103685B69984700286DD1E7
:109C1000D4F8840C01AF9FED430A483032F016F9B6
:109C20000AAACDED080A04AB8DED091A8DED070ADD
:109C300012E9070083E8070087E80700384630F09C
:109C400045F905F5D840D4F8843CB0EE409A303060
:109C5000D3ED2D8A66F0D4FF32F016FDD4F8883C9F
:109C6000D6F8E001B0EE408AD3EDAA9A03685B6CA7
:109C70009847DFED2D7AB4EEE79AF1EE10FA02DCA8
:109C800096F8DC3103B1B0B1DFED287A68EEA78A2F
:109C9000F3EE0E7AF4EEE78AF1EE10FA0BDCF0EE5A
:109CA000087AB4EEE78AF1EE10FA04DCF5EEC09A19
:109CB000F1EE10FA30DBD4F8845C40F27F10B7EE9E
:109CC000001ADFED1B0A2B685E6ED4F8883C93ED1A
:109CD0009C0A2CF0DBFD2846B0470BB0BDEC048B92
:109CE000F0BDD4F8840C0368DB6D0FE005F580450A
:109CF000D4F8840CD5F8B42D0368B2F90820002AF2
:109D000003DCD6F8D821022AEED11B6E0BB0BDECD5
:109D1000048BBDE8F0401847D4F8840C0368DB6D71
:109D20009847DAE79F0CB3450080BB44E02E6542BC
:109D300000000000F8B500F5A04605460C4696F870
:109D4000D431B1EBD31F4DD0274B00221A6000292C
:109D500044D065F0B9FA122165F0FEF996F8D431D5
:109D600005F5565005F5405764F3C71384F0010418
:109D70003030214686F8D4318EF0B6F934B197F8F8
:109D8000F6321BB9B6F0F8F9C7F8F80287F8F642D0
:109D90002021D6F8E001B7F9444503689B6998474C
:109DA00038B1D6F8E00103685B69984780F0010399
:109DB000D8B296F9D431002B14DAD6F8043293F8DD
:109DC000D1307BB163070DD560B105F59E4001220E
:109DD0000D213030BDE8F840F8F760BB65F074FA4B
:109DE0001C21B9E7F8BD00BF58AD00302DE9F84F90
:109DF00000F5A04504462DED048BD5F8043293F808
:109E0000D1604EB901212046FFF794FF95F9D43176
:109E1000002B32DA01214DE095F9D421002A22DA13
:109E2000D5F8E00103681B6C984706460028EDD181
:109E3000D5F80432204693ED0C8AF8F7EBFCB4EE2B
:109E4000C80AF1EE10FAE1D5D5F8043293F8A9303A
:109E5000032BDBD163F0BCFB4FF48011392263F09C
:109E60006DFB3146CFE700F5E042DFF89C9192F8B8
:109E7000342032B30023C9F80030634B93ED007AED
:109E8000B4F95C32B8EE477A1BB9B4F85A32A4F888
:109E90005C32B4F85C32DFED5D6A07EE903AF8EEC2
:109EA000E77A67EEA67AB4EEE77AF1EE10FAACBF85
:109EB000012100212046BDEC048BBDE8F84FFFF7DF
:109EC00075BE93F807B000F5C043D3F8840C03685F
:109ED0009B6D98478046D5F8E00103685B69984719
:109EE000002800F08980D5F8D831F7EE007AF0EE3E
:109EF000088A022B08BF804648FEA78A04F5DB4784
:109F00006437384688F034FA013004F5D8400CBF85
:109F100001230223303009EE903A66F071FE32F0F0
:109F2000B3FB04F5D840B0EE409A6830A2F00CF8CC
:109F30002046B0EE408A0CF03DFE00285FD004F5CC
:109F40009C407C3066F05AFDDFED317A90ED007A6E
:109F5000B4EEE77AF1EE10FA4CBF4FF0010A4FF081
:109F6000000A384688F004FA012805D0384688F0FF
:109F7000FFF9431C5E425E41BBF1000F41D0B8F1D6
:109F8000000F3ED0F8EEE97AB4EEE79AF1EE10FA5F
:109F900037D8642319EE902AB0EEC88A12FB03F773
:109FA00007EE907AF8EEE77AB4EEE78AF1EE10FA6F
:109FB00027D5BAF1000F24D01EB3D9F80030B4F978
:109FC0005C2207EE903AB8EE677A1AB9B4F85A22D2
:109FD000A4F85C22B4F85C2207EE902AF8EEE77A47
:109FE00067EEA87AB4EEE77AF1EE10FA7FF50AAFE1
:109FF0000133C9F8003009E7F7EE008A7EE7B24680
:10A00000AFE70023F5E700BF58AD0030CDCC4C3EA4
:10A010000000484300F5FD53DFED217A9FED217AE2
:10A0200030B5044693ED021A87B031EE271AD4ED0D
:10A03000997A6D46F0EEE77A93E80700F4EEC77A76
:10A0400085E80700F1EE10FA04F5D84000F1300081
:10A050000BD5B4F95A32F7EE006A07EE903AF8EEF3
:10A06000E77A86EEA77A84ED997AD4ED991A9DED78
:10A07000000ADDED010A66F035FD2046FFF7B6FE69
:10A080002046FEF757FB2046FEF73AFA2046FEF739
:10A09000DDF8204607B0BDE83040FEF791B900BFBB
:10A0A0000AE81C410000003410B504461D202DEDC7
:10A0B000028B71F093FF60B304F5A043D3F8E00185
:10A0C00000F098FA192108EE100A04F584505CF0AB
:10A0D0005BFA02281AD00338012808D804F59C40FE
:10A0E0007C3066F08BFC90ED008ABDEEC88AB8EE3D
:10A0F000C88A9FED090A04F5DB4028EE000A6430A7
:10A10000BDEC028BBDE8104088F052B99FED038A88
:10A11000EDE7BDEC028B10BD0AD7233C0000000028
:10A12000114A0260114A02F17001426081601049D7
:10A13000C160043101610839416120398161A2F5B2
:10A14000CD5102F5C452C1610A4942630162A1F5D1
:10A15000D451094A4162A1F58B6182638162043165
:10A16000C16204310163704738F71308706500302D
:10A17000C49C0030BC9C0030003300301C2968D8DF
:10A18000DFE801F0130F171B26232E1F672A673203
:10A190006767363A3D4044474A4E52575B5F6767B0
:10A1A000640000F5E0405030704700F5F140703039
:10A1B000704700F5E1401030704700F5E1404C3049
:10A1C000704700F5EB406C30704700F5EF40F2E768
:10A1D00000F5EE400430704700F5EE40483070471F
:10A1E00000F5F0406430704700F5EC402C307047CB
:10A1F00000F5EC406830704700F5E840704700F526
:10A20000EF40D0E700F5EB402830704700F5F44010
:10A21000D1E700F5F340D2E700F5F4406030704735
:10A2200000F5F5402430704700F58040D0F8E00A92
:10A23000704700F5ED403C30704700F5F8400830BD
:10A24000704700F58040D0F8D80C704700F5F94011
:10A25000704700207047000073B50B68054608463C
:10A260000C469B6B16469847034605F59F400F4AE0
:10A2700004210096403067F07DF865F025F82368EA
:10A28000054620461B6898470A210246284664F086
:10A2900083FF074B93F8D5319B0641BF054A1378DE
:10A2A00043F00403137002B070BD00BFA0DE1308BA
:10A2B0003880003084AF003000F58043002200F584
:10A2C000A04083F8CC2ED0F8E0010368DB68184783
:10A2D00070B5054608680C46164603685B699847E2
:10A2E00090B1306803685B69984768B905F5A04389
:10A2F000D3F8042292F8D12032B193F9D431002B53
:10A3000002DB2846F8F79CFA04480DF0BFFA2068F3
:10A310000368BDE870409B68184700BF34AE00304A
:10A3200070B500F5A04504460C4ED5F8E001036871
:10A33000DB6998473074D5F8E00103681B689847DB
:10A34000F070D5F8E0010368DB6B9847014604F52F
:10A35000DA50BDE87040083055F0FEBC65AF003003
:10A360001F4B37B5144693F8F9210D46D20703D495
:10A3700093F8D5315B0704D400232B60236003B02E
:10A3800030BDC36A01A9DFED176A1B689FED161A7D
:10A39000B3F9083060EE811A07EE103A836A20EEB6
:10A3A000011A68461B68B8EEC77AB3F9083067EE41
:10A3B000260A07EE903AF8EEE77A27EEA60A2DF085
:10A3C00007FBDFED0A6A9DED007ADDED017A27EEED
:10A3D000267A67EEA67A85ED007AC4ED007ACEE79C
:10A3E00038800030530469390AD7233C0000C84242
:10A3F00030B500232DED028B89B0B0EE408A029378
:10A4000006AD039302AC324B93F8F92112F0010F21
:10A4100003D193F8D5315B070BD494E8030085E8AA
:10A4200003009DED060ADDED070A09B0BDEC028BC5
:10A4300030BD836ADFED276A1B68B3F9083007EE89
:10A44000903AC36A1B68F8EEE77AB3F9083067EE12
:10A45000A67A07EE103AB8EEC77ACDED037A27EE6A
:10A46000267AF1EE476AB0EEC77ACDED026ADFEDEB
:10A470001A6AB4EEE67AF1EE10FA06D5F0EEE77A53
:10A48000F4EEE67AF1EE10FAC7D403AA2146134897
:10A49000F8F706FADDED027A9DED037A2046F0EE3C
:10A4A000E77AB0EEC77AF4EE477AF1EE10FA37FEAB
:10A4B000870A2FF059FC04A88DED040ACDED050A9A
:10A4C0002FF004FD204688EE000A2FF07DFCA4E763
:10A4D00038800030530469390000003438300030CF
:10A4E000094B93F9D421002A0CDAB5EEC00AF1EE3B
:10A4F00010FA07D9D3F8043293F8A900C31E5842C2
:10A50000584170470020704738800030436A1B680C
:10A5100093F8D13043B1054B93F8D40100F0A0007B
:10A52000203818BF01207047012070473880003064
:10A5300010B5436A04461868D1B10221A2F0C2FCEA
:10A54000236A9FED0C1A1868F0EE410A0368B0EE1A
:10A55000410ADB699847236A074A00211868D2ED4F
:10A56000000A03689FED030ADB6CBDE81040184742
:10A570000121E3E7000000007865003010B5436A70
:10A5800004461868002930D00221A2F09BFC236AFF
:10A5900018689AF057F9636A1B6893F8A930012B81
:10A5A00004D8236A012118689AF052FE636918687A
:10A5B0009DF0C8FD636918689DF04CFE63699FEDCE
:10A5C0000C0A18689DF09AFF636918689DF0EEFF09
:10A5D000236A9FED071A1868F0EE410A0368B0EE8F
:10A5E000410ADB69BDE8104018470121CDE700BFF3
:10A5F0000000000013B5044601A90C480CF078FBDC
:10A6000010B1019802B010BD636918689CF058FD44
:10A6100018B9074BD3F85C0CF4E701AA03210548ED
:10A6200018F062FB0028F4D0EBE700BF38300030B0
:10A6300038900030909C0030F0B504462DED048B2E
:10A6400089B0002940F0F68083687C4E03F5805382
:10A65000B3F93655642DB8BF6425FFF7CBFF6268A8
:10A66000A8422046B2F93430AABF96F8D551012548
:10A67000C5F38015002BD5BF63695B421B6807EEED
:10A68000903AD4BF93ED978AB8EEE78AB2F93230A8
:10A69000002BB8BF5B429BB25B4207EE903AA368C7
:10A6A000F8EEE77A03F58053B3F93675F4EEC87A1D
:10A6B000F1EE10FA38FE278A642FB8BF6427FFF73F
:10A6C00099FF6369391AA26B1B6800EE101AD2ED6C
:10A6D000001A93ED991AD3ED0E0AB8EEC00A2CF0C9
:10A6E00061FD6368F0EE480A40F25320B3F932305E
:10A6F000002BB8BF5B429BB25B4201EE103AB8EE52
:10A70000C11A2CF0C3F86369B0EE408A18689CF057
:10A71000D7FC96F8D63107461B0778D448489EF0F8
:10A720006BFC002873D0002F71D09FED469A01A9D1
:10A7300043488DED019A8DED029A9EF0E5FC0028CC
:10A7400075D0A069A1F0F2FB03AB03C883E8030056
:10A75000194601A82FF0ECFA05A88DED050ACDEDFC
:10A76000060A2FF0B3FBF0EE409A374805A9DFED5B
:10A77000377A034624388DED059AD3ED008A8DEDA6
:10A78000069A68EEA78A8DED079A9EF0E7FCF4EE34
:10A79000E89AF1EE10FA08DDF0EEE88ADFED2C7AA7
:10A7A000F4EEE78AF1EE10FA45D5DDED077A9FED7C
:10A7B000297AF4EEC77AF1EE10FA28DD9FED267AB9
:10A7C000F4EEC77AF1EE10FA21D56368F2EE0E7A54
:10A7D000B3F93230002BB8BF5B429BB208EE103A9F
:10A7E000BAEEEF8A88EE277A67EE297AF5EEC07A1C
:10A7F000F1EE10FA48BFDFED137A37EEC88AFAEEB1
:10A80000047AB4EE678AF1EE10FA37FE888A63693B
:10A81000B0EE480A294618689CF0E2FC63691868A3
:10A8200009B0BDEC048BBDE8F0409DF0BFBEF0EE7A
:10A83000499A9AE700259FED038AE8E738800030BF
:10A840003C9E003000000000609E00300000C842C6
:10A850000000003400000C4200004843436A1868BE
:10A8600003689B681847000038B52DED028B03681C
:10A870000446DB6F9847236B2948F0EE408A1B683B
:10A88000B3F908500CF034F8041E4FF47A724FF00C
:10A8900000012846D8BF4FF4FA742CF05FF8B6EEEA
:10A8A000000A84422ADD07EE900AB8EEE77A07EE46
:10A8B000904AF8EEE77A27EE007A87EE278A4FF47F
:10A8C0005C7038EEC00AF5EE087AB7EE001AB1EE09
:10A8D000400AFEEE000A80EE270A2BF0D7FFF7EEC3
:10A8E000007A77EEC07A28EE000A20EE080A20EE01
:10A8F000080AA7EE880ABDEC028B38BD031BC4F51D
:10A900007A7407EE103A07EE904AB8EEC77AF8EE7E
:10A91000E77A27EE007A87EE278A38EE008ACEE7BC
:10A92000383000302DE9F04700F5E04300F5A0484D
:10A9300004460E4617462DED028B93F84C5082B01C
:10A9400083F84C20D8F8E00103681B689847B042B0
:10A9500023D104F540531A2F83F8F47209D140B97A
:10A9600004F5C04304F59A44D3F8843CA269C3F8C3
:10A97000D8207C4B93F8D531980606D4012528467B
:10A9800002B0BDEC028BBDE8F087BD42F6D0764A3E
:10A99000137843F002031370F0E71B2E0AD104F57D
:10A9A000E14039464C3002B0BDEC028BBDE8F047C7
:10A9B00001F0D6B931462046FFF7E0FB054601908D
:10A9C00018B9204662F07CFAD9E7D8F8043293F837
:10A9D000D1A003688AF001095B69984704F5EC434C
:10A9E000019A2C339A4208BF0120BAF1000F08D116
:10A9F0000198494603685B689847054648BB5B4A2F
:10AA000022E098F9D431002B80F29E80002800F0DB
:10AA10009B80DFF850A1DAF8E00103685B69984792
:10AA20000546002840F090800198FFF71DFFB0EE2A
:10AA3000408AAAF5A040F7F7EDFEB4EEC08AF1EE29
:10AA400010FA40F381804A4A01992046FFF704FC3E
:10AA500095E704F5A34101AA20466031FFF738FCD1
:10AA6000D8F8E00103681B68984704F5405388F85C
:10AA7000E4010198C8F8E00183F8F47203681B68E8
:10AA80009847014604F59B403A463C3063F06AFF24
:10AA900004F59F40002140306EF06CFCF31E012B4A
:10AAA00002D9B11F4D424D4104F5C04704F547504E
:10AAB00087F8525F243082F06BF9D8F8E001036820
:10AAC0001B689847C21E04F58043504203F6E841D4
:10AAD00003F618535041D7F8842C012E87F8E00C68
:10AAE0000968C2F8D410D7F8842C1B68C2F8D83093
:10AAF00001D00B2E06D104F59A42D7F8843C126897
:10AB0000C3F8D8202046FFF70BFC164B93F8D5313D
:10AB10009B063FF53CAF31E716480CF0CBFA002816
:10AB20007FF466AFD8F8E00103685B6998470028B6
:10AB30003FF45EAF019803685B69984705460028BB
:10AB40007FF456AF0C4A7FE7019803681B6998476A
:10AB50000028E1D007480CF09BFA05460028DBD11D
:10AB6000064A71E73880003084AF00304A68150823
:10AB7000C0DE130838300030D2DE1308CC1B1508B5
:10AB80000148FFF7CFBE00BF383000301FB5044684
:10AB90008DED010A85F004FC01A9A26B636992EDB9
:10ABA000001A00221B68039203AAD3ED990A93EDC1
:10ABB0000E0A84F063F9DDED037A9FED0B7AF0EE77
:10ABC000E76AF4EEC76AF1EE10FA09D49DED017A56
:10ABD000F4EE477AF1EE10FA77FE277ACDED017A9E
:10ABE0009DED010A04B010BD00000034436A1868EE
:10ABF0000368DB691847000038B5436A05461C68DE
:10AC000094F8D11061B92046A2F05CF96B6A1B6818
:10AC100093F8A90018B1012814BF0320022038BD01
:10AC2000164803783BBBFFF75BFC20BB144A92F845
:10AC3000D43103F0A003202B17D0B5EEC00AF1EEFB
:10AC400010FA10D592F8D6315B070CD401212046BA
:10AC5000A2F038F96B6A1B6893F8A930012B0CBF7E
:10AC600002200320DBE70221F1E720460221A2F0C7
:10AC700029F90420D3E70120D1E700BF34AE00302A
:10AC80003880003008B5124B2DED028B93F8F92176
:10AC9000D20719D493F8D5315B0715D58368DFED5A
:10ACA0000D7A03F5805303F2747203F5EF6392EDAE
:10ACB000008AD3ED000A28EE278A2CF043FE28EE06
:10ACC000000ABDEC028B08BD9FED030AF9E700BF47
:10ACD000388000300000C842000000000148F7F74B
:10ACE0000BBE00BF383000300148F8F71BBA00BF78
:10ACF000383000300148FFF715BE00BF3830003053
:10AD0000F0B55F4E04460D4696F8F9312DED028BF5
:10AD100013F0010F8FB005AF5FD143689B899A078D
:10AD20001CD5584865F06AFEDFED577A90ED007A41
:10AD3000B4EEE77AF1EE10FA10DD64F0C5FA3D21C9
:10AD400064F00AFA09220521A6F5A040FFF7EAFD02
:10AD500020B9092202212046FFF7CCFF636893F94E
:10AD60005430002B39D000230593089323691868C9
:10AD7000A0F052FE236AB0EE408A186803681B6D8B
:10AD8000984708AAF0EE400A3946B0EE480A204635
:10AD9000FFF7E6FADDED057A9FED3C7AF0EEE77A13
:10ADA000F4EEC77AF1EE10FA08D5DDED087AF0EE90
:10ADB000E77AF4EEC77AF1EE10FA0ED496F8D631AF
:10ADC0001B0704D464F080FA492164F0C5F996F8B1
:10ADD000D63143F0080386F8D63195ED027A08A8FB
:10ADE00095ED005AB1EE477A95ED016AB7EEC55A76
:10ADF000B7EEC66AB7EEC77A9FED1F0B8DED085B05
:10AE00008DED0A6B8DED0C7B31F04AFF636908A96B
:10AE10008DED0A1B8DED0C2B8DED080BDFED1C0A63
:10AE20009FED1C0A18689CF0ABFF636918689DF0E1
:10AE300011FA636918689DF0B9FB236A1D6863699C
:10AE400018689CF033FB384613498DED020ACDEDAE
:10AE5000030A8DED041AFCF785F9079B02A9284621
:10AE6000009397E80C0099F01DFD0FB0BDEC028B2C
:10AE7000F0BD00BFAFF300800000000000005940AB
:10AE800038800030809C003000002F4400000034E7
:10AE900000007A44000000000CAD00302DE9F041C4
:10AEA000AA4D0026044695F8D5312DED028B5A06A1
:10AEB00092B00596069603D5436918689BF0FEFF8D
:10AEC00095F8F931DB0755D463689B899F071BD53B
:10AED0009F4865F093FDDFED9F7A90ED007AB4EE28
:10AEE000E77AF1EE10FA0FDD64F0EEF93D2164F03F
:10AEF00033F9092205219848FFF714FD20B90922EA
:10AF000002212046FFF7F6FE636893F954308BB3B5
:10AF10009148F8F707F9E3689FED908AB6EE000ACA
:10AF20001B6820469FED8E7AD3ED0A7AF4EEC87A3C
:10AF3000F1EE10FA67FE877A27EE800AFFF758FADB
:10AF4000CDED060A8DED050AB0EEC00AB4EEC80AD2
:10AF5000F1EE10FA40F1AC80F0EEE00AF4EEC80A2F
:10AF6000F1EE10FA40F1A4807E4BB3F8403E980712
:10AF700000F1AE8095F8D7316FF3820385F8D731B1
:10AF800095F8D6311A0700F1A88077489EF034F87A
:10AF900095F8D7310EAF60F3820313F0040F85F8F4
:10AFA000D73140F09C80606901230E963A460F9697
:10AFB00005A900689BF0CAFF636918689DF04AF90B
:10AFC000636918689CF072FAA3688DED0B0ACDEDE9
:10AFD0000C0A8DED0D1AD3ED007AF5EEC07AF1EE84
:10AFE00010FA52DD614B20469FED618AB3F934358A
:10AFF00000EE903AF8EEE00ACDED030AFFF7FAFA18
:10B00000A368B7EE002A07EE900ADDED030AD3ED40
:10B01000001AB8EEE71A9FED4F0A31EE822A61EE70
:10B02000881A22EE082A2BF057FBDFED527A20EE29
:10B03000270ADFED517A20EE270A05F145FEDFED04
:10B040004F7A0BA820EE270A20EE088A2EF03EFF4A
:10B05000B4EEC08AF1EE10FA17D5C8EE006A9DED85
:10B060000B7ADDED0C7A636927EE267A67EEA67A15
:10B070008DED0B7ACDED0C7A1B68D3F8C422C3F8A2
:10B08000D022D3F8C822C3F8D422236A38463C49D8
:10B090001C68FCF767F8109B0BA92046009397E803
:10B0A0000C0099F0FFFB12B0BDEC028BBDE8F08103
:10B0B00095F8D631190704D464F006F9492164F0F3
:10B0C0004BF895F8D63143F0080385F8D63151E7AF
:10B0D00095F8D6316FF3C303F7E7002058E70DF179
:10B0E0001C08214807964146089609960A969EF044
:10B0F0000BF828B9A069A0F019FF03C888E803007D
:10B10000A069A0F01BFF09AA014617489EF062F84B
:10B110009DED087A9DED076A0123B7EEC77A606955
:10B12000B7EEC66A00930B960BAB0C9609AA39468C
:10B130008DED0E6B8DED107B00689BF03FFF95F859
:10B14000D7315B077FF52FAF36E700BF388000307F
:10B15000809C003000002F44383000300000003464
:10B1600000007A43389000303C9E00303860003058
:10B170000000C8420AD7233C35FA8E3C0AE81C413D
:10B180000CAD003013B504460191FFF787FE01991D
:10B19000204602B0BDE81040FFF74EBA1FB5194B6C
:10B1A000044693F8D6311B0729D4002301A9164879
:10B1B0000193029303939DF0B1FD032807D8DFE8C4
:10B1C00000F0150E020801A92046FFF799FD04B012
:10B1D00010BD0D489DF0C4FD30B10128F7D100210C
:10B1E0002046FFF7CFFFF2E70121F9E762F0F0F91F
:10B1F00040F242324FF4801162F0A0F9EFE70021F3
:10B20000EFE700BF38800030209F003008B50346CC
:10B2100019B9064A92F9042E1AB91846FFF7B2FF77
:10B2200008BDBDE80840FFF7B9BF00BF3890003047
:10B230000148FEF77FBD00BF38300030004870473E
:10B24000F87F00300148F7F743BB00BF38300030CB
:10B250000020704700207047002070470020704792
:10B260000020704700207047002070470020704782
:10B27000002070479FED010A704700BF00000000EA
:10B280000020704700207047002070470120704761
:10B290000020704700207047002070470120704751
:10B2A0000020704701207047012070470020704740
:10B2B000012070470120704700487047E4DE130802
:10B2C00000487047E4DE1308836803F5805393F861
:10B2D0008837DB0706D50023022280F83C30024B7A
:10B2E000C3F8D821012070473880003090F83C30F6
:10B2F00053B9836803F5805393F88837DB0742BF5F
:10B30000034B0122C3F8D821002380F83C3070475A
:10B3100038800030012380F83C3070472DE9F04739
:10B320002DED0C8BF0EE409A94B020EE000A002533
:10B33000F0EE60AA0446B0EE41CA8946A0EEA00A2B
:10B340009046F7EE00CA1F460295039504950595B1
:10B35000B7EEC00A0695079505F120FEB7EEC00BC3
:10B36000A3689FEDD8DA03F58053B4EEEC0A03F23C
:10B37000447203F5E963F1EE10FAD3ED000A92EDA1
:10B38000009AC8BFCCEE807A29EE0D9AC4BF69EE50
:10B39000A79A6AEEA7AAB0EE690A2CF0D3FAA368BE
:10B3A00029EE009A03F58053B0EE6A0A03F2447264
:10B3B00003F5E963D2ED008AD3ED000A2CF0C2FA5E
:10B3C000A36868EE8D8A03F5BA5203F5BB5392ED7C
:10B3D000078A68EE808AD3ED000AB0EE4C0A2CF0A2
:10B3E000B1FA636828EE0D8A93F96C3028EE008A72
:10B3F000002B00F0ED80236A9FEDB30A18684830F7
:10B4000030F024FDB0EE60AACDED0C0A8DED0D1AE2
:10B410008DED0B0A2BF0DEF9BDEEC0BA40F6B83266
:10B42000AA491BEE100A2BF089FA4342B0EE4A0AF1
:10B4300007EE903A6368F8EEE77A93ED197A67EED3
:10B44000877ACDED027A2BF0C5F9FDEEC0BA40F651
:10B45000B8329E491BEE900A2BF070FA42426368A4
:10B4600007EE902A049593ED1A7AF8EEE77A93F9AD
:10B470006C30022B67EE877ACDED037A6ED1944B58
:10B48000B8EECBBAB3F934350AEE103A236AB8EE07
:10B49000CAAA1A68B4EECABAF1EE10FA3DDDA36882
:10B4A0003AEE4B0ADFED8B0A03F5BA53A16B92ED2E
:10B4B000051A93ED017AD1ED001A27EE0D7AC7EE49
:10B4C000200A2BF06FFEDDED027A37EE800A8DED5B
:10B4D000020AB8EEEB0A236A1A68B4EECA0AF1EE61
:10B4E00010FA34DDA3683AEE400AA16B03F5BA53B3
:10B4F00092ED061AD1ED001AD3ED010A20EE8DDA95
:10B50000DFED740ACDEE200A2BF04CFEDDED037A60
:10B5100037EE800A8DED030A20E0B1EE4A0AB4EE60
:10B52000C0BAF1EE10FAD4D5A36830EE4B0AA16B85
:10B5300003F5BA53DFED670AD1ED001A93ED017AF6
:10B5400092ED051A27EE0D7AC7EE200AB9E7B1EEA3
:10B550004AAAB4EECA0AF1EE10FAC3D4236A0EAEB8
:10B560009FED590A08ADD3F800A00AF1480030F069
:10B570006DFC14AB8DED110ACDED120A8DED131A91
:10B580009FED550A13E9070086E8070085E80700E4
:10B59000284630F05BFC05AB02AA314650468DEDE3
:10B5A0000E0ACDED0F0A8DED101A99F00DFE6368AD
:10B5B00093F96C30022B16D1DDED057A39EE279A1E
:10B5C000DDED067A78EEA78ADDED077A38EE278A78
:10B5D00089ED009AC8ED008A87ED008A14B0BDECB1
:10B5E0000C8BBDE8F087F0EEE99ADFED3C0AF0EE57
:10B5F000EAAAAD20B0EECCCACDED019AB7EE001AA2
:10B60000F4EEE9AACDED08AA8DED0ECAF1EE10FA1E
:10B6100048BF01ADD5ED007AF4EECC7ADFED307A9B
:10B62000F1EE10FAD8BF354695ED007A87EE270A7D
:10B630003CEEC00A2BF02AF9E36905A8D3EDED7AB8
:10B6400020EE270A30F002FC8DED071AB0EEC91A81
:10B65000B520F0EEC07A8DED050ACDED060A39EE83
:10B66000000A31EE671AB0EEC11AF1EE410A2BF072
:10B670000DF9B0EE409A9DED060AB0EEE81ABA2038
:10B68000F0EEC07A38EE800A31EE671AB0EEC11AD9
:10B69000F1EE410A2BF0FAF8F0EE408A9DED070A30
:10B6A000B0EEC81ABF20F0EEC07A38EE000A31EED4
:10B6B000671AB0EEC11AF1EE410A2BF0E7F8B0EECE
:10B6C000408A85E70000C8429F0CB34548F4FFFF5D
:10B6D0003860003000007A44D3023739000000009F
:10B6E00000A08C4510B52DED028B836A044686B010
:10B6F00018686FF099F9E36AB0EE408A18686FF045
:10B7000093F9636B8DED010A18686FF08DF905AB45
:10B71000B0EE401A03A92046B0EE480A04AADDEDB7
:10B72000010AFFF7FBFD636A186890F8D110002941
:10B730003CD1A1F0C7FB2046FFF796F8636AB0EE54
:10B74000408A1B6893F8A91001293FD0032946D0ED
:10B7500051B9236A0121186899F0FCFC236A186822
:10B7600099F05AF89FED218A236A9DED030A186823
:10B77000A368026803F58053DDED040A9DED051A08
:10B7800093F888379B074CBF136BD36A9847236A9B
:10B79000174AB0EE480A18680021D2ED000A036883
:10B7A000DB6C984706B0BDEC028B10BD114B93F9D2
:10B7B000D521002A06DBD3F8D831022B04D190F82A
:10B7C000A9300BB90121B4E70221B2E7236A186856
:10B7D00099F0C0FC236A186899F034F8C2E7D97967
:10B7E0000029C1D12046FFF723FDBDE7000000007E
:10B7F0007865003038800030836803F6583393ED65
:10B80000000AB5EEC00AF1EE10FA01DCFFF726B827
:10B81000704700007047000000207047022070470A
:10B8200000207047002070470120704700207047BB
:10B8300081F001007047000001207047012070472F
:10B840000048704778DF13080048704784DF13080A
:10B8500038B54369044618689BF070FD18B96369F0
:10B8600018689CF0ADFD636920461D68FFF7EAFC8F
:10B870006368B3F93820B3F9363001EE102A00EED0
:10B88000903A4342B8EEC11A284600EE103AF8EE5C
:10B89000E00AB8EEC00A9BF021FC636920461D68EF
:10B8A000FFF7D0FC6368B3F93820B3F9363001EE06
:10B8B000102A00EE903A4342B8EEC11A284600EE34
:10B8C000103AF8EEE00AB8EEC00A9BF07DFC0120C9
:10B8D00038BD000030B504462DED028B436985B0BC
:10B8E0001D68FFF7AFFC6368B3F93820B3F9363051
:10B8F00001EE102A00EE903A4342B8EEC11A2846F3
:10B9000000EE103AF8EEE00A5E4DB8EEC00A9BF089
:10B91000E5FB2046FFF7E8F9B5F9343508EE103AB3
:10B92000236A1868B8EEC88A03681B6D984702AA94
:10B93000F0EE400A01A9B0EE480A2046FEF710FDDD
:10B94000636B18686FF070F82046FFF79BF9236B64
:10B95000F0EE408A20461B68B3F9083000EE103A3A
:10B96000B8EEC00AFFF7BAF92046B0EE408A8DED76
:10B97000030AFFF767FC6368B3F93630B0EE480A94
:10B9800001EE103A43422B2000EE903AB8EEC11A75
:10B99000F8EEE00A2AF07AFF20468DED030AFFF761
:10B9A0002BF9042813D8DFE800F0032F252A4B00D9
:10B9B000236A186898F030FF236A0021186899F00C
:10B9C00047FC63699FED300A18689CF097FD236A75
:10B9D000B0EE681ADDED020A18689DED010A0368F1
:10B9E000DB699847636918689CF0E0FD05B0BDEC21
:10B9F000028B30BD236A0121186899F029FC236A63
:10BA0000186898F01FFFDCE7204D2B7863B9636856
:10BA100045209FED1F1ADFED1C0A93ED040A2AF062
:10BA200035FF28460BF018FF20469DED030AFFF76F
:10BA3000ADF803A915488DED030A0BF049FFC6E7E1
:10BA4000636A02211868A1F03DFAB5F9343502AAFB
:10BA500001A900EE103A0F48B8EEC00A84F01AFCB3
:10BA600020469DED030AFFF791F80B488DED030A80
:10BA70000BF080F963699DED030A18689BF016FCD2
:10BA8000A5E700BF386000300000000034AE003091
:10BA900000007A44949D0030F87E0030002070470A
:10BAA00090F82133002B14BF1B20032070470000A7
:10BAB000002070470120704790F8DC02062804D06F
:10BAC000A0F10A0358425841704701207047000016
:10BAD000012070470020704790F82103034A044B6F
:10BAE000002814BF10461846704700BF18E013081E
:10BAF000CD7B150890F82103034A044B002814BF9E
:10BB000010461846704700BF24E01308CD7B150887
:10BB100090F8DC020B3818BF01207047054BD3F8B2
:10BB2000343D13F001031ABF90F8210380F00100A7
:10BB30001846704738700030024BD3F8340DC0F30C
:10BB4000C01070473870003090F8DC3223B9034BD6
:10BB5000187880F0010070470020704708AE003070
:10BB600038B590F8DC420546012C01D0002038BDE4
:10BB7000C368186803681B6998470028F6D1EB680A
:10BB800020461B6883F89C48F1E70000C368002248
:10BB900001201B6883F89C28704700007FB50023B4
:10BBA00005460C4680F82133B0F86C30012B01D8E3
:10BBB000002941D06B6A224E1B6893F8D1304BBBF1
:10BBC0000723204885F8DC320368022B02D10021CC
:10BBD000FBF7A0F8DFED1C0A0124EB68B0EE601A59
:10BBE0001868F0EE601AB0EE600A9FF003FA05F5EF
:10BBF000207085F8204331F03BF9144805F014F922
:10BC000096F8D63112486FF3C30386F8D6319CF00C
:10BC10008FFF11E096F9D431002BD1DA05F13C0009
:10BC200033F096F804460028CAD12846FFF706FBF1
:10BC3000084A022165F09EFB204604B070BD00BF9B
:10BC4000388000300CAD0030000000003CA7003010
:10BC5000209F00302CE0130810B50446094890F8E6
:10BC60000C31012B03D100F5847031F069F90648DD
:10BC700090F8511D00F54F6071F012FC002384F81C
:10BC8000213310BD38A000303890003008B5034B88
:10BC9000D3F88C0C9EF02EFD012008BD38900030AA
:10BCA00008B5034BD3F88C0C9EF006FD012008BDAF
:10BCB0003890003008B5034BD3F88C0C9EF00CFD87
:10BCC000012008BD38900030C3681B6818699BF0DC
:10BCD0002BBD000038B5D0F8E03204460D461BB944
:10BCE000B4F04AFAC4F8E002B4F046FAD4F8E0320C
:10BCF000C01A4FF47A73B0FBF3F0B4F8DE32984216
:10BD000009D32046FFF79AFA2B88044A062165F0EA
:10BD100031FB012038BD0020FCE700BF48E01308DC
:10BD200090F8DC32052B05D1054BD3F8943CD8684C
:10BD30009BF06ABCC36818680368DB68184700BFDB
:10BD40003890003090F8DC328B4206D00B2B80F814
:10BD5000DC1202D10148FCF70DBF704738300030CB
:10BD6000F8B505463C300F46264E33F075FC0446C8
:10BD7000002842D0012385F87130234BD6F8E0210A
:10BD80009A4212D1012385F82133D6F8E0010368E5
:10BD90001B6898473A4601461C4862F0E3FD96F856
:10BDA000D5319B0623D42046F8BD3A4603212846C8
:10BDB000FEF7A0FF0028E5D185F871002846FFF7BF
:10BDC0003DFA134A042165F0D5FA63F07DFA1B228F
:10BDD0000A2163F0E1F996F8D54114F02004E2D08D
:10BDE0000C4A0024137843F004031370DBE7094A7C
:10BDF000137843F002031370D5E72846FFF71EFAC5
:10BE0000054ADFE73880003004A10030F47D0030BF
:10BE10005CE0130884AF00307BE0130830B50446C3
:10BE200085B00F480BF034F90546B0B1072301A9DE
:10BE300084F8DC320023019302930393E3681868CB
:10BE40009EF0C6FBE36801A90022186803685B68DE
:10BE5000984700210348FAF75DFF284605B030BD3A
:10BE6000383000300CAD0030F0B5414F05460C467F
:10BE7000D7F8642CD7F8603C1343D7F85C2C1343F5
:10BE80002DED028B87B00CD161F0A2FB4FF49B72B9
:10BE90004FF4801107B0BDEC028BBDE8F04061F0BB
:10BEA0004DBB8069A0F044F82046B0EE408A16F001
:10BEB0000FFF032839D1EB6801A918689EF070FCC8
:10BEC000064690B3DDED017A636838EE678A009329
:10BED000284B0021DFED287A93F9D4319FED270A12
:10BEE000002B009B264827FE800A38EE008ABDEE14
:10BEF000C88A18EE102A9342ACBF00930092FAF75A
:10BF000009FF6B6918689CF05BFADDED007A314639
:10BF10002846B8EEE70A0BF095FF00212846FFF708
:10BF200011FF07B0BDEC028BF0BD94E80F0002AE2C
:10BF300086E80F00D7F8603C6A4602213046049339
:10BF4000D7F8643C059316F0CFFE78B963F0BCF9DE
:10BF50000222152163F020F9DDED037AF8EEE77A8D
:10BF600077EE887AFDEEE77ACDED007A0026AFE72E
:10BF70003890003038800030000000000000C842D7
:10BF80000CAD003030B5C3688BB004460D46186860
:10BF90009EF0FAFB88BB002301930293039394F86D
:10BFA000DC32F3B90022002304A92046CDE90423A2
:10BFB000CDE90623CDE908230BF07EFF88B19DED86
:10BFC000067B9DED045BF7EEC76BB7EEC55B9DEDA1
:10BFD000087B8DED015ACDED026AB7EEC77B8DED82
:10BFE000037AE368DDED010A9DED021ADDED031A27
:10BFF0009FED0C0A18689EF0FDFFE368294618685B
:10C000009EF022FF054650B107480368022B02D07C
:10C010000021FAF799FE01212046FFF793FE2846FA
:10C020000BB030BD000000000CAD003010B52DEDA0
:10C03000028BC3680446DFED358A1B684269D3ED85
:10C040000A0A9FED338AF4EEE80A93ED060A1068B7
:10C05000F1EE10FA60FE880A9AF0B2FEE3686269B7
:10C060001B681068D3ED0A0A93ED060AF4EEE80A9D
:10C07000F1EE10FA60FE880A9AF018FF63691868FA
:10C080009BF01EF818B9636918689BF0CBFFE36852
:10C0900062691B68106893ED080A93ED0C1AD3EDE2
:10C0A000070AB0EEC00A9BF019F8E36862691B68E2
:10C0B000106893ED080A93ED0C1AD3ED070AB0EE61
:10C0C000C00A9BF081F8636918689BF037F918B9CA
:10C0D000636918689CF074F900210E48FAF71AFE9B
:10C0E0000D4886F063FA0D4880F05EFB0C4A20464E
:10C0F0000221B2F8D63123F48163A2F8D631BDEC27
:10C10000028BBDE81040FFF71DBE00BF00000034E9
:10C1100000007A430CAD00301C9E00301C620030E1
:10C12000388000300C4B10B50446D3F8940C90EDD9
:10C130000F0A00F1200190F860209DF063FF07488E
:10C140000368022B02D00821FAF7E4FD20460521FE
:10C15000BDE81040FFF7F6BD389000300CAD003060
:10C1600010B52DED028BC3680446DFED2F8A1B68E6
:10C170004269D3ED0A0A9FED2D8AF4EEE80A93EDA9
:10C18000060A1068F1EE10FA60FE880A9AF018FEAE
:10C19000E36862691B681068D3ED0A0A93ED060A2A
:10C1A000F4EEE80AF1EE10FA60FE880A9AF07EFEDC
:10C1B000636918689AF084FF18B9636918689BF07E
:10C1C00031FFE36862691B68106893ED080A93ED1C
:10C1D0000C1AD3ED070AB0EEC00A9AF07FFFE368AD
:10C1E00062691B68106893ED080A93ED0C1AD3ED91
:10C1F000070AB0EEC00A9AF0E7FF636918689BF07F
:10C200009DF818B9636918689CF0DAF800210848AD
:10C21000FAF780FD09212046FFF794FD0123BDECCC
:10C22000028B84F8043310BD0000003400007A4310
:10C230000CAD003010B504460748D0F8343D9B07DC
:10C2400004D50121A0F58040F6F7AAF92046BDE803
:10C2500010400BF023BC00BF3870003030B589B0FF
:10C260000446FEF753F930B10021204609B0BDE87D
:10C270003040FEF783B9636A02211868A0F022FEFD
:10C28000E368186803685B69984701461048FCF743
:10C2900051FF636918689CF089F9236A1D68636916
:10C2A00005AC18689BF002F920460A498DED020A98
:10C2B000CDED030A8DED041AFAF754FF079B02A98E
:10C2C0002846009394E80C0098F0ECFA09B030BDD1
:10C2D000383000300CAD003038B50446FEF716F9A2
:10C2E000054628B120460021BDE83840FEF746B992
:10C2F000636A02211868A0F0E5FD29462046BDE8E2
:10C300003840FEF783BF00000021014807F0D0B994
:10C310009CA8003030B5174D89B09FED170A044630
:10C3200005F5C043D3F8940C9DF0DAFE014628468B
:10C33000FCF700FF636918689CF038F9236A1D68F0
:10C34000636905AC18689BF0B1F820460B498DED88
:10C35000020ACDED030A8DED041AFAF703FF079BDD
:10C3600002A92846009394E80C0098F09BFA09B0C3
:10C3700030BD00BF38300030000000000CAD003090
:10C3800030B589B00446FEF7C1F830B1002120462F
:10C3900009B0BDE83040FEF7F1B8636A02211868C1
:10C3A000A0F090FDE368186803685B699847014650
:10C3B0001048FCF7BFFE636918689CF0F7F8236A21
:10C3C0001D68636905AC18689BF070F820460A493F
:10C3D0008DED020ACDED030A8DED041AFAF7C2FEC7
:10C3E000079B02A92846009394E80C0098F05AFA9B
:10C3F00009B030BD383000300CAD003030B52DED17
:10C40000028B83B00446FEF781F820B9636A1B688B
:10C4100093F8D23043B90021204603B0BDEC028B23
:10C42000BDE83040FEF7AAB894F8E432DA071DD42C
:10C43000E3681D682B6828469B689847D5ED097A04
:10C4400094F8E432B4EEE70AF1EE10FA4CBF0122A0
:10C45000002262F3000384F8E43207D4204603B0DC
:10C46000BDEC028BBDE83040FFF7F8BE94F8E43233
:10C470009B0732D4E368DFED448A1B686269D3ED21
:10C480000A0A9FED428AF4EEE80A93ED060A106864
:10C49000F1EE10FA60FE880A9AF092FCE368626995
:10C4A0001B681068D3ED0A0A93ED060AF4EEE80A59
:10C4B000F1EE10FA60FE880A9AF0F8FC63691868D9
:10C4C0009AF0FEFD18B9636918689BF0ABFD94F80B
:10C4D000E43243F0020384F8E4322D4BD4F8EC222A
:10C4E000D3F85C3C9B1A07EE903AB8EEE78AF1EE7F
:10C4F000047AB0EEC87AB4EEE77AF1EE10FA38D5E5
:10C5000094F8E43243F0040384F8E432204684EDE6
:10C51000BA8AFEF7C3FC6369A26BB1EE480A1B68D6
:10C52000D2ED001A93ED991AD3ED0E0A2AF03AFED5
:10C53000636940F25E401B6893ED961AD3ED970A4B
:10C540002AF0A4F92046FEF721FB12488DED010ADE
:10C550000AF010FC63699DED010A18689AF0A6FEC6
:10C560006369186803B0BDEC028BBDE830409CF0F5
:10C570001DB8D4EDBA7A68EE277AF5EEC07AF1EEFE
:10C5800010FAC3D5BCE700BF0000003400007A43B6
:10C5900038900030F87E003030B52DED028B83B03E
:10C5A0000446FDF7B3FF20B9636A1B6893F8D230E5
:10C5B00043B90021204603B0BDEC028BBDE83040FA
:10C5C000FDF7DCBF636940F27640DFED327A642527
:10C5D0001B6894EDCB0A93ED961AD3ED970A20EEE3
:10C5E000270A2AF053F92046FEF7D0FA236AB0EE64
:10C5F000408A186803681B6D9847274B6846B3F953
:10C60000343507EE903AB4F82433F8EEE77A13FBAA
:10C6100005F307EE103A94F92633B4EEE70A13FB5C
:10C6200005F3F8EEC76AF1EE10FA07EE103ACDED19
:10C63000006AB8EEC77A77FE807A9FED180AF4EEAA
:10C64000407A8DED017AF1EE10FA58BFB0EE670A2C
:10C650002DF058FC236A0121DDED010A1868B4F8B9
:10C660002833026813FB05F39DED000A126A01EE00
:10C67000103AB8EEC11A90476369B0EE480A1868DC
:10C680009AF014FE636918689BF090FF03B0BDEC4C
:10C69000028B30BD0000C8423860003000007A4490
:10C6A00010B5436A02461C6894F8D10068B1084B83
:10C6B00093F8D41111F0200308D00B0603D592F89B
:10C6C0000433012B02D994F8D20010BD0020FCE7FE
:10C6D0003880003010B50446FEF7E0FB00219FEDE6
:10C6E000060A636918689AF07BFD6369BDE810402B
:10C6F00018689BF05BBF00BF0000000010B5044647
:10C70000FEF7CCFB0121636994EDC60A1868B1EE0F
:10C71000400A9AF065FD6369BDE8104018689BF017
:10C7200045BF000070B52DED048B82B00446FFF7C5
:10C73000B7FF014638B9204602B0BDEC048BBDE816
:10C740007040FDF7F5BE636A02211868A0F0BAFBDD
:10C75000236A1B6893ED2E8AB3F00EFDB44B054699
:10C76000B3F8D43103F4814373B194F80433022B4A
:10C770000AD12046FEF762FDAE4BAF4A062164F0B7
:10C78000F9FD032384F80433A06860307FF0BCFA1D
:10C7900050B1A06860307FF0C1FA28B194F804333A
:10C7A000012B11D9022B1FD094F80433082B00F26F
:10C7B0009381DFE813F023003D006A0021015B0153
:10C7C00063017B018A012D0009212046FFF7BAFA97
:10C7D0002046FEF733FD974B984A062164F0CAFDC8
:10C7E000082384F80433DFE72046FEF727FD914B4A
:10C7F000924A062164F0BEFD0323F2E7904BD3F882
:10C800008C0C03681B69984710B12046FFF7A8FC01
:10C8100094F80433082B00F28881DFE813F06601F6
:10C820006E016E0176017601760176017E017E0150
:10C83000A069C4F808539FF07BFBA3689FED817A41
:10C8400003F5BF5384EDC50AD3ED067AF4EEC77A3B
:10C85000F1EE10FA46DB9FED7C7A67EE877AE368AB
:10C860001B6893ED087A4FF07E53B0EEC77AC4F898
:10C8700010330223F4EE477A84F80433F1EE10FA11
:10C8800048BFB0EE677A84EDC67AD4EDC77A9FEDE3
:10C890006D9AF0EEE77AF4EEC97AF1EE10FA2DD542
:10C8A00063699FED6A7AD4EDC67A1B6867EE877A72
:10C8B00093EDAA7AB4EEE77AF1EE10FA38DCD4F808
:10C8C0000833D4EDC47AEB1AB3F5FA6F33D2B4EE71
:10C8D000678AF1EE10FA37FE888A84EDC48AC4F8BC
:10C8E0000C5395E76368B3F93230002BB8BF5B4255
:10C8F0009BB207EE903AF8EEE77AB0E7D4EDC58A3E
:10C90000A0699FF015FB38EEC00AD4EDC77AB4EEEB
:10C91000E70AF1EE10FAC3DD0623204684F804335B
:10C92000FEF78CFC434B4A4A042164F023FD6FE779
:10C93000C4F808536CE7A36803F5805303F2EC7264
:10C9400092ED007A67EE877AF4EEC87AF1EE10FA8B
:10C95000C5D403F5FE63D3ED007AF4EEC97AF1EEA7
:10C9600010FA29DB3B4E96F8703EDB0708D406230D
:10C97000204684F80433FEF761FC2E4B364AD3E799
:10C98000A6F580400AF016F9B0B196F98E3E9BB933
:10C99000B6F9723EDFED2C6A07EE103AA36803F594
:10C9A000BF53B8EEC77AD3ED047A67EEA67AB4EE39
:10C9B000E77AF1EE10FA92DCD4F80C03281AB0F5FD
:10C9C000FA7F7FF625AF0323204684F80433FEF771
:10C9D00035FCA368D4EDC47A062103F5BF531F4A82
:10C9E00093ED037A134B27EE277AB7EEC77A8DEDD6
:10C9F000007B64F0BFFC0BE7636918689BF04AFD9D
:10CA0000A06860307FF080F978B12046FEF716FC10
:10CA1000084B134A062164F0ADFCA06860307FF03B
:10CA200061F9042384F80433F2E60523FAE700BF32
:10CA300038800030B8E01308C6E01308D0E01308CF
:10CA400038900030000000340000C842333373BF18
:10CA5000E2E0130838700030FDE013082DE1130800
:10CA600055E1130800007A440000FA43A0686030E2
:10CA70007FF04AF910BB052384F80433A368D4F887
:10CA80000C0303F5BF535FED097A1FED097A2D1AE8
:10CA9000D3ED056AA6EEA77A07EE905AF8EE677A0C
:10CAA000F4EEC77AF1EE10FA3FF5B2AE002194ED44
:10CAB000C50A20460BF0C6F90723B3E7A06860302B
:10CAC0007FF02CF90028D6D1A2E61A4B1B78002B58
:10CAD0003FF49EAE0823A5E760F07AFD4FF4A8620C
:10CAE0004FF4801160F02AFD92E6204602B0BDECC2
:10CAF000048BBDE87040FFF7B1BB204602B0BDEC2F
:10CB0000048BBDE87040FFF7F9BD204602B0BDECD4
:10CB1000048BBDE87040FFF7DDBD204602B0BDECE0
:10CB2000048BBDE87040FFF785BB02B0BDEC048B01
:10CB300070BD00BF08AE0030F0B5044687B00846AF
:10CB40000E4616F0C5F80328074602AD16D1E36875
:10CB500018689DF061FC012810D1294612480AF09E
:10CB6000C7F8044638B102993A46C829B8BFC82167
:10CB7000304616F083F8204607B0F0BD0B4B0FCBC4
:10CB800085E80F00304616F0A3F80146284616F057
:10CB900007F904460028EED003992846019116F0C3
:10CBA00097F801990246E3E738300030909C003056
:10CBB000083230B504461D4685B00FCA84E80F0020
:10CBC000134301BFAB68A360EB68E360636893B98C
:10CBD000204616F07DF803AA0146284616F084F890
:10CBE00060B103992046019116F072F8019902464E
:10CBF000204616F043F8204605B030BD6968284647
:10CC00000191F1E730B50B6985B004460BB94B696A
:10CC100053B3002308316D46C4F800330FC985E8CB
:10CC20000F0029462046FFF787FF98B9124B0122D3
:10CC30002846D3F85C1C16F021F862F045FB02226E
:10CC4000152162F0A9FA2046FEF7F8FA0B4A0221F4
:10CC500064F090FB29462046FFF794F910B9084884
:10CC6000FCF77CFB05B030BD0123C0F8003305B0F4
:10CC7000BDE83040FFF7DAB93890003070E11308B2
:10CC80003830003030B508318FB0054606AC0FC9DA
:10CC900084E80F00134312D1002303A903930493E4
:10CCA00005931A4BD3F88C0C9DF078FC022203A953
:10CCB0000AA816F01DFB0C9B08930D9B0993079B7C
:10CCC00093B9204616F004F80AAA0146104816F057
:10CCD0000BF898B10A992046019115F0F9FF0199D6
:10CCE0000246204615F0CAFF21462846FFF74AF9BA
:10CCF00010B90848FCF732FB0FB030BD0348D0F83C
:10CD00005C1C00F658400191E7E700BF3890003006
:10CD1000909C00303830003038B504460D46FFF79F
:10CD2000B1FF0023C4F8E032AB88A4F8DE3238BD8E
:10CD30007FB50D460446FFF7A5FF6E4605F10801D5
:10CD40000FC986E80F00134306D1234BD3F8602C9C
:10CD5000D3F8643C0292039304F53B720121304600
:10CD600015F0C2FF94F8E43270B923F005032046B1
:10CD700043F0050384F8E432FEF760FA174A06210F
:10CD800064F0F8FA04B070BD23F00703626984F818
:10CD9000E4320023C4F8E832E36810681B6893EDBE
:10CDA000080A93ED0C1AD3ED070AB0EEC00A9AF008
:10CDB00095F9E36862691B68106893ED080A93EDC2
:10CDC0000C1AB0EEC00AD3ED070A9AF0FDF908215B
:10CDD0002046FEF7B7FFD5E7389000309CE11308F6
:10CDE0002DE9F0438DB088461C4607466D46134634
:10CDF0000A4601462846DDE91469FFF7D9FE95E8A1
:10CE00000F0084E80F0007A815F032FFB8F80430CF
:10CE1000F3B9B8F8001005AA07F13C00013189B256
:10CE200031F040FFA0B1234605AA39462846FFF756
:10CE3000BFFE95E80F0086E80F00BDF81630A3F19D
:10CE400052025342534189F800300DB0BDE8F083DF
:10CE500094E80F0086E80F000023F4E770B58B8894
:10CE600092B004460D461646002B47D10DA815F08A
:10CE7000FFFE29880BAA04F13C00013189B231F090
:10CE800011FF00283AD0BDF82E1052291CD019D815
:10CE9000112913D80F2913D933462A46214603A84E
:10CEA000FFF786FE03AB214607A80BAAFFF780FE1B
:10CEB000E36807A918689EF007F801E01329EBD092
:10CEC00012B070BD5E29FAE707AD03A815F0D0FED9
:10CED000284615F0CDFE0DF10B0332460BA9204676
:10CEE000CDE9005303ABFFF77BFFE0689DF80B3003
:10CEF0002A4603A900689DF0BDFFE1E70120DFE7B6
:10CF000070B51F4B88B004460E466D460FCB85E8C2
:10CF10000F00E36818689DF037FC98B1E368186863
:10CF200003681B69984768B1E368294618689DF053
:10CF30007FFA38B960F04CFB40F2C4524FF48011D4
:10CF400060F0FCFA214604A82B463246FFF730FE7B
:10CF500004A92046FFF716F820B90A48FCF7FEF9A5
:10CF600008B070BD002304AA31462046C4F8E03260
:10CF7000B388A4F8DE32FFF771FF0028F0D1ECE7A8
:10CF8000909C003038300030F0B52C4B91B0044606
:10CF90000E4604AD0FCB85E80F00E36818689DF0DE
:10CFA000F3FB98B1E368186803681B69984768B198
:10CFB000E368294618689DF03BFA38B960F008FB31
:10CFC00040F2A4624FF4801160F0B8FA0CAF08A8E8
:10CFD00015F04EFE384615F04BFE0DF10F032A46B4
:10CFE00031462046CDE9007308ABFFF7F9FEE06853
:10CFF0009DF80F303A4608A900689EF07BFA20B9E8
:10D000000F48FCF7ABF911B0F0BD002508AA314676
:10D010002046C4F8E052B388A4F8DE32FFF71EFFC2
:10D020000028EDD007480368022B02D02946F9F703
:10D030008BFE01212046FEF785FEE4E7909C003040
:10D04000383000300CAD0030DFED0A7A91ED041A73
:10D05000D1ED030A91ED020A21EE271A8B884FF4D5
:10D060007A7160EEA70A044820EE270A594303F0BC
:10D07000E5BE00BF0000C8423CA7003037B50446FB
:10D080000D46B3F079F8C4F8F402D5ED027AF5EE66
:10D09000C07AF1EE10FA17DD9FED137A67EE877A0A
:10D0A000FCEEE77AC4EDBC7A2046FEF7C7F8D4F868
:10D0B000F0224FF47A730621B2FBF3F30B4A03B06C
:10D0C000BDE8304064F056B97FF0B2F9002395F91D
:10D0D0000D20009395F90C1095F90E307FF0C4F8EF
:10D0E000C4F8F002E0E700BF00007A44B4E113089E
:10D0F00010B5B1F90A300446A0F8243391F90C3088
:10D1000080F82633B1F90D30A0F82833B1F90F308B
:10D1100007EE903AF8EEE77AC0EDCB7AB3F02CF850
:10D120000B21C4F830032046BDE81040FEF70ABECC
:10D1300038B504460D46B3F01FF89FED067AC4F8E3
:10D14000FC02D5ED027A67EE877AFDEEE77AC4ED50
:10D15000BE7A38BD00007A444A7C0B460548003A46
:10D1600091F91010D3ED030A18BF012293ED020AC2
:10D17000F9F7F4BD0CAD003070B51B4E044686B017
:10D180000D46D6F8E00103681B689847042806D1CD
:10D190006B88102B0FD0732B20D000201CE0D6F80A
:10D1A000E00103681B6898470328F6D194F8DC3245
:10D1B000062BF2D1ECE705F1080102ACDFED0B0A1A
:10D1C0000FC984E80F000023B0EE600A214608482A
:10D1D0001A46009303F0A0FC06B070BD2046294615
:10D1E000FFF7BAFF0120F7E73880003000000000A9
:10D1F0003CA70030D1F8093000EE103AB5EEC00A75
:10D20000F1EE10FA11DD0B7A084ADFED097A022BF4
:10D21000D2F88C0C20EE270A01D19DF04DBA032BD9
:10D2200001D19DF059BA9DF065BA70473890003031
:10D230000000C8428B88012B05D00B693BB94B69B4
:10D240002BB9CB681BB900210348FAF7FFBB0022BA
:10D2500008310148FAF7A8BB3830003038B5124D14
:10D260000C4605F54F6095F8511D70F0FBF868B15C
:10D2700095F8511D05F54F6070F0FCF830B9DFED01
:10D280000B0A94ED040A0A48F9F7D8FD94ED041A44
:10D290000022D4ED020A94ED030A95F8511D0548C9
:10D2A000BDE8384070F018B9389000300000000038
:10D2B0000CAD0030289D00304B7A012B08D0022B9A
:10D2C00010D0CBB9826802F5805282F824357047BD
:10D2D0008068D1F80A3000F5A85000EE103A1830F6
:10D2E000A6F0BEB98068D1F80E3000F5A85000EE67
:10D2F000103A1830A6F0C8B9704700007FB50B6926
:10D3000004460E460BB94B69BBB300236D4684F847
:10D31000043306F108030FCB85E80F0029462046A9
:10D32000FFF70AFC98B9164B01222846D3F85C1C7B
:10D3300015F0A4FC61F0C8FF0222152161F02CFF5A
:10D340002046FDF77BFF0F4A022164F013F82946BF
:10D350002046FEF717FE20B90B48FBF7FFFF04B08D
:10D3600070BD09212046FEF7EDFCB38807EE903A28
:10D37000F8EE677AC4EDC77AF1E7FEF7F1FEF4E75D
:10D3800038900030C4E113083830003010B5044C38
:10D39000237813B1034885F003F9207810BD00BF4E
:10D3A00008AE00301C9E003090F80403072894BF9C
:10D3B0000020012070470000094B13B50446D3F844
:10D3C0008C0C019103681B69984730B10199204684
:10D3D00002B0BDE81040FEF77DBC02B010BD00BF3A
:10D3E0003890003090F8E43213F0010018BFC3F316
:10D3F00080007047094A034692F8A10868B192F884
:10D40000A028043A012A07D85B6A1B6893F8A90090
:10D41000431E5842584170470020704738A00030E2
:10D4200010B50446B2F0A8FED4F8FC32C01AD4F805
:10D43000F83223EAE37398424FF0000084BFC4F847
:10D44000F802012010BD000010B5036804465B6DB2
:10D450009847D4F8F83223EAE37398424FF000007B
:10D460003CBFC4F8F802012010BD000004480321AD
:10D4700008B5F9F74FFC0248BDE80840F9F742BD8E
:10D480000CAD00301C4B70B50446D3F88C0C0E4626
:10D4900003681B699847054610B90025284670BDEA
:10D4A000D4F8E0325BB9B2F067FEB4F8DE32C4F80B
:10D4B000E00223B1114A537843F001035370B2F0F4
:10D4C0005BFED4F8E022B4F8DE32801A4FF47A72B0
:10D4D000B0FBF2F09842E0D323B9084A537843F006
:10D4E000010353702046FDF7A9FE3388044A062144
:10D4F00063F040FFD2E700BF3890003084AF0030C7
:10D5000048E0130810B590F8DC320446042B124BA7
:10D510000AD1D3F88C0C03681B69984718B12046D0
:10D52000FEF700FE002010BDD3F8943CDFED0B7A2F
:10D53000D3ED126A0B7986EEA77A07EE903AF8EEF1
:10D54000E77AB0EEC77AB4EEE77AF1EE10FAACBF44
:10D5500001200020E7E700BF38900030DB0FC94012
:10D56000094B13B50446D3F88C0C019103681B6971
:10D57000984730B10199204602B0BDE81040FEF74F
:10D58000A9BB02B010BD00BF389000308B8813B12A
:10D59000024803F071BC0120704700BF3CA7003077
:10D5A00010B50446B2F0E8FDD4F8F432C01AD4F84D
:10D5B000F03298424FF0000084BFC4F8F00201201E
:10D5C00010BD000038B505460C46B2F0D5FD4FF44D
:10D5D0007A72D5F83033C01A23895343984294BFE6
:10D5E0000020012038BD00001FB50B46014618463B
:10D5F0002CF04AFF68468DED000B8DED021B2CF0E0
:10D6000071FFB7EEC00B05B05DF804FBF0B5514DEE
:10D6100004460E461746D5F8940C2DED028BB0EE5D
:10D62000408A8FB09CF030FBDFED4B8AF0EEC87A79
:10D63000F4EEE87AF1EE10FA07D49FED480AD5F837
:10D64000940C28EE000A9CF081FBD5F8940C90ED28
:10D650000F0AB0EEC00A0FB1B1EE400A9CF066FBB3
:10D66000002303A9D5F8940C0393049305939CF02D
:10D6700089FBA0699EF058FC03A92EF0D1FB0AA8F3
:10D680008DED0A0ACDED0B0A8DED0C1A2EF0FCFF84
:10D69000DFED337AB4EEE70AF1EE10FA56DD02223E
:10D6A00003A90AA815F024FE71683046019115F00F
:10D6B0000FFB019902460AA815F0E0FAE3680AA9EF
:10D6C00018689DF0C1FB10B92648FBF747FEA0691A
:10D6D0009EF02CFC90ED017A90ED006A06A8B7EE62
:10D6E000C77AD5F8941CB7EEC66A20318DED066B6B
:10D6F0008DED087BFFF778FF1B4B1B68022B1AD0C0
:10D70000D5F8943C00211848D3ED0E7AF4EEE87A6F
:10D71000F1EE10FAB8BFD3ED047AB4EEE70AF1EEF9
:10D7200010FA10DDDFED117AB4EEE70AF1EE10FA2F
:10D7300009DDF9F709FB04212046FEF703FB0FB0D2
:10D74000BDEC028BF0BDF9F7E5FAF4E72046FEF7F1
:10D75000E9FCF4E738900030000000340000C842D3
:10D7600000009643383000300CAD00300000FA4322
:10D7700030B585B00C460A460F4B01460546684653
:10D78000FFF716FA6288A388122A4FEA132305D1FD
:10D79000227ED20744BF03EB83035B0007EE903A7F
:10D7A000227A69462846B8EE670AC2F34002FFF7BC
:10D7B0002DFF05B030BD00BF909C00301FB590F824
:10D7C000DC32052B1DD1124BD3F8943CDC68A068E9
:10D7D0009EF0ACFB90ED017A90ED006A04F52271A9
:10D7E000B7EEC77A6846B7EEC66A8DED027B8DED5F
:10D7F000006BFFF7F9FEBCEEC00A10EE100A04B091
:10D8000010BDC368186803689B689847F3E700BFBA
:10D810003890003010B5012104460A4805F0CCFAD2
:10D8200028B120460321BDE81040FEF78BBA5FF017
:10D83000CFFE4FF496724FF48011BDE810405FF0B8
:10D840007DBE00BF9CA8003010B5012104460B48E6
:10D8500002F03EFE48B95FF0BBFE4FF400724FF499
:10D860008011BDE810405FF069BE044803F0F2FA91
:10D8700020460621BDE81040FEF764BA3CA7003000
:10D880008B880BB1FFF7E0BF7047000038B5044646
:10D890000D4687484FF4807109F060FC28B12A4694
:10D8A00004F13C01834861F091F86B885E2B4DD800
:10D8B000512B05D8103B9AB20F2A21D900205DE0E8
:10D8C000523B0C2BFAD801A252F823F017DA0208C7
:10D8D000BDD80208C5D90208DDD90208BDD80208A2
:10D8E000BDD80208BDD80208BDD80208BDD80208BC
:10D8F000BDD8020821DA02082BDA020835DA02085C
:10D900000F2BDBD801A252F823F000BFD3D90208B5
:10D91000E7D90208F1D90208FBD902080FDA020898
:10D92000DDD90208C5D90208BDD80208BDD8020851
:10D93000BDD80208BDD80208BDD80208BDD802086B
:10D94000BDD80208BDD8020805DA0208C92B00F0CC
:10D95000908014D8B22B00F082800AD8722B6ED03F
:10D96000732B77D0702BA9D129462046FFF7E0FB17
:10D970002DE0B32B78D0BD3B5842584138BDDE2B4B
:10D9800000F08B8011D8CD2B79D0CF2B96D1A988E0
:10D99000002979D148487EF0E3FE2046FDF74EFC91
:10D9A000464A062163F0E6FC11E04AF268629342BF
:10D9B00078D04AF2CF62934280D129462046FFF7C1
:10D9C00097FB04E005F108012046FEF74DFA01201F
:10D9D000D4E729462046FFF793FAF8E72946204680
:10D9E000FFF710F9F3E729462046FFF74BF9EEE77A
:10D9F00029462046FFF7BCFEE9E729462046FFF707
:10DA00008BF9E4E729462046FFF792F9DFE7204645
:10DA1000FFF700FFDBE729462046FFF7B5FAD6E718
:10DA200029462046FFF72CFFD1E729462046FFF77D
:10DA300025FBCCE729462046FFF760FCC7E7D5ED7C
:10DA4000027A9FED1F7A67EE877AFDEEE77AC4EDE2
:10DA5000BE7ABCE729462046FFF77EFBB7E729469A
:10DA60002046FFF7C7FBB2E729462046FFF7E2FB57
:10DA7000ADE705F108011348F9F700FAA7E72946D1
:10DA80002046FFF7EBFBA2E701210B487EF068FE82
:10DA90002046FDF7D3FB0C4A83E729462046FFF7D3
:10DAA000D3FA94E729462046FFF706FC8FE700BF2C
:10DAB00038300030F47D00301C620030F8E113088B
:10DAC0000000C8420CAD003007E2130890F8DC32C9
:10DAD000022B04D0032B04D1034805F03DB90120EB
:10DAE00070470020704700BF9CA8003038B50C4B31
:10DAF0000446D3F8345D90F8DC3205F00405032BBE
:10DB00000AD1084805F040F994F8DC3235B110B973
:10DB1000023B5842584138BD0020F5E70120FAE7A2
:10DB2000387000309CA800300F4A10B513780446B6
:10DB300043F0800313700D4B93F9D421002A09DBC5
:10DB4000FEF76CF970B9204608220921BDE81040A3
:10DB5000FDF7D0B801220E21A3F1D000BDE810409E
:10DB6000F4F79CBC10BD00BF84AF0030388000309B
:10DB7000F8B5D0F8004305465CB1012C1AD05FF02F
:10DB800027FD4FF4FC624FF4801101245FF0D6FCB6
:10DB900007E0184BD3F88C0C03681B69984710B941
:10DBA00000242046F8BD2846FEF740FA0123C5F8B8
:10DBB0000033F6E7104F97F9D431002BF0DA436ABF
:10DBC0001B6893F8A960012EEAD13C3031F0B2F81D
:10DBD00004460028E5D1D7F8043293F8D13033B1A8
:10DBE00032460D21A7F1D000F4F758FCD9E73446AE
:10DBF000D7E700BF389000303880003038B5614B2F
:10DC000004460D46D3F8E0215F4B9A4201D0002034
:10DC100021E04B885E2B65D8512B1DD8103B9AB262
:10DC20000F2A39D92046FDF709FB6B88574A042192
:10DC300063F0A0FB08E0C93B01229BB202FA03F3A8
:10DC4000534A1A40002AEDD02046FDF7F7FA2988FA
:10DC50006BF0EEFB012038BD523B0C2BE2D801A249
:10DC600052F823F05FDD020825DC020823DD0208FC
:10DC700037DD020825DC020825DC020825DC020865
:10DC800025DC020825DC020825DC020865DD020827
:10DC90006BDD02083FDD02080F2BC3D801A252F84A
:10DCA00023F000BF31DD02080FDC020845DD020869
:10DCB0004BDD020859DD020837DD020823DD0208CA
:10DCC00025DC020825DC020825DC020825DC020828
:10DCD00025DC020825DC020825DC020825DC020818
:10DCE00051DD0208732B49D006D8702B43D0722B1C
:10DCF00098D1FFF7A9FB17E04AF2CF62934237D0E1
:10DD000090D8DE2B09D8C82B95D8B32B02D8B12BCD
:10DD100088D999E7BD2B97D084E74AF2686293428D
:10DD2000F9E72046FFF732FB00283FF470AF8BE79E
:10DD3000FFF7A8FBF8E72046FFF71AFFF4E7FFF725
:10DD400033FBF1E7FFF7DEFBEEE7FFF735FBEBE731
:10DD5000BDE83840FFF746BBFFF74CFBE4E7FFF7B1
:10DD6000FFFBE1E7FFF712FCDEE7FFF719FCDBE75B
:10DD7000FFF728FCD8E7FFF753FBD5E7FFF776FB63
:10DD8000D2E700BF3880003004A1003018E2130849
:10DD90005100200090F8DC32032B0BD0062B06D06C
:10DDA000012B0AD1C368186803681B681847044828
:10DDB00002F004BA034805F03FB80020704700BFE6
:10DDC0003CA700309CA8003030B590F8203385B0D7
:10DDD0000446F3B1684614F04BFF694641480DF024
:10DDE00099F950B104F13C0031F022FC002304F514
:10DDF000207084F820332FF03BF894F8DC320B2BA2
:10DE00002DD8DFE803F029484C504854585C606432
:10DE1000586800F5207004F13C052FF029F890B106
:10DE200094F84030012B0ED194F8DC32012B0AD14A
:10DE3000284631F057FA50B12046FDF7FFF92A4A3B
:10DE4000022163F097FA284631F07EFAD5E72046A2
:10DE5000FDF7F4F9254AF3E72046FEF7EBF994F8CD
:10DE60002133002B3BD094F84430C3BB94F84020BE
:10DE7000022A34D084F821331D4CD4F8E001036821
:10DE80001B6898472D220146A4F5117005B0BDE826
:10DE9000304060F067BD2046FEF7E0F9DFE720463E
:10DEA000FEF71AFADBE72046FEF72EFAD7E7204600
:10DEB000FEF730FAD3E70F4803F032FCCFE72046F5
:10DEC000FEF75EFACBE72046FEF798FAC7E7204652
:10DED000FEF728FCC3E72046FEF75EFBBFE705B070
:10DEE00030BD00BFD04B003034E213085CE21308B1
:10DEF000388000303CA700307047000070470000B9
:10DF00007047000090F8210080F001007047000089
:10DF1000024B436040F60403038170470001020591
:10DF200090F86001704700000F2070470020704794
:10DF3000002070470020704700207047004870475D
:10DF40001CE313080048704728E3130810B50A4C77
:10DF500004F580432046D3F8B43DB3F9083000EE11
:10DF6000103AB8EEC00AF4F7C7FC04F5E840BDE883
:10DF70001040FCF70BBE00BF3830003070B5184CB5
:10DF80001D4604F5405304F5E8462DED028BB3F928
:10DF9000343582B008EE103A04F5C04304F58044ED
:10DFA000D3F8840CB8EEC88A0368CDE900211B6D54
:10DFB00098473046F0EE400AB0EE480ADDE900210D
:10DFC000FCF7CEF9D4F8B80D6CF02EFD3046FCF716
:10DFD00059FE85ED000A02B0BDEC028B70BD00BF9A
:10DFE00038300030F8B51C4D05F5405405F5C046F5
:10DFF0002846D6F8887CF4F76BFCB4F9703501EE4E
:10E00000103AB4F96E3500EE903A4342B8EEC11AB8
:10E01000384600EE103AF8EEE00AB8EEC00A99F081
:10E020005DF82846D6F8886CF4F752FCB4F97035E0
:10E0300001EE103AB4F96E3500EE903A4342B8EE74
:10E04000C11A304600EE103AF8EEE00AB8EEC00A07
:10E05000BDE8F84099F0B8B83830003038B5124D06
:10E06000124CD5F8840C03689B689847642100F132
:10E070008C02204660F0A4F8D5F8840C0368DB68B5
:10E080009847652100F18C02204660F099F8D5F898
:10E09000840C03681B699847662100F18C022046B6
:10E0A000BDE8384060F08CB838900030F47D003026
:10E0B000014808F0EDBF00BF383000303C30ACF014
:10E0C000EFBC000008B55FF083FA62224FF48011C4
:10E0D000BDE808405FF032BA08B55FF079FA562221
:10E0E0004FF48011BDE808405FF028BA08B55FF032
:10E0F0006FFA6F224FF48011BDE808405FF01EBA3E
:10E1000073B51F4D0646D5F8E00103681B6B9847B1
:10E11000044680B395F9D531002B2FDBD5F80432B6
:10E1200093F8D1403CB395F8D43103F0A003202BF1
:10E1300024D1D5F8E00103681B689847052808D06A
:10E14000D5F8E00103681B689847A0F110035C4212
:10E150005C410C4A2146304602F668430193A2F521
:10E160000053D3F82C3F0093D2F8883CD2F8842C8B
:10E17000ACF046FC0446204602B070BD0024FAE72D
:10E1800038800030389000303C30FFF7B9BF0000D5
:10E190003C30AAF0E7BE0000002380F8473080F84A
:10E1A000623070477FB5234D04462348F4F7BAFF29
:10E1B00095F9D431002B36DA23682046DB6898477E
:10E1C000B5EEC00AD5F804021C4DF1EE10FA4CBFB2
:10E1D000012102219EF076FED5F8840C96F032FBE8
:10E1E000D5F8840C012197F033F8236802AA01A91D
:10E1F0001E69204603ABB047D5F8840C9DED031A89
:10E200000368DDED020ADB699DED010A98479FED89
:10E210000C0AD5F8880C9AF071F9D5F8880C9AF0A8
:10E22000C5F904B070BD204604B0BDE87040ACF044
:10E23000FDBE00BF388000303830003038900030EC
:10E24000000000003C30FFF7ADBF00000120704728
:10E25000012070470120704713207047012070474C
:10E260000020704700207047012070470048704729
:10E2700050E41308004870475CE413080F4B30B5B6
:10E280000446D3F8E00185B0036803911B68984702
:10E2900013284FF0000303990DD10125DFED080A83
:10E2A00020461A46B0EE600ACDE9003502F03EFB8A
:10E2B000284605B030BD1846FBE700BF3880003067
:10E2C0000000000002F004B903F02ABA11207047E0
:10E2D00001207047002070470020704700207047E1
:10E2E00000487047F0E4130800487047F8E413084A
:10E2F00038B54369044680691D689DF01DFE2EF007
:10E30000C3F9DFED1B0A284698F05AFD6369A0693E
:10E310001D689DF011FE2EF0B7F9DFED150A2846B5
:10E3200098F0C4FD6369186899F07CFE6369DFEDBD
:10E33000110A1868B0EE600A9FED0D1A98F0CEFE33
:10E340006369DFED0C0A1868B0EE600A9FED081AE9
:10E3500098F03AFF6369186898F0F0FF18B963699C
:10E3600018689AF02DF800230120236438BD00BFFF
:10E3700000803B4400007A4370B52DED028B88B0DD
:10E380000446FCF7C3F870B120460021FCF7F6F80C
:10E3900063699FED310A186808B0BDEC028BBDE8D7
:10E3A00070409AF0ABB8636A022118689EF08AFD4B
:10E3B0002A4B93F8D5315B0603D56369186898F04A
:10E3C0007DFD9FED258A03AA606901A901238DEDDA
:10E3D000018A8DED028A8DED038A8DED048A006835
:10E3E00098F0B4FD6369186899F034FF236A1D68DA
:10E3F0002B68DE6B6369186899F058F8012205A94B
:10E40000CDED060A8DED071A28468DED050AB0EE12
:10E41000480AB0476369B0EE480A186898F046FFAA
:10E42000636918689AF0C2F8236C8BB1B1F0A4FE4E
:10E43000E36BC01A236C98420AD30C2205210848CA
:10E44000FCF770FA20B90C2202210548FCF76AFAA1
:10E4500008B0BDEC028B70BD0000000038800030B9
:10E460003830003038B504460D46B1F085FEC4E9B9
:10E470000F0538BD07207047012070470020704706
:10E480000020704701207047004870478CE5130852
:10E490000048704794E5130838B5002304462DED75
:10E4A000028B80F83C30C368DFED318A1B6842691B
:10E4B000D3ED0A0A9FED2F8AF4EEE80A93ED060ADF
:10E4C0001068F1EE10FA60FE880A98F079FCE368B3
:10E4D00062691B681068D3ED0A0A93ED060AF4EE30
:10E4E000E80AF1EE10FA60FE880A98F0DFFC636932
:10E4F00020461D68FCF7A6FE6368B3F93820B3F91F
:10E50000363001EE102A00EE903A4342B8EEC11ABE
:10E51000284600EE103AF8EEE00AB8EEC00A98F08D
:10E52000DDFD636920461D68FCF78CFE6368B3F966
:10E530003820B3F9363001EE102A00EE903A43420B
:10E54000B8EEC11A284600EE103AF8EEE00AB8EE2E
:10E55000C00A98F039FE084BD3F8940C9BF072FD7A
:10E5600006480821F8F7D6FB0120BDEC028B38BD28
:10E570000000003400007A43389000300CAD0030C9
:10E5800030B52DED048BC36804469FED888A89B0B1
:10E590001B684269D3ED0A7ADFED850AF4EEC87A8A
:10E5A00093ED060A1068F1EE10FA67FEA00A98F0E3
:10E5B00007FC636920461D68FCF744FE6368B3F9F5
:10E5C0003820B3F9363001EE102A00EE903A43427B
:10E5D0002846784D00EE103AB8EEC11AF8EEE00A7F
:10E5E000B8EEC00A98F07AFDD5F8940C9BF08AFE3C
:10E5F000A5F5805393F8F931D90747D4D5F8943C61
:10E600001A8BD20742D593ED0E9AB4EEC89AF1EE6A
:10E6100010FAB8BF93ED049AE36AF0EE498A1868DD
:10E620006CF002FAD5F88C3CD3ED067AA36B20EEA1
:10E63000270AD3ED007AE0EE278AB0EE490AF5EE1C
:10E64000C08AF1EE10FAD8BFDFED5B8AF0EE680AFF
:10E6500027F0B6FF28B9B0EE680AD5F8940C9BF005
:10E6600075FB636893F95130272B0FD0A36A1868A4
:10E670006CF0DAF9F0EEC07AB0EE407AF4EEC87AD7
:10E68000F1EE10FA20D5002384F83C30236B2046AD
:10E690001B68B3F9083000EE103AB8EEC00AFCF778
:10E6A0001DFB2046FCF772FA2046B0EE408AFBF7CD
:10E6B0002DFF002847D00021204609B0BDEC048B77
:10E6C000BDE83040FBF75ABFD5F8943C9FED3B0ABC
:10E6D000D3ED0F6AD3ED137AF4EEC86AA36B27EE7D
:10E6E000800AD3ED007AF1EE10FA67EE277A10DB9C
:10E6F00045209FED331ADFED300A37EE800A28F00F
:10E70000C5F8012384F83C30D5F8940C9BF00EFB3F
:10E71000BCE79FED2C7AF4EEC76AF1EE10FA05D84B
:10E7200049209FED251ADFED280AE6E7F0EEE66ABC
:10E73000F4EEC86AF1EE10FAE3D594F83C30002B01
:10E7400007FE800ADDE7636A022118689EF0BAFBC3
:10E750001E4808F00FFBB0EE480AD5F8940C9BF069
:10E76000BFFC01461A48FAF7E5FC6369186899F09E
:10E770001DFF236A1D68636905AC186898F096FE52
:10E78000204614498DED020ACDED030A8DED041AE1
:10E79000F8F7E8FC079B02A92846009394E80C00D0
:10E7A00096F080F809B0BDEC048B30BD0000003459
:10E7B00000007A433890003000000000E02E6542EF
:10E7C0000000B442000000B40000B4C2F87E003083
:10E7D000383000300CAD0030144B10B5D3F8943CF9
:10E7E00088B0DC68A0689DF0A1FB90ED017A90ED07
:10E7F000006A6946B7EEC77A04F52270B7EEC66ABA
:10E800008DED027B8DED006B2BF03EFE04A88DEDAF
:10E81000040B8DED061B2BF065FEB7EEC00BFCEE76
:10E82000C07A17EE900A08B010BD00BF38900030D3
:10E83000024BD3F8943CD86898F0E6BE389000308C
:10E840000B2070470120704700207047012070475F
:10E85000002070470048704728E6130800487047BA
:10E8600030E6130801207047DFED237AF4EEE70A63
:10E8700008B5F1EE10FA2DED028BF0EE408AB0EE05
:10E88000608A35DDDFED1D7AF4EEE70AF1EE10FA6D
:10E890002ED5F6EE007ADFED1A6A9FED1A0AB7EE72
:10E8A000001A872070EEE77ADFED170AF0EEE77ABC
:10E8B00087EEA67A30EE470A27F0E8FFDFED137AFD
:10E8C0008A209FED131A20EE270ADFED120A20EEB0
:10E8D000280A27F0DBFF30EE080A8D20B7EE001A79
:10E8E000DFED090ABDEC028BBDE8084027F0CEBF82
:10E8F0009FED050AEFE700BFAC1C5A3ED578493FB3
:10E900008FC2753E9A99993F00000000FAEDEBBA6C
:10E910009A99993E9A9999BE7E4B30B52DED048B0C
:10E92000B3F9343583B0044600EE903A01AA694643
:10E93000F8EEE00AB0EE600AFBF712FDA0699DF068
:10E94000FBFAE369D0ED008A0546D3EDEE6AD3ED1C
:10E95000F17A90ED016A3B2027EEE80AA36868EEA1
:10E96000A68A9FED6D1A03F5BA53DFED6C0AA6EE89
:10E97000260AE6EE278ADFED6A7AB0EEE87AB4EE90
:10E98000E77AF1EE10FA58BFB0EE677ADFED657AFC
:10E99000C7EE275A9DED007AF7EE007A77EEE57A1A
:10E9A00067EE877A93ED077A67EE877A9FED5E7A56
:10E9B00087EE879A27F06AFF3C209FED571ADFED1C
:10E9C000570AB0EE408AB0EE680A27F05FFF626B2C
:10E9D000DFED567AF0EE408A1268BAEE000A544B28
:10E9E0004520B2F90820D3ED006A07EE102A9FED0A
:10E9F000511ADFED510AB8EEC77A27EE277ADFED1C
:10EA00004F7AA6EEA77AF4EE007AA7EE678A83ED36
:10EA1000007A28EE000A8DED000A27F037FFDDEDC1
:10EA2000017A9FED477AF0EEE77A464B8DED000ACA
:10EA3000F4EEC77AF1EE10FA51D593ED007ADFEDDE
:10EA4000427A77EE277AB2EE007AF4EEC77AF1EEE8
:10EA500010FA58BFF0EE477AC3ED007A67EEA87A55
:10EA6000CDED017A636A186890F8D110002939D188
:10EA70009EF028FA636A1B6893F8A910012939D01F
:10EA8000032940D039B9236A186896F0E1FB236A5C
:10EA9000186895F0C1FE236AB0EE491ADDED010A4F
:10EAA00018689DED000A0368DB69984795ED028AB6
:10EAB0002046FBF7D9FE2046F0EE400AB0EE480AA9
:10EAC000FFF7D2FE236A626801211868D2ED020ABC
:10EAD0000368DB6C984703B0BDEC048B30BD0022AB
:10EAE0001A60BFE7194B93F9D531002BB4BF012150
:10EAF0000221BDE7236A186896F0AAFB236A18680A
:10EB000095F0A0FEC7E7D9790029C4D12046FCF7CB
:10EB10008FFBC0E73860003000000C4400000CC4DC
:10EB20000000FA4400409C45000034420AD7233DCF
:10EB30005CAD003000A08C4500A08CC58FC2753F35
:10EB40000000003460AD00308FC2F53C38800030EA
:10EB50000E2070470020704700207047002070474B
:10EB60000020704700487047C4E61308004870470B
:10EB7000C4E6130870B52DED028B436A04461B688A
:10EB800093F8D130FBB9052384F848302046FBF7D1
:10EB90006BFE636A0221B0EE408A18689EF092F91B
:10EBA00094F95030E2696BB3D2F86C535D4394F83A
:10EBB0004820052A4FD8DFE812F02B005F008300C1
:10EBC000B000DD001C01836A1B68B3F90830002B1C
:10EBD000B8BF5B429BB2B3F57A6FD4D2C36A1B68ED
:10EBE000B3F90830002BB8BF5B429BB2B3F57A6F24
:10EBF000C9D2B1F0C1FAE36CC01A40F6C41398420E
:10EC0000C1D8C3E794F95150D2F870235543CEE7E9
:10EC1000226A94F95110106849F640429FED7E1A1D
:10EC200053435143026800EE103A00EE901AD26A44
:10EC3000B8EEC00AF8EEE00A904741F29313DFED18
:10EC4000777A9D4238EE278A05DD94F950308BB1F2
:10EC5000012384F84830236AB0EE480A6268002134
:10EC60001868D2ED020A0368BDEC028BDB6CBDE8CC
:10EC7000704018470223ECE7226A05F50C559FED1A
:10EC8000661A106849F64042F0EE410A27355343B0
:10EC9000026800EE103AD26AB8EEC00A9047DFED83
:10ECA000607A43F2BA4338EE678AB5EEC08AF1EE75
:10ECB00010FAD8BF9FED588A9D42CCD80423C8E7EC
:10ECC000236A49F640429FED541A186894F951306E
:10ECD000B0EE410A5343026800EE903AD26AF8EE71
:10ECE000E00A9047DFED4E7AE36942F2283238EECF
:10ECF000678AD3F86C33B5EEC08AF1EE10FAD8BF4C
:10ED00009FED458A002BB8BF5B429342A3DD41F2E1
:10ED100094139D429FDD03239BE7236A49F64042FB
:10ED20009FED3D1A186894F95130B0EE410A5343F3
:10ED3000026800EE903AD26AF8EEE00A9047DFED02
:10ED4000387AE36944F24E6238EE678AD3F86C335E
:10ED5000B5EEC08A03F50C532733F1EE10FAD8BF95
:10ED60009FED2D8A93423FF676AF2E4B9D42FFF6E4
:10ED700072AFA3E7236A002194ED111A1868D4ED4D
:10ED8000100A036894ED0F0A1B6A9847DFED237A97
:10ED900094F9502038EE278AE3691AB393EDDB7AB1
:10EDA000D4ED0F7AB8EEC77A77EEC77A9FED1E7A68
:10EDB000F0EEE77AF4EEC77AF1EE10FA3FF64BAFD9
:10EDC0000D2294F849101948FBF7ACFD024618B91A
:10EDD00001461648FBF7A6FD60F076FA162160F0B2
:10EDE000BBF938E793EDDC7AD4ED107AB8EEC77A48
:10EDF000DAE70D2294F849100C48FBF793FD024620
:10EE000018B901460948FBF78DFD60F05DFA022252
:10EE10000D2160F0C1F91EE700000000CDCC4C3E92
:10EE20008FC2753E6DEEFFFF0000FA4338300030B0
:10EE300073B5474D0446D5F8E00103685B6B98470E
:10EE400018B90026304602B070BD95F9D531002BB7
:10EE50005FDBA36A1B68B3F90830002BB8BF5B42C5
:10EE60009BB2B3F57A6FECD2636A1B6893F8D160FA
:10EE7000002EE6D095F9D431002BE2DBD5F8E00185
:10EE8000002503681B68984784F8485084F84900B7
:10EE9000B1F072F9E36AE064A4F850501B68B3F96A
:10EEA0000830B3F5967F43DD012384F8513060F0DC
:10EEB0000BFA152160F050F9264B5320B3F9343585
:10EEC00001EE103AE369B8EEC11A93EDDB0AB8EE31
:10EED000C00AF1EE410A8DED011ACDED000A27F0CE
:10EEE000D5FCE369542084ED0F0A93EDDC0A9DED17
:10EEF000011AB8EEC00ADDED000A27F0C7FCE3698D
:10EF000084ED100AD3EDDD7AF8EEE77AC4ED117ADC
:10EF100098E7D5F8E00103681B689847012890D06E
:10EF2000D5F8E00103681B689847002891D188E76D
:10EF300013F5967F01DAFF23B7E7A36A1B68B3F9DD
:10EF40000830002BACBF0123FF2384F85030AEE71C
:10EF5000388000303860003016207047002070473D
:10EF600000207047012070470020704781F00100A9
:10EF700070470000012070470048704758E71308A9
:10EF8000004870476CC7130803681BB1007900F094
:10EF90000100704718467047F7B5474D044695F98C
:10EFA0006D6FA5F58045002E00F082804348FFF785
:10EFB000EBFF064600287BD0636920461F68FCF7FC
:10EFC00041F96368B3F93820B3F9363001EE102AFD
:10EFD00000EE903A4342B8EEC11A384600EE103ABD
:10EFE000F8EEE00AB8EEC00A98F078F863692046B7
:10EFF0001F68FCF727F96368B3F93820B3F9363096
:10F0000001EE102A00EE903A4342B8EEC11A38469B
:10F0100000EE103AF8EEE00AB8EEC00A98F0D4F824
:10F0200005F5C043D3F8880C98F088F918B96369DE
:10F03000186899F0C5F9B5F95C3204F13C001BB9C8
:10F04000B5F85A32A5F85C32B5F85C320027D4ED39
:10F05000260A00EE103AB8EE400A61F0E3FC04F133
:10F060005C00C4F8A070019086F0B8FC0023019801
:10F0700084F8A530B5F95C321BB9B5F85A32A5F859
:10F080005C32B5F85C32B7EE000A07EE903AF8EE63
:10F09000E77A80EE270A86F0C5FC09489CF048FF15
:10F0A000DFED087AC4F8C87020EE270A84ED310A33
:10F0B000304603B0F0BD00BF38700030A07F003094
:10F0C000A09C00300AD7233C10B50446FBF728F873
:10F0D000154B204640F83C3B61F098FC134BF1EE99
:10F0E000041A9FED132A236504F15C00114B9FED78
:10F0F000121ADFED120A9FED120A636586F0A6FC74
:10F10000002320460F49C4F8A830C4F8AC30C4F836
:10F11000B030C4F8B430C4F8B830C4F8BC3055F0DE
:10F120007FFF204610BD00BF6CE81308CDCCCC3D5E
:10F130000AD7233B0000404000803B459A99993E06
:10F14000CDCC4C3E04E813082DE9F0432DED028BA5
:10F150009BB0914604460D46B1F00EF8B9490646FB
:10F1600004F15C07A1F108004FF000082AF0E0FD6F
:10F1700094ED161AF0EE608A7E20F1EE410A27F037
:10F1800085FB94ED161AB0EE408A7F20F1EE410A1D
:10F19000B0EE680A27F07AFBF0EE400A8DED110A16
:10F1A000B0EE480A04F13C008DED108A61F054FC89
:10F1B000A548CDED130A9FEDA58A8DED120A9CF0AE
:10F1C000B7FED4ED327A8920D4ED140AE0EE087A45
:10F1D00094ED151AB0EE670A27F058FB12A82AF032
:10F1E000F3FD12A99A480CF0D1FD14A938468DED13
:10F1F000140ACDED150A86F0D3FA3846CDF85880BA
:10F20000CDF85C8086F00EFB8DED160ACDED170A69
:10F21000B9F1000F00F001810123C4F8D06084F837
:10F22000CC308C4E04F1A80116A82AF0A9FDB6F93D
:10F23000343516A800EE103AB8EEC00A2AF0C4FD24
:10F2400016A983480CF08EFD18A928468DED180AE2
:10F25000CDED190A2AF094FDB6F9343595ED007A12
:10F2600007EE903AB0EEC77AF8EEE77AB4EEE77AB6
:10F27000F1EE10FA00F3CF8095ED017AB0EEC77A87
:10F28000F4EEC77AF1EE10FA4CBF0123002384F8A4
:10F29000A530CA20B6F9343595ED000A5A4207EE7A
